S00A000047572E737265637C
S214400000A55AA55A0100000000000000001040005C
S21440100000F042202114440075604500776045009A
S214401010796045007B6045007D604500000000002B
S2144010200000000000000000000000007F60450057
S214401030B360450000000000B5604500B76045005D
S21444010047573334342056302E322E352032303250
S214440110332E31312E362031323A30300A0D00003B
S20C4401803412AA5500000000E9
S214440200A55AA55A01000000000000000010440052
S2144402100000000000104400000000000000000041
S2144402200000000000000000000000000000000085
S2144402300000000000000000000000000000000075
S2144402400000000000000000000000000000000065
S2144402500000000000000000000000000000000055
S21444100000F0422021144400756045007760450096
S214441010796045007B6045007D6045000000000027
S2144410200000000000000000000000007F60450053
S214441030B360450000000000B5604500B760450059
S214441040B9604500B9604500B9604500B9604500DF
S214441050B9604500B9604500B9604500B9604500CF
S214441060B9604500B9604500B9604500B9604500BF
S214441070B9604500B9604500B9604500B9604500AF
S214441400B9604500B960450000BF00BF00BF00BFDB
S214441410FFF7FABF000000000000000000000000D4
S21444142072B64FF000004FF000014FF000024FF04C
S21444143000034FF000044FF000054FF000064FF055
S21444144000074F4801684FF0807201EA0201002904
S2144414501CD14C4801684FF0807241EA0201016099
S214441460494801684FF0010241EA020101604748D9
S21444147045F6F02101604AF20F5101604048016888
S2144414804FF0807201EA02010029F7D040484149F2
S2144414900160414801684FF00000814200D003E0FB
S2144414A03E4880F3088803E03D4880F3088822E0FD
S2144414B03C484CF2205101604DF6281101603A48F0
S2144414C03A4901600AE03A484CF2205101604DF630
S2144414D028110160374835490160FFE7364800283F
S2144414E009D03649364A521A013A04DD0020002310
S2144414F009C1083AFCDA3348002810D03249086853
S2144415004FF0010240EA020008603049304A521A5D
S214441510013A04DD0020002309C1083AFCDA2D48CC
S214441520002810D02C4908684FF0010240EA020017
S21444153008602A492A4A521A013A04DD0020002348
S21444154009C1083AFCDA274800684FF05A31884205
S214441550F9D0114801684FF00000814200D001E004
S21444156014F0ACFD14F0D6FD62B614F0D1FD00F0D4
S2144415703BF800BFFEE700BFAFF30080AFF3008048
S21444158010C32D4030C32D4004C32D4000C02D4011
S21444159008ED00E0001043200400264000F04220FE
S2144415A0000043201000274000002740400000FF72
S2144415B010C0464000C046400100000000004020E5
S2144415C0004044200100000094EF00E000000020AA
S2144415D0000001200100000090EF00E00000000041
S2144415E000800000002540202DE9F04F87B05B4C7A
S2144415F001F060FC5A4816F0AFFA5A494E200025CE
S21444160026F05AFC58481DF037FC58481DF058FC44
S21444161001F0C3FB4CF24453E05800F021F901F0CA
S214441620FFFD00F045FA00F021FA00F09FF950491A
S214441630002020F09DFD4F49002020F0AFFD002102
S214441640084620F055FE002144F62062084620F065
S2144416500BFE2846013501F05DFF062DF9D101F059
S21444166099FB4CF23853444D4FF47A7054F8038047
S214441670E75805F1040BE25854F803900592E258F3
S2144416800292E2580392E2580492E25854F803A0B5
S214441690E6582C46019201F044FB08F0E1F937483D
S2144416A001F070FC00F0B4F82A6806F57A739A42A2
S2144416B002D32E6808F0C1F922680AF1C8039A4298
S2144416C003D3D4F800A008F0B1F9019B2268643330
S2144416D09A4203D32368019308F095F9049B226841
S2144416E032339A4201D323680493039B226814330B
S2144416F09A4203D32368039303F09AFB029B22681F
S2144417000A339A4203D32368029308F040F92268C6
S21444171009F105039A4203D3D4F8009008F0B5F8CB
S214441720059B226802339A4203D32368059300F04C
S21444173070F822687B1C9A4200D32768DBF80020A6
S21444174008F101039A4203D3DBF8008008F04AF913
S21444175008F08CF90DF034FFA6E700BF744841202A
S214441760B8994600E8034020FCA646002CA2460052
S2144417707417402068174020AC0D42201C90460049
S214441780024B586800F00300704700BF0000264034
S214441790024600F03F00931010B583EA5203540803
S2144417A0534084EA121483EA121384EAD2049B0157
S2144417B084EA521403F0400314F0010F43EA000392
S2144417C00CBF80240024234319B99A4218BFFF2033
S2144417D010BD01290CBF1846FF20F9E73C2A0CD05F
S2144417E07D2A0AD0FE2A08D0BF2A06D092B20144E7
S2144417F0814204D1D043C0B270470022F7E710F8C4
S214441800013B1A4492B2FF2A84BFFF3A92B2EFE7F2
S21444181070470BF071BF704710B50C4C002001F0B8
S214441820E3F92080012001F0DFF9094B2288188073
S214441830084B1A800BF03DF90BF05EF90BF080F97B
S2144418400BF0A2F9BDE810400BF0C2B95A1840207C
S2144418505818402004184020704770477047704717
S214441860002110B50446084619F030FB012100203B
S21444187019F02CFB0221002019F028FB032100203C
S21444188019F024FB002019F01DFA0E49002019F027
S2144418902FF90D4BA2B20020197819F067FA0B49BC
S2144418A0002019F0D9FD0A49002019F0D5FD094950
S2144418B0002019F0D1FD08490020BDE8104019F079
S2144418C0CBBD00BF749E4600AC9E4600FC9F4600BF
S2144418D0DC9F4600BC9F46009C9F4600F8B50D46DC
S2144418E006461F4928461F4F0FF0BEF8044670B1FF
S2144418F04CF24453F85806F54553123307EB830726
S2144419007D60032E2BD8DFE806F01A212427002119
S21444191028460FF09FF880B94CF24453F8580EF01E
S21444192099FE29460EF0EEFE0EF03EFA00220E4BCD
S2144419300EF0BCFB0EF068FDDDE72046DBE782B226
S21444194000210020BDE8F84019F0D0BF82B2012142
S214441950F7E782B20221F4E782B20321F1E7F8BD49
S2144419600000C842744841200000594008B5034866
S2144419701EF074FC024B187008BD00BFF4A9460064
S214441980D4474020F7B50123104C114D6370A21C78
S214441990EB68A91C0F480235009335F8023C1EF04C
S2144419A0FFFA00222073A01C6178134615F8017BC9
S2144419B0013310F8016BDBB2B7421CBF0122002191
S2144419C00A2BF3D102B1617003B0F0BDD447402076
S2144419D0A81F402008AA46004B7C062B0AD10122A9
S2144419E0054B1A74CA7B1A2A04D1032203F1110147
S2144419F01EF016BE704700BFA81F40204B7C062B27
S214441A000AD10122054B1A74CA7B2A2A04D103221E
S214441A1003F111011EF004BE704700BFA81F40200A
S214441A201FB500231A210446039301238DF807307B
S214441A301EF03CFF0B4B03930B4B1A7C002AFCD046
S214441A401B7C63B102A920461EF034FE8DF80700C5
S214441A50039B5A1E039213B19DF80730F1E704B076
S214441A6010BD00BF006A1800A81F402008B5A1207A
S214441A701DF048FA00220A49A1201DF042FA094BFB
S214441A80094902220120C3F8F413C3F8982DC3F879
S214441A90F813C3F8902D0549BDE808401DF032BF41
S214441AA0FBFC4500000029400400280068A94600C5
S214441AB008B5A2201DF026FA00220B49A2201DF0EC
S214441AC020FA0A4B0A4A01210020C3F8E023C3F84F
S214441AD0AC1DC3F8E42302220649C3F8A42DBDE88E
S214441AE008401DF04FBC00BF01FD450000002940E2
S214441AF0020028008CA9460010B508221749012088
S214441B004FF480341DF0BAFF012308221449002004
S214441B101DF024FD002108461DF06EFE022801D16A
S214441B20013CF7D14FF48034002101201DF0B0FF72
S214441B30022801D1013CF7D1094A0823A2F1080042
S214441B4012F8011B013B10F8014BA14204BF0131BE
S214441B5002F8011C13F0FF03F2D110BDBC1F402055
S214441B60C41F402082B00190019B5A1E0192002B54
S214441B70FAD102B07047044B4FF400224FF4FA7087
S214441B80C3F8C022FFF7EEBF00002940044B4FF4D1
S214441B9020124FF4FA70C3F8C022FFF7E3BF00BF29
S214441BA0000029402DE9F04104460D461046002920
S214441BB03ED1DFF8908050260B46C1B2564308F11A
S214441BC010072846BA19B0441AF0A0FE1C484FF431
S214441BD0FB534FF4FB62D8F81410083603FB040397
S214441BE03744D3F8FC3802FB043203F17A0602F594
S214441BF0107C02F5427240F82C1098F8581040F8C1
S214441C002210FB2212FB046200EB4212A94211D8B6
S214441C104FF4FB520133642102FB0404B3FBF1F29C
S214441C2001FB1233C4F8FC3804F521540123236025
S214441C30BDE8F08117F8016B013502F8016BE5E762
S214441C4074484120D44740202DE9F04104460D46CF
S214441C50104600293ED1DFF8908050260B46C1B28C
S214441C60564308F521670120BA19B0441AF04EFECF
S214441C701C484FF4FB534FF4FB62D8F8141A08364A
S214441C8003FB04033744D3F8FC3802FB043203F165
S214441C907A0602F5107C02F5427240F82C1098F849
S214441CA0581A40F82210FB2212FB046200EB421240
S214441CB0A94211D84FF4FB520133642102FB0404B9
S214441CC0B3FBF1F201FB1233C4F8FC3804F521549B
S214441CD001232360BDE8F08117F8016B013502F853
S214441CE0016BE5E774484120D44740202DE9F04194
S214441CF004460D46104600293ED1DFF89080502613
S214441D000B46C1B2564308F546770220BA19B0448A
S214441D101AF0FCFD1C484FF4FB534FF4FB62D8F812
S214441D201C13083603FB04033744D3F8FC3802FB81
S214441D30043203F17A0602F5107C02F5427240F84A
S214441D402C1098F8601340F82210FB2212FB046211
S214441D5000EB4212A94211D84FF4FB5201336421DE
S214441D6002FB0404B3FBF1F201FB1233C4F8FC3863
S214441D7004F5215401232360BDE8F08117F8016B74
S214441D80013502F8016BE5E774484120CC58402001
S214441D902DE9F04104460D46104600293ED1DFF8B1
S214441DA0908050260B46C1B2564308F61857032077
S214441DB0BA19B0441AF0AAFD1C484FF4FB534FF42A
S214441DC0FB62D8F81C1D083603FB04033744D3F8DB
S214441DD0FC3802FB043203F17A0602F5107C02F565
S214441DE0427240F82C1098F8601D40F82210FB22EE
S214441DF012FB046200EB4212A94211D84FF4FB5284
S214441E000133642102FB0404B3FBF1F201FB1233F9
S214441E10C4F8FC3804F5215401232360BDE8F0815E
S214441E2017F8016B013502F8016BE5E77448412069
S214441E30CC5840202DE9F04104460D461046002972
S214441E403ED1DFF8908050260B46C1B2564308F583
S214441E50C4670420BA19B0441AF058FD1C484FF41D
S214441E60FB534FF4FB62D8F82416083603FB0403EE
S214441E703744D3F8FC3802FB043203F17A0602F501
S214441E80107C02F5427240F82C1098F8681640F818
S214441E902210FB2212FB046200EB4212A94211D824
S214441EA04FF4FB520133642102FB0404B3FBF1F20A
S214441EB001FB1233C4F8FC3804F521540123236093
S214441EC0BDE8F08117F8016B013502F8016BE5E7D0
S214441ED074484120C46940202DE9F04104460D462B
S214441EE0104600293ED1DFF8908050260B46C1B2FA
S214441EF05643A8F1D8070520BA19B0441AF006FD8F
S214441F001C484FF4FB534FF4FB6258F8D41C083675
S214441F1003FB04033744D3F8FC3802FB043203F1D2
S214441F207A0602F5107C02F5427240F82C1018F836
S214441F30901C40F82210FB2212FB046200EB421273
S214441F40A94211D84FF4FB520133642102FB040426
S214441F50B3FBF1F201FB1233C4F8FC3804F5215408
S214441F6001232360BDE8F08117F8016B013502F8C0
S214441F70016BE5E774484120BC7A40204FF4FB529D
S214441F80054B02FB0033D3F8F808D3F8FC38C31AE1
S214441F9058425841704700BF744841202DE9F74FD6
S214441FA0D14D0021D14E4FF4FB692C4641F698782A
S214441FB037464FF0640A0846FFF7E0FF58BBD6F8AA
S214441FC0F83809FB013202F5427257F822C008FB82
S214441FD0014200924FF4FB524A4302EB43123A4406
S214441FE0019200F1010EC0B2844500F2A88009FBBC
S214441FF00132013385F820C002F5107257F82220CA
S2144420006A624FF0010285F82120B3FBFAF20AFB1C
S2144420101233C6F8F8380131454406F5FB5606290E
S214442020C9D194F82130012B19D1002384F82130EA
S214442030636AB3F5407F00F0CF8000F29F80B3F52B
S214442040BA7F00F0D28000F28B80422B00F0D98019
S2144420507FD8402B00F0C380412B00F0C38041F66C
S214442060B973E25C012A0FD10022E25441F6BC73F4
S214442070E358932B00F0D68000F2C680912B00F0F4
S214442080CB80922B00F0CB8043F65173E25C012A5E
S21444209014D10022E25443F65473E358962B00F0CE
S2144420A0E98000F2CA80822B00F0E18000F2BD8015
S2144420B0722B00F0E580732B00F0E58045F6E9636B
S2144420C0E25C012A14D10022E25445F6EC63E3585C
S2144420D09B2B00F0F98000F2E4808D2B00F0088101
S2144420E000F2D780722B00F0F880732B00F0F88053
S2144420F047F68163E25C012A0BD10022E25447F69C
S2144421008463E358722B00F0F980732B01D102F0FC
S214442110ADFD49F61963E25C012A40F0F7800022DF
S214442120E25449F61C63E358722B00F0EA80732BA2
S21444213040F0EC8003B0BDE8F04F02F0C7BD019A12
S21444214002EB000B009A9BF840BF02F800B07046C2
S21444215047E740F25512934281D101F0F9FC7EE7FD
S214442160B3F5BE7F44D040F22122934243D0B3F528
S214442170BC7F7FF474AF01F035FD70E740F28552C2
S214442180934226D00DD8B3F5AE6F19D0B3F5B06FE1
S21444219019D040F2013293427FF461AF01F0E2FD80
S2144421A05DE740F29552934210D040F277729342E4
S2144421B024D0B3F5B26F7FF452AF01F0A1FE4EE7E0
S2144421C001F0DCFD4BE701F029FE48E701F0AAFEEA
S2144421D045E701F06DFE42E701F0A4FD3FE701F05C
S2144421E03CFC3CE701F04CFC39E701F0D9FC36E70F
S2144421F001F01AFD33E701F035FD30E701F0AAFEA1
S2144422002DE701F05FFC2AE740F2511293427FF437
S2144422103BAF01F007FF37E701F0AEFE34E701F0CD
S214442220D1FE31E701F0E0FE2EE78C2B25D0922B31
S2144422307FF444AF02F058F840E7AA2B26D007D8DC
S2144422409A2B0ED0A02B7FF439AF02F06DF935E708
S214442250C82B09D0B3F5F36F7FF430AF02F02EFAF3
S2144422602CE702F021F929E702F0EAF926E701F023
S214442270A9FF23E702F0C0F820E701F0CDFF1DE7F1
S21444228001F026FF1AE701F06BFF17E702F098F912
S21444229014E7932B2FD0972B7FF42AAF02F0FEFA45
S2144422A026E7C92B13D007D8A12B13D0AA2B7FF42B
S2144422B01FAF02F0C3FB1BE740F2997293427FF4D0
S2144422C017AF02F0A1FC13E702F040FB10E702F060
S2144422D0F5FB0DE702F07AFB0AE702F003FA07E79C
S2144422E002F048FA04E700BF608740207448412063
S2144422F002F022FCFCE602F06FFAF9E602F098FCE3
S21444230007E703B0BDE8F04F02F0C2BC03B0BDE837
S214442310F08FEB4BEB4A5969DFF8D0C30A40EA49E1
S2144423202DE9F0475A610022E84D4FF00008E84E88
S2144423304FF000095A6583F86F201A67E54CDFF8BA
S214442340B0E3DFF8B0A3C3E90212197C21F0070119
S2144423501974596A29405962196C01F0004119648C
S214442360596C31405964996C01F0604141F4C8217C
S2144423709964D949C3E91312996D01F0704199657E
S214442380D96D2940D965196E01F000411966B3F834
S214442390641001EA0C01A3F86410B3F8681001EA6B
S2144423A00C01A3F86810596F01F07F415967986F84
S2144423B0CA49D3F89870084083F88C209867D3F8B5
S2144423C0800000F07F40C3F88000D3F8840000F01B
S2144423D07F40C3E92102D3F890002040C3F8900020
S2144423E0D3F8940000F07C40C3F89400BC480740FF
S2144423F0C3F89870D3F89C7007F04047C3F89C70B5
S214442400D3F8A0703740C3E92872D3F8A8700F40B9
S214442410C3F8A870D3F8AC7007F04047C3F8AC7064
S214442420D3F8B47007F04047C3F8B470D3F8B87024
S21444243007F07F47C3F8B870B3F8B07083F8BB2092
S21444244062F30D07A3F8B07093F8BC7027F0030747
S21444245083F8BC70D3F8C070C3F8D4A007F0004724
S214442460C3F8C070D3F8C4700740C3F8C470D3F838
S214442470C87007F07047C3F8C870D3F8CC7007F03C
S2144424807F47C3F8CC70B3F8D07007EA0E07A3F8BA
S214442490D070D3F8D87007F04047C3F8D870D3F854
S2144424A0DC7007F07847C3E9377293F8E47062F358
S2144424B0000783F8E470D3F8E87007F07E4747F4E3
S2144424C08037C3F8E870D3F8EC703740C3F8EC7044
S2144424D0D3F8087107F04047C3F80871D3F80C7175
S2144424E03740C3E94372D3F814710F40C3E940221E
S2144424F0C3E93E89C3F81471D3F81871A3F82821A8
S21444250007F0404783F85421A3F86C21C3F838A158
S214442510C3E9467293F8207127F0030783F82071C5
S214442520D3F8247107F06047C3F82471D3F82C71AC
S21444253007F07047C3F82C71D3F8307107F07F4723
S214442540C3F83071B3F8347107EA0E0ED3F83C7111
S2144425500740A3F834E1C3F83C71D3F8407107F060
S2144425607847C3F84071B3F8447107F47847A3F842
S2144425704471D3F8487107F07E4747F48037C3F870
S2144425804871D3F84C713E40C3F84C61D3F850615F
S21444259006F06046C3F85061D3F868612E40C3E93C
S2144425A05689C3F86861D3F87061A3F874212E4045
S2144425B0C3F8782183F88021C3F87061D3F87C612E
S2144425C083F8E42106F07F46A3F8A021C3F8A421AB
S2144425D0C3F87C61D3F88461A3F8A8212640C3F8E5
S2144425E0AC2183F8B021C6F30747C3F88461C3F827
S2144425F0B42107F0E10683F8B821C3F8BC2183F878
S2144426008661D3F8C46183F8C02106F07C46354F12
S214442610C3F8C461D3F8C8610640C3E97722C3E966
S2144426206222C3E96422C3E96622C3F8C861D3F8C8
S214442630D06183F8942206F00046C3F82C2283F82F
S2144426403022C3F8342283F83822C3F83C2283F875
S2144426504022C3F8442283F82822C3E97462D3F89C
S21444266048620640C3F84862D3F84C623740B3F831
S214442670526206F40046C3F84C72A3F8526293F8CA
S214442680986226F01F0646F0010683F89862B3F86F
S2144426909C6262F30906A3F89C6293F8A06226F053
S2144426A00F0683F8A06293F8A46262F3020683F8E6
S2144426B0A462D3F8206230400B4EC3E988021BE084
S2144426C0E883402000E01FE00000E2810000F0FFC5
S2144426D0000080FF0000FEFF0080204E0000FCFF4C
S2144426E00000C0FFFF0000FE00E0FFFF00C0FFFF49
S2144426F000F0FFFF0000C04B93F8A80262F303000B
S21444270083F8A802D3F8000200F07040C3F8000231
S214442710D3F8080283F8042200F00040A3F8DC2231
S214442720C3F8E022C3F80802B3F80C0200EA0C0C23
S214442730D3F814020540D3F81802A3F80CC2084094
S214442740C3F81802D3F8C4022040C3F8C402D3F82E
S214442750AC0200F07E40C3F8AC02D3F8B00200F0FE
S2144427600040C3F8B00293F8B40220F00F0083F898
S214442770B402D3F8B80200F07840C3F8B802D3F8ED
S214442780BC0200F07F40C3F8BC02B3F8C00230403D
S214442790A3F8C002D3F8D80200F00040C3F8D80229
S2144427A093F8E40262F30000C3E9842583F8E40264
S2144427B0C5F30745D3F8E80262F3071500F07F40F7
S2144427C083F81652C3F8E802D3F8EC02D3F8F4526E
S2144427D0084005F07845C3F8EC02D3F8F802C3F88D
S2144427E0F45200F07840D3F80453C3E9BE0293F899
S2144427F0000305F0784562F30000C3F80453D3F8A9
S214442800085383F80003D3F8F00205F07F4500F040
S2144428104040C3F80853C3F8F002B3F80C03304002
S214442820A3F80C03D3F8100300F07E40C3F810035B
S214442830D3F814032040C3E9C50293F81C0362F39B
S214442840000083F81C03D3F8200300F07F40C3F84D
S2144428502003D3F824030140C3F82413D3F82813E1
S2144428600C40D3F8481301F07841C3F82843C3E931
S214442870B289C3E9D21293F85013C3F8542362F3CF
S2144428800001C3F8642383F85013D3F8401301F0CF
S2144428904041C3F84013D3F8441301F07841C3F8D9
S2144428A0441393F8581362F3000183F85813D3F88B
S2144428B05C1301F07F41C3F85C1393F8621321F074
S2144428C0030183F8621393F8681362F3000193F8E4
S2144428D06E2322F0030283F86813C3E9CC8983F895
S2144428E06E23BDE8F08741F69873084900225843A2
S2144428F00B182830DA64084483F848202023013B28
S21444290000F8012B13F0FF03F9D17047608740208D
S21444291041F6987310B558430B4C41F692732218FF
S214442920D35A28225A4300231118503010442144C5
S2144429301A46204481F870304B67013300F8012B67
S214442940DBB2202BF9D110BD608740202DE9F84337
S2144429509946234B0546884603EB00139B6A402B57
S21444296031D820494FF4FB5303FB001342F644018D
S2144429705B5843B341F698761B4C00274FF0280C1F
S21444298006FB00F3E11801F5FC511031F8B2484556
S2144429901BD328467543FFF7A6FF41F6907160198E
S2144429A028260122435A06FB035513442C4484F834
S2144429B07120C4F8748084F87090C824B3FBF4F291
S2144429C004FB12334352BDE8F883088812F807E044
S2144429D00CFB003020443844013780F850E0D5E7FB
S2144429E0A81F4020744841206087402041F69872D2
S2144429F041F692732DE9F34102FB00F14E4D044635
S214442A006A18D05A282202FB00122A4492F87020F0
S214442A10082A31D8494B082203EB04139A62282328
S214442A2041F6947603FB00F241F6987320466343DE
S214442A30D118EF18503329441344414A2B4402EB2F
S214442A40041200934B6FB95D19F0E8FE012C8046E2
S214442A502FD143F62C711C206B5C0133B3FBF0F290
S214442A6000FB12336B54B8F1000F2BD0B8F1020FB1
S214442A7040D002B0BDE8F081102A04D82F4B102273
S214442A8003EB0413CAE7182A05D82C49182301EB8C
S214442A9004118B62C3E7202A04D82849202301EB7B
S214442AA00411F6E7402ABAD82449402301EB04111E
S214442AB0EFE7BB5D0E210133B3FBF1F201FB1233AA
S214442AC0BB55D0E72046FFF723FF41F6987041F602
S214442AD09271604328242E18735A04FB030401336E
S214442AE0C8202544B3FBF0F200FB123385F871800E
S214442AF07352BEE72046FFF70BFF41F6987041F647
S214442B0092710022444328202E19735A00FB034432
S214442B100133C820254485F87120B3FBF0F200FB4E
S214442B201233064A7352D2E92231013341F100018D
S214442B30C2E922319DE700BF60874020A81F40209D
S214442B40CC1F4020F8B500240A4D41F698760A4F2B
S214442B5006FB04F22821E0B2D35B01FB03232B449B
S214442B6093F87130012B01D1FFF740FF0134062C56
S214442B70EED1F8BD60874020F2A6402008B50B2170
S214442B80034825F0E1F8034B83F8280908BD00BF45
S214442B9002172940BC7A402001290A4628BF012250
S214442BA0072819D8DFE800F004070B0D1012141696
S214442BB000210A4801E00A21094825F08CB80C2176
S214442BC0F7E702210748F8E70D21F2E70E21F0E780
S214442BD00F21EEE70021F5E7704700BF02172940B2
S214442BE0101729400017294007281AD8DFE800F0B4
S214442BF004070B0E1013151708210B4801E00B2190
S214442C000A4825F0A1B801210948FAE70B21F4E760
S214442C1004210848F5E70521FBE70821F9E70A21DE
S214442C20F7E7FF20704700BF0617294002172940E0
S214442C30121729400417294001284FF002010CBFFF
S214442C400022012210B50446034825F044F8034AFE
S214442C504CF24053D45010BD0817294074484120C4
S214442C6005281DD8DFE800F003080C1014180D4A98
S214442C704CF27453D05A70470A4A4CF27653F9E7EA
S214442C80084A4CF27853F5E7064A4CF27A53F1E791
S214442C90044A4CF27C53EDE7024A4CF27E53E9E791
S214442CA0FF2070477448412008B50621002013F0E1
S214442CB092FD024A4CF27453D05208BD74484120E7
S214442CC010B50221012013F086FD064C4CF27653D3
S214442CD02B21E052012013F07EFD4CF27E53E0524D
S214442CE010BD00BF7448412010B50321022013F0E4
S214442CF072FD094C4CF278530421E052022013F042
S214442D006AFD4CF27A530521E052022013F063FD2B
S214442D104CF27C53E05210BD74484120002113F01D
S214442D2047BC084A4CF2385382B00749D3580093FC
S214442D300B68009A9B1A0193019B8342F8D902B010
S214442D40704700BF74484120AC0D422038B50F4D43
S214442D500F4C95F890305BB901234CF23C5285F801
S214442D609030A3580133A350BDE8384006F03ABE2D
S214442D700BF0DEF94CF23C52002385F89030A35811
S214442D800133A3504CF23852EBE700BFA81F402053
S214442D90744841200020FFF74FBF10B58D20244CC7
S214442DA01CF0B0F8002223498D201CF0AAF88F208E
S214442DB01CF0A8F8002220498F201CF0A2F8972087
S214442DC01CF0A0F800221D4997201CF09AF89A207F
S214442DD01CF098F800221A499A201CF092F81949D7
S214442DE000201EF0D7FB184902201EF0D3FB1749DB
S214442DF00A201EF0CFFB16490D201EF0CBFB2146C1
S214442E00012200201EF048FE04F59671012202209D
S214442E101EF042FE04F26C5101220A201EF03CFED3
S214442E2004F28C5101220D20BDE810401EF034BE41
S214442E30804B4120A11F4600A71F4600AD1F4600F9
S214442E40B31F4600F4AA4600C8AA46009CAA4600F9
S214442E5070AA460010B48AB90949D1F86C3891F87A
S214442E60B848CA18013301F6B801DBB282F85846AE
S214442E7010BC012241F84C3C1EF05EBF10BC7047AB
S214442E807448412010B48AB90949D1F8743891F885
S214442E90D848CA18013301F6D801DBB282F858473D
S214442EA010BC012241F8643C1EF046BF10BC70477B
S214442EB074484120194B012142F64400002219501F
S214442EC044F2A470195046F20470195048F26460F3
S214442ED019504AF2C45019504CF22450195042F634
S214442EE048015A5044F2A8715A5046F208715A5052
S214442EF048F268615A504AF2C8515A504CF2285126
S214442F00C3E9C1225A504CF248524CF250319950BF
S214442F104CF244524FF448619950704774484120EB
S214442F2010B5064B4FF4FB5404FB003042F64803FE
S214442F30C15042F64C03C25010BD00BF74484120F5
S214442F40094BD3E9C1218A420BD01A4492F8042291
S214442F5002700020D3F804230132D2B2C3F804230B
S214442F6070470120704700BF7448412007B50122CE
S214442F700DF107018DF8070000201EF0E1FB03B0B9
S214442F805DF804FB0FB470B5C2B0002446AA02AE86
S214442F9052F8041B304601920FF086FC30460CF083
S214442FA041FDC5B2E3B29D4204D842B0BDE870408C
S214442FB004B07047305D0134FFF7D8FFF2E708B538
S214442FC08E201BF09FFF96201BF09CFF0748FFF7C0
S214442FD0D9FF074900201DF05DFA012005491DF080
S214442FE059FA0548BDE80840FFF7CCBF708E460046
S214442FF044AA460018AA4600788E46000B2938B5DF
S214443000044614D142F644030E4D00220E48EA50BC
S214443010FFF7B8FF42F64803EB581BB142F64C02A2
S214443020A85898472046BDE838401AF06DB9074B73
S2144430301A6832B1002206481A60BDE83840FFF7E5
S214443040A1BF38BD744841207E8E4600B4704120EE
S2144430509A8E46000B2938B505460E4C13D144F2D9
S214443060A47300220C48E250FFF78CFF44F2A87386
S214443070E3581BB144F2AC72A05898472846BDE8C2
S21444308038401AF041B944F2A073E2580AB100221B
S214443090E25038BD74484120B98E46000B2938B5F5
S2144430A0044614D146F204730E4D00220E48EA50EC
S2144430B0FFF768FF46F20873EB581BB146F20C72F2
S2144430C0A85898472046BDE838401AF01DB9074B23
S2144430D01A6832B1002206481A60BDE83840FFF745
S2144430E051BF38BD74484120D58E460074AF412048
S2144430F0F18E46000B2938B504464FF4FB55134869
S21444310015D105FB040542F6440300221048EA5054
S214443110FFF738FF42F64803EB581BB142F64C0221
S214443120A85898472046BDE838401AF0EDB805FB45
S214443130040404F52154236833B10023054823606E
S214443140BDE83840FFF71EBF38BD00BF7448412075
S2144431500F8F46002B8F46000B2938B504464FF494
S214443160FB55134815D105FB040542F644030022DB
S2144431701048EA50FFF706FF42F64803EB581BB1E7
S21444318042F64C02A85898472046BDE838401AF004
S214443190BBB805FB040404F52154236833B100236B
S2144431A005482360BDE83840FFF7ECBE38BD00BF95
S2144431B0744841204A8F4600668F46000B2938B52E
S2144431C004464FF4FB55134815D105FB040542F657
S2144431D0440300221048EA50FFF7D4FE42F6480360
S2144431E0EB581BB142F64C02A85898472046BDE817
S2144431F038401AF089B805FB040404F521542368C2
S21444320033B1002305482360BDE83840FFF7BABE13
S21444321038BD00BF74484120858F4600A18F4600C4
S21444322038B50A243C4D2946002013F0E5FE38B153
S214443230013C14F0FF04F6D121463848FFF7A2FEBD
S2144432400A24374D2946012013F0D6FE38B1013CF6
S21444325014F0FF04F6D101213048FFF793FE0A2408
S214443260304D2946022013F0C7FE38B1013C14F015
S214443270FF04F6D102212948FFF784FE00222A499A
S214443280B4200A241BF03DFE00222849B5201BF03A
S21444329038FE00222649B6201BF033FEB4201BF02D
S2144432A031FEB5201BF02EFEB6201BF02BFE002070
S2144432B013F038FB38B1013C14F0FF04F7D1214633
S2144432C01C48FFF75FFE0A24012013F02BFB38B19D
S2144432D0013C14F0FF04F7D101211648FFF752FED3
S2144432E00A24022013F01EFB38B1013C14F0FF04FC
S2144432F0F7D102210F48FFF745FE0121002013F0C5
S21444330093FB0121084613F08FFB01210220BDE800
S214443310384013F089BB00BFE09D4600DC8F460072
S214443320849D4600289D4600D5754500DB754500BE
S214443330E1754500C08F460038B51C4C05462068EC
S21444334004302044FFF7FCFD012801D1012038BD9C
S2144433502368E21810790A2810D00D280ED00828C1
S21444336015D123B1013B12482360FFF70BFE2368B7
S214443370AB42EBD325440020E87006E00D48FFF747
S21444338001FE23680020234418712060DFE7A0F183
S21444339020035E2BEBD8FFF7E9FD2368E1180133E1
S2144433A00A792360303A81F80421E0E774484120E2
S2144433B0F18F46000090460010B58020FFF7BCFF12
S2144433C090B90A4C23797BB10949201D0CF020FBA7
S2144433D020B90848BDE81040FFF7D4BD211D064873
S2144433E0BDE81040FFF7CEBD10BD00BF7448412075
S2144433F0F58F4600FB8F4600039046002DE9F04FBC
S214443400082389B0002492463B4A054689464FF035
S21444341064081068EDB2516802AF012622468DF862
S21444342010408DF81C40DFF8E8B0CDE905346B4415
S21444343003C35146484624F04EFC04AA214640F2B3
S21444344055532846CDF8048000978DF81C608DF8B7
S2144434501040059419F046FE284B04AA21462846F7
S21444346002934FF607738DF81060ADF80C300623C0
S214443470CDE9007805935B4619F034FE204A0623CE
S214443480214602924FF6FF72059328465B46ADF8F6
S2144434900C2004AA8DF81060CDE9007819F022FEBD
S2144434A0184A062321460292284604AA05935B46F8
S2144434B0ADF80C408DF81060CDE9007819F012FE96
S2144434C0114B124A214628468DF81060CDE9023247
S2144434D0082304AA05935B46CDE9007819F002FE5A
S2144434E00A20FFF71EFC32465146484624F0F3FBBA
S2144434F009B0BDE8F08F00BF348446001000500089
S21444350010019FFF1002C00071020304050607085D
S214443510F100DA182DE9F0410446002855D16D2013
S2144435201BF0F0FC2246C0496D201BF0EAFC6E20DE
S2144435301BF0E8FC2246BD496E201BF0E2FC01224B
S2144435400821BB4824F0C7FB01220521B84824F0D3
S214443550C2FBB84AB849204619F056F8012120461D
S2144435601AF014F822460E21204619F06BFE204627
S21444357019F0EAFF2346B14A0E21204619F082F993
S2144435802346AF4A0E21204619F0C0F9FEF7C1FE85
S2144435902046FFF7A8F9AB4B012242F644015A50A5
S2144435A003F521531A6041F698700023A64A444313
S2144435B0A648A35004441A46013384F8712028349C
S2144435C0C82BF9D10020BDE8F081012846D0022856
S2144435D040F0898074209E4F1BF094FC00229D4945
S2144435E074201BF08EFC75201BF08CFC00229A493C
S2144435F075201BF086FC01220421984824F06BFBBE
S21444360001220621964824F066FB0025954A20466A
S2144436109549DFF8B88218F0F7FF204619F094FF72
S21444362005F10E0658F83530904A0220F6B223F0DB
S21444363060430135314619F025F93A4600233146B0
S2144436400220503719F062F90B2DE9D17D4B012247
S21444365046F204715A5003F5CE43A3E77120844FD3
S2144436601BF050FC0022834971201BF04AFC722058
S2144436701BF048FC0022804972201BF042FC224684
S2144436800721774824F027FB22460221734824F07A
S21444369022FB0025794A20467949DFF8348218F01F
S2144436A0B3FF204619F050FF05F11C0658F8353094
S2144436B0744A0120F6B223F060430135314619F0CE
S2144436C0E1F83A46002331460120503719F01EF9F6
S2144436D0042DE9D144F2A4715A4B01225A5044F2C3
S2144436E0A0715A505FE7032859D0042800F0F480AC
S2144436F005287FF458AF7B20634D1BF003FC002263
S21444370062497B201BF0FDFB7C201BF0FBFB002268
S2144437105F497C201BF0F5FB01220E21504824F023
S214443720DAFA01225B48114624F0D5FA5A4A5B4934
S214443730204618F069FF204619F006FF0122554935
S2144437402046FFF75BFE564A5449204618F05CFF75
S214443750204619F0F9FE2B68524A0E2123F06043A6
S214443760204619F08FF800234F4A0E21204619F0C0
S214443770CDF8AB684B4A0F2123F06043204619F03E
S21444378081F80023494A0F21204619F0BFF84CF22D
S21444379024512C4B01225A504CF22051A1E7772059
S2144437A0434F1BF0AFFB0022424977201BF0A9FB96
S2144437B078201BF0A7FB00223F4978201BF0A1FB92
S2144437C0012200213D4824F086FA01223B48002588
S2144437D01146DFF8008124F07EFA394A39492046FA
S2144437E018F012FF204619F0AFFE05F10E0658F801
S2144437F03530354A0320F6B223F06043013531466E
S21444380019F040F83A46002331460320503719F061
S2144438107DF80A2DE9D148F264610A4B01225A50D8
S21444382048F260615DE700BF05ED45000BED4500DD
S21444383008172940D4A14600984140203C20402007
S214443840444C402074484120F0A6402060874020E5
S214443850446040204DED450053ED45000E17294089
S2144438600C17294024A14600483840205C204020BC
S214443870A45A40202FED450035ED45007CA1460076
S214443880F03C40204C204020548746008FED4500B5
S21444389095ED4500101729403C844600502A4020A8
S2144438A01CA046008C204020447E4020947E40202D
S2144438B0446A40206BED450071ED450006172940EB
S2144438C0CCA04600A03340206C204020C48746004D
S2144438D01C884600748746007920294D1BF012FB4D
S2144438E00022284979201BF00CFB7A201BF00AFBA7
S2144438F0002225497A201BF004FB01220A21234892
S21444390024F0E9F901220921204824F0E4F9204A68
S2144439102049204618F078FE204619F015FE092264
S2144439201A492046FFF76AFD1B4A1A49204618F0F2
S2144439306BFE204619F008FE2B68184A0E2123F029
S2144439406043204618F09EFF0023154A0E21204669
S21444395018F0DCFFAB68114A0F2123F06043204681
S21444396018F090FF00230F4A0F21204618F0CEFF90
S2144439704AF2C4510C4B01225A504AF2C051B0E6A6
S214443980648746007DED450083ED450008172940D1
S2144439903C844600F82E402074A046007C204020FC
S2144439A04474402094744020744841200000000031
S2144439B041F69872084B02FB003310B503EB8104C2
S2144439C0E278A07800EB0220627802EB002213F83B
S2144439D0210000EB022010BD6087402010B5094B43
S2144439E041F6987404FB0030130A00EB810181F819
S2144439F0282081F82930130C120E81F82A3081F8D9
S214443A002B2010BD6087402013B502AB044603E963
S214443A10060041F69871094A9DF8043001FB0022DD
S214443A20009903F03F0321F06041FEF78FFF2046E4
S214443A3002B0BDE81040FEF756BF00BF888740205E
S214443A40FDF70CBF70477047704770477047704724
S214443A5070477047704770477047074B074A196866
S214443A6058799160197941EA002191819979DB79F5
S214443A709173D373704700BF60874020E88340202B
S214443A800E490F4810B54A780B7802F0010443EA11
S214443A900423C2F34104C2F3C10243EA442343EA83
S214443AA0C2238A7843EA4233CA7843EA4253426995
S214443AB002F060421343436110BD00BF608740205C
S214443AC0E8834020074B08491B7803F003021B0990
S214443AD003F0040313430A7C22F0070213430B74D7
S214443AE0704700BF60874020E88340200549064B66
S214443AF00A7E1B7822F01F0203F01F0313430B7643
S214443B00704700BFE8834020608740200549064B45
S214443B100A7F1B7822F01F0203F01F0313430B7720
S214443B20704700BFE8834020608740200649074B23
S214443B3091F820201B7822F00F0203F00F03134362
S214443B4081F82030704700BFE883402060874020DB
S214443B50114B124810B55A78997802F003041B7832
S214443B6043EA0423C2F3810443EA8423C2F30114E0
S214443B70920943EA043343EA823301F00302C1F371
S214443B80810143EA0243426A120D43EA8143120525
S214443B901343436210BD00BF60874020E883402043
S214443BA00E4B0F4A5878197841EA00215879118506
S214443BB0997801F00F0182F82A10D97882F82B10F0
S214443BC0197941EA002191859979DB7901F00F0151
S214443BD082F82F3082F82E10704700BF608740204E
S214443BE0E88340200E4B0F4A5878197841EA002162
S214443BF058791186997801F00F0182F83210D978F5
S214443C0082F83310197941EA002191869979DB7953
S214443C1001F00F0182F8373082F83610704700BF43
S214443C2060874020E88340200C4B0D4A587819782A
S214443C3041EA002158791187997801F00F0182F8FA
S214443C403A10197941EA002191879979DB7901F094
S214443C500F0182F83F3082F83E107047608740205C
S214443C60E88340202D492E4A10B50B78487803F057
S214443C707F0343EAC013887843EAC033C87843EAEC
S214443C80C053106C00F00040034348791364C0F3FB
S214443C9040040B79897982F8443000F001031B0212
S214443CA043EA4423C0F3800443EA8423C0F3C004B5
S214443CB043EAC423C0F3001443EA0433C0F3401475
S214443CC043EA4433C0F38014C00943EA843343EAE6
S214443CD0C03301F0010043EA0043C1F3400043EA25
S214443CE04043C1F3800043EA8043C1F3C00043EA43
S214443CF0C043C1F3001043EA0053C1F34010C1F37C
S214443D00801143EA405343EA8153516C21F4FF0146
S214443D1021F4FE410B43536410BD00BF608740202E
S214443D20E88340200D4A0E4810B55178137801F0C8
S214443D300F04C1F3001143EA042343EA01339178A4
S214443D4043EA4133D17843EA4153816C01F0604100
S214443D500B4383645368C36410BD00BF6087402030
S214443D60E8834020034A044B1168526819655A6533
S214443D70704700BF60874020E8834020244A254996
S214443D8070B55578137805F003069078D47843EAEE
S214443D900623C5F3810643EA8623C5F30116AD0917
S214443DA043EA063343EA8533C0F3011543EA054341
S214443DB0850900F00F0043EA854304F0030543EA0F
S214443DC00553C4F3810543EA8553C4F30115A40996
S214443DD043EA056343EA84638C6D04F070442343EA
S214443DE054798B651379D27981F85C30230104F0D9
S214443DF0030403F4706343EA0233CA6D43EA005093
S214443E00054B40EA046013401843C86570BD00BFC4
S214443E1060874020E8834020FF0000FC70B5224DB8
S214443E20224A2C78E878C4F3401604F00F03297924
S214443E3043EA0613C4F38016E40943EA461343EA06
S214443E4084136C7843EAC413AC7843EAC43300F072
S214443E50030443EAC453C0F3810443EA4463C0F30F
S214443E600114800943EAC46343EA4073106E00F0C9
S214443E700040034301F0030013668B0803F0040379
S214443E800343880800F0080003438808C90900F083
S214443E901000034343EA411392F8641021F03F01B3
S214443EA00B4382F8643070BD60874020E88340202E
S214443EB0114A124810B55178137801F0030443EAC6
S214443EC00423C1F3810443EA8423C1F3011489091A
S214443ED043EA043343EA8133A0F868305388A0F8B1
S214443EE06A309388A0F86C30937980F86E30D37932
S214443EF080F86F3010BD00BF60874020E8834020C4
S214443F00064B074A1968587911671979DB7941EAEB
S214443F10002182F87630A2F87410704760874020FB
S214443F20E8834020084A09491378907881F8783025
S214443F3053781843D378064A9B0443EA0023886F91
S214443F40024013438B67704760874020E8834020D5
S214443F50FF0000FC08B5054B18880CF07FFB0449AD
S214443F600CF0D0FB034BD86708BD00BF60874020E9
S214443F70CDCCCC3DE8834020104B41F69871104A96
S214443F80595C82F8801041F69B71585C41F69A71F0
S214443F90595C41EA0021A2F8811041F69D71585CB3
S214443FA041F69C71595C41EA0021A2F8841041F61E
S214443FB09F715B5C82F88630704700BF6087402004
S214443FC0E8834020064A41F69871064B5158C3F898
S214443FD0881041F69F71525C83F88C20704700BF6E
S214443FE060874020E88340200C4A41F69F730C4982
S214443FF010B541F69974D05C41F69873D35C125D63
S21444400002F0010243EA0223D1F89020520C43EA1C
S214444010402352041343C1F8903010BD60874020BB
S214444020E8834020284941F69973284A70B5C85C0D
S21444403041F69A73CD5C41F69B7300F00306CC5C64
S21444404041F69873CB5C43EA0623C0F3810643EA01
S2144440508623C0F30116800943EA063343EA8033D5
S21444406005F00300C5F3810543EA004304F003006A
S21444407043EA854343EA0053C4F38100A40943EA70
S2144440808053D2F8940043EA046300F07C40034330
S21444409041F69F70C2F8943041F69C73CB5C82F82C
S2144440A0983041F69D73CB5C095C1B0203F47C5349
S2144440B043EA8133D2F8981021F47F1121F47C51DD
S2144440C00B43C2F8983070BD60874020E883402098
S2144440D0214843F63073214930B5C35A5BBAA1F838
S2144440E09C3043F63373C25C43F63273C2F3011515
S2144440F0C45C930943EA850304F00F05240943EAA4
S214444100051343F63675455DED0843EA0523C2F3C9
S214444110800543EA4533B1F89E5005F440452B43A9
S214444120A1F89E3043F63473C55C43F63573C35CDE
S21444413043EA0523A1F8A030C2F3C003520143EA80
S214444140440302F060021A4391F8A23023F07F033E
S2144441501A4381F8A22030BD60874020E88340207F
S214444160164A43F63073164910B5D35A5BBAA1F8CB
S214444170A43043F63273D05C43F63373D35C43EADD
S2144441800023A1F8A63043F63673D05C43F6347366
S214444190D45C43F63573D35C43EA042200F001034F
S2144441A0C0F3400043EA4203D1F8A820920C43EA05
S2144441B0404392041343C1F8A83010BD60874020A2
S2144441C0E8834020124A43F63071124B515A49BA9A
S2144441D0A3F8AC1043F63271505C43F63371515C2D
S2144441E041EA0021B3F8AE0061F30D0043F63671A0
S2144441F0A3F8AE0043F63770515C125C42EA0122E3
S214444200B3F8B01062F30D01A3F8B010704700BFC6
S21444421060874020E883402030B543F63073304C06
S2144442203049E35A5BBAA1F8B43043F63673E05CDF
S21444423043F63773E25C43F63273E55C00F00303FF
S21444424043EA8503C0F3800543EA8523C2F3800529
S21444425043EAC523850943EA0533B1F8B65005F465
S21444426040452B43C2F3C005A1F8B63043F633733A
S214444270E35C81F8B830C0F3C0031B0243EA45232D
S21444428002F0030543EA852343F63475655D43EA45
S2144442900533C0F30015C0F3401043EA0553C2F398
S2144442A0001543EA45539509120943EA8553D1F864
S2144442B0B85002F0020225F47F05024325F47F45F8
S2144442C02B43C1F8B83043F63573E35C81F8BB3012
S2144442D091F8BC3023F003031A4381F8BC2030BD68
S2144442E060874020E8834020F0B543F63273404F61
S2144442F0404DFE5C43F63473F95C43F63373C6F3C1
S214444300801CF85C43F63573FC5C43F63673FA5C03
S214444310F30943EA4C0343F6317C42EA042217F895
S2144443200CC043EA8C03C6F3401C43EA8C23C6F312
S214444330001C43EACC23C1F3400C43EA0C3343F657
S214444340307C17F80C7043EA4733C6F3C00743EA99
S2144443504753C6F3800743EA8753C0F3001743EA3C
S214444360C753470943EA0763C4F30117A40943EA5A
S214444370C763C6F3400706F0010643EA477343EAB9
S2144443808673D5F8C06006F00046334301F0010654
S214444390C5F8C030C2F30903C0F3C00243EA86231B
S2144443A043EAC223C0F3800243EA0233C0F3400226
S2144443B000F0010043EA4233C1F3C00243EA8033CB
S2144443C043EAC433C1F3001443EA44438C09C1F3BB
S2144443D0800143EA844343EA025343EA4151D5F811
S2144443E0C4309B0D9B051943C5F8C410F0BD00BFEF
S2144443F060874020E8834020284843F6307343F6DD
S21444440036722749F0B5C35A43F63275845C43F690
S21444441035725BBA455D825CA709A1F8C83043F69D
S214444420337347EA820743F63772C65C43F63473FF
S214444430825CC35CB009B1F8CAC042EA042240EACE
S2144444408500C6F3810543EA0623C6F3011640EA0F
S2144444508520144DC3F309030CEA050C43EA86236E
S21444446040EA0C0043EA0733A1F8CA00C4F38100CB
S214444470C4F3011443EA8053D1F8CC0000F07F40E3
S2144444800343C1F8CC30C2F30903B1F8D02043EA61
S214444490842315402B43A1F8D030F0BD60874020DC
S2144444A0E883402000F0FFFF1D4943F630731D4863
S2144444B0F0B5CB5A43F632745BBA0E5DA0F8D430EE
S2144444C043F63373CA5C43F63573CD5CC2F381045A
S2144444D043F634732F09CB5C44EA870443F63677B5
S2144444E043EA0223C95D41EA052144EA8111A0F862
S2144444F0D610C3F30901C2F3001343EA41039109FA
S214444500C2F3401243EAC62343EAC16343EA427312
S214444510D0F8D82002F040421343C0F8D830F0BD5B
S21444452060874020E883402070B5234943F63674BC
S21444453043F6357543F630730C5D4E5DCB5AA5098C
S2144445401E485BBA45EA860543F63776A0F8DC3063
S21444455043F633738E5DCA5C43F6347346EA0424EA
S21444456043F63276CB5C8E5D910943EA022341EAF8
S2144445708601C2F38006C3F3090341EA8621B0F8F4
S214444580DE6006F478463143A0F8DE10C2F3C0017C
S21444459043EA8123C2F30011520943EAC52343EA9E
S2144445A0415343EA8453C0F8E03090F8E43062F371
S2144445B0000380F8E43070BD60874020E8834020E4
S2144445C01D4A43F630731D4870B5D35A5BBAA0F8FB
S2144445D0E83043F63273D45C43F63473D55C43F622
S2144445E03373D15C2B09C5F3C00543EA011143F686
S2144445F03673D65C43F63573D35CDB0043EA561217
S214444600C4F3400343EA450304F00105A40843EA1F
S214444610850343EAC403B0F8EA4004F47E442343E3
S214444620A0F8EA3041EA0233D0F8EC20D20DD205A5
S2144446301343C0F8EC3070BD60874020E8834020C8
S2144446401B4943F631731B4830B5CB5C80F8F030D9
S21444465043F63273CA5C43F63573CD5C43F6347323
S214444660CC5C43F63073C95C93091B0243EA81234E
S214444670C2F3401143EA8143C2F38001C2F3C0024D
S21444468043EAC143D0F8F01043EA02532A0905F03E
S2144446900F0543EA4253084A43EA45630A40134334
S2144446A0C0F8F030230943EA041480F8F44030BDDF
S2144446B060874020E8834020FF0000E0074943F637
S2144446C03073074ACB581BBAC2F8003143F63473EA
S2144446D0CB581BBAC2F80431704700BF60874020ED
S2144446E0E8834020214845F6C863214930B5C35A7B
S2144446F05BBAA1F8083145F6CB63C25C45F6CA639B
S214444700C2F30115C45C930943EA850304F00F051C
S214444710240943EA051345F6CE65455DED0843EAAC
S2144447200523C2F3800543EA4533B1F80A5105F43C
S21444473040452B43A1F80A3145F6CC63C55C45F6A3
S214444740CD63C35C43EA0523A1F80C31C2F3C0032E
S214444750520143EA440302F060021A4391F80E31D0
S21444476023F07F031A4381F80E2130BD6087402032
S214444770E8834020164A45F6C863164910B5D35A0E
S2144447805BBAA1F8103145F6CA63D05C45F6CB63F4
S214444790D35C43EA0023A1F8123145F6CE63D05CDD
S2144447A045F6CC63D45C45F6CD63D35C43EA042239
S2144447B000F00103C0F3400043EA4203D1F8142159
S2144447C0920C43EA404392041343C1F8143110BD9B
S2144447D060874020E8834020F0B545F6CA632D4FF5
S2144447E02D4CFD5C45F6CC63F95C45F6CB63C5F3CE
S2144447F0801CFE5C45F6CD63F85C45F6CE63FA5CF9
S214444800EB0943EA4C0345F6C96C42EA002217F822
S2144448100CC0C2F3090243EA8C03C5F3401C43EAC6
S2144448208C23C5F3001C43EACC23C1F3400C43EA73
S2144448300C3345F6C86C17F80C7043EA4733C6F396
S2144448400017760943EA475343EA8653C0F30116F2
S214444850800943EA4663C5F3400605F0010543EA8A
S214444860C66343EA0573D4F8245105F060452B43E8
S214444870C4F8243101F0010342EA832242EAC0200C
S214444880C1F30012890940EA423040EA8131A4F873
S2144448902811F0BD60874020E8834020284845F62C
S2144448A0C86345F6CE622749F0B5C35A45F6CA658D
S2144448B0845C45F6CD625BBA455D825CA709A1F887
S2144448C02C3145F6CB6347EA820745F6CF62C65C91
S2144448D045F6CC63825CC35CB009B1F82EC142EAAB
S2144448E0042240EA8500C6F3810543EA0623C6F35C
S2144448F0011640EA8520144DC3F309030CEA050C5F
S21444490043EA862340EA0C0043EA0733A1F82E0123
S214444910C4F38100C4F3011443EA8053D1F8300150
S21444492000F07F400343C1F83031C2F30903B1F8C5
S214444930342143EA842315402B43A1F83431F0BD97
S21444494060874020E883402000F0FFFF1D4945F67D
S214444950C8631D48F0B5CB5A45F6CA645BBA0E5DCB
S214444960A0F8383145F6CB63CA5C45F6CD63CD5CDA
S214444970C2F3810445F6CC632F09CB5C44EA870432
S21444498045F6CE6743EA0223C95D41EA052144EA77
S2144449908111A0F83A11C3F30901C2F3001343EAA4
S2144449A041039109C2F3401243EAC62343EAC14392
S2144449B043EA4253D0F83C21920D92051343C0F883
S2144449C03C31F0BD60874020E8834020184845F6D7
S2144449D0C863184930B5C35A5BBAA1F8403145F6A6
S2144449E0CC63C55C45F6CA63C45C45F6CB63C35C1E
S2144449F043EA042245F6CD63E409C35CB1F84201B8
S214444A0043EA0523ED09C3F3090343EA85230A4D24
S214444A1028400343A1F84231C2F30903B1F84421C4
S214444A2043EA84232A401343A1F8443130BD00BFEF
S214444A3060874020E883402000F8FFFF1D4A45F683
S214444A40C8631D4870B5D35A5BBAA0F8483145F6DA
S214444A50CA63D45C45F6CC63D55C45F6CB63D15C7F
S214444A602B09C5F3C00543EA011145F6CE63D65C6F
S214444A7045F6CD63D35CDB0043EA5612C4F34003E9
S214444A8043EA450304F00105A40843EA850343EAE0
S214444A90C403B0F84A4104F47E442343A0F84A31A0
S214444AA041EA0233D0F84C21D20DD2051343C0F864
S214444AB04C3170BD60874020E88340201B4945F652
S214444AC0C9631B4830B5CB5C80F8503145F6CA63A1
S214444AD0CA5C45F6CD63CD5C45F6CC63CC5C45F606
S214444AE0C863C95C93091B0243EA8123C2F380016D
S214444AF043EA8143C2F3C001C2F3401243EAC143CE
S214444B00D0F8501143EA02532A0905F00F0543EA48
S214444B104253084A43EA45630A401343C0F85031B7
S214444B20230943EA041480F8544130BD608740208A
S214444B30E8834020FF0000E030B545F6C863304CBB
S214444B403049E35A5BBAA1F8183145F6CE63E05CC7
S214444B5045F6CF63E25C45F6CA63E55C00F00303C2
S214444B6043EA8503C0F3800543EA8523C2F3800500
S214444B7043EAC523850943EA0533B1F81A5105F4D7
S214444B8040452B43C2F3C005A1F81A3145F6CB6322
S214444B90E35C81F81C31C0F3C0031B0243EA45239F
S214444BA002F0030543EA852345F6CC65655D43EA92
S214444BB00533C0F30015C0F3401043EA0553C2F36F
S214444BC0001543EA45539509120943EA8553D1F83B
S214444BD01C5102F0020225F47F05024325F47F456A
S214444BE02B43C1F81C3145F6CD63E35C81F81F3195
S214444BF091F8203123F003031A4381F8202130BD75
S214444C0060874020E8834020074945F6C863074A42
S214444C10CB581BBAC2F8603145F6CC63CB581BBAA6
S214444C20C2F86431704700BF60874020E883402064
S214444C300C4947F664630C48CA5C47F66563CB5C2C
S214444C4043EA022247F66263CB5C03F00F0343EA6F
S214444C500213D0F86821120D12051343C0F86831C8
S214444C60704700BF60874020E8834020064A47F6E6
S214444C706263D15C47F66363D35C044A43EA012328
S214444C80A2F86C31704700BF60874020E88340201C
S214444C900C4949F6FC530C48CA5C49F6FD53CB5CB8
S214444CA043EA022249F6FA53CB5C03F00F0343EA85
S214444CB00213D0F87021120D12051343C0F8703158
S214444CC0704700BF60874020E8834020064A49F684
S214444CD0FA53D15C49F6FB53D35C044A43EA0123B6
S214444CE0A2F87431704700BF60874020E8834020B4
S214444CF010B51B4C20890BF0B1FC1A490BF002FD91
S214444D00194BA27B1860194B60891A600BF0A6FCFD
S214444D1017490BF0F7FC17490BF0EAFB0BF044F885
S214444D200DA3D3E900230AF0DFFE0BF08DFB124BF4
S214444D30124A1860E37BA08903F00F0313600BF05C
S214444D408DFC0F490BF0DEFC0E490BF0D1FB0E4BED
S214444D50186010BDAFF30080C3F5285C8FC2D53F02
S214444D60E8834020CDCCCC3DA41F40208C1F40205F
S214444D700AD7A33C00C02344981F4020881F4020E5
S214444D80ACC52737ACC5A73E901F4020124A1349EE
S214444D90137D03F003000860C3F3830010499B09A6
S214444DA0086010490B60537D0F49C3F34100086007
S214444DB0C3F3C1000D4903F0010308700C490B60AE
S214444DC053690C49C3F347330B60D38A0A4AC3F387
S214444DD047131360704700BFE8834020781F402085
S214444DE0741F4020701F4020681F4020641F4020CE
S214444DF06C1F4020581F4020601F4020074B084A25
S214444E001B7CC3F300011170C3F34001054AC3F38E
S214444E1080031170044A1370704700BFE883402033
S214444E20561F4020551F4020541F4020FFF7E6BF22
S214444E3008B5FFF7E3FFBDE80840FCF70DBD174A89
S214444E40174992F8243003F003000860C3F3810046
S214444E5014490860C3F3011013499B0908601349B9
S214444E600B6092F82530124903F003000860C3F340
S214444E70810010490860C3F301100F499B0908607C
S214444E800E490B6092F826300D4A03F00301C3F333
S214444E90810311600B4A1360704700BFE8834020CB
S214444EA07C1A4020781A4020741A4020701A4020F9
S214444EB06C1A4020681A4020641A4020601A402029
S214444EC05C1A4020581A402010B5194C208D0BF01F
S214444ED0C5FB18490BF016FC17490BF009FB174B9A
S214444EE0174A186094F82A30A08D03F00F011B0966
S214444EF01160144A136094F82B30134A323B136003
S214444F000BF0ACFB11490BF0FDFB11490BF0F0FA2A
S214444F10104B114A186094F82E3003F00F011B0909
S214444F2011600E4A136094F82F200D4B1A6010BD82
S214444F30E88340200AD7A33B0AD72343501F402088
S214444F404C1F4020481F4020441F40200AD7A33A05
S214444F50F8D32342401F40203C1F4020381F4020A7
S214444F60341F402010B5194C208E0BF077FB18499F
S214444F700BF0C8FB17490BF0BBFA174B174A1860DF
S214444F8094F83230A08E03F00F011B091160144AC6
S214444F90136094F83320134B1A600BF05FFB1249EE
S214444FA00BF0B0FB11490BF0A3FA114B114A1860F1
S214444FB094F8363003F00F011B0911600E4A136053
S214444FC094F837200D4B1A6010BD00BFE88340208C
S214444FD00AD7A33B0AD72343301F40202C1F402028
S214444FE0281F4020241F40200AD7A33AF8D3234240
S214444FF0201F40201C1F4020181F4020141F402004
S21444500010B5174C208F0BF029FB16490BF07AFB92
S21444501015490BF06DFA154B154A186094F83A305A
S214445020A08F03F00F011B091160124A13600BF0A6
S21444503015FB11490BF066FB10490BF059FA104B5F
S214445040104A186094F83E3003F00F011B091160B3
S2144450500D4A136094F83F200C4B1A6010BD00BFF5
S214445060E88340200AD7A33B0AD72343101F402097
S2144450700C1F4020081F40200AD7A33AF8D32342E7
S214445080041F4020001F4020FC1E4020F81E4020E5
S21444509010B53E4C3E4A94F84030B4F8400003F015
S2144450A00101C0F3C7101160C3F34001394A1160CF
S2144450B0C3F38201384AC3F341131160374A13607D
S2144450C00BF0CCFA36490BF01DFB0BF0E1FC354BEC
S2144450D01860206CC0F3C7300BF0C0FA30490BF0B0
S2144450E011FB0BF0D5FC304B1860B4F84200C0F30B
S2144450F0C7100BF0B3FA2D490BF0FAF90BF0C8FCC5
S2144451002B4B94F8442018602A4B1A6094F8453088
S214445110294A03F001011160C3F34001274A116094
S214445120C3F38001264A1160C3F3C001254A1160C7
S214445130C3F30011244A1160C3F34011234A11609B
S214445140C3F38011224ADB091160224A136094F8A3
S2144451504630214A03F001011160C3F340011F4A5F
S2144451601160C3F380011E4A1160C3F3C0011D4A97
S2144451701160C3F300111C4A1160C3F340111B4A6B
S214445180C3F3801311601A4A136010BDE8834020AD
S214445190F41E4020F01E4020EC1E4020E81E402016
S2144451A00AD7233CE41E4020E01E40200000204254
S2144451B0DC1E4020D81E4020D41E4020D01E402056
S2144451C0CC1E4020C81E4020C41E4020C01E402086
S2144451D0BC1E4020B81E4020B41E4020B01E4020B6
S2144451E0AC1E4020A81E4020A41E4020A01E4020E6
S2144451F09C1E402038B5264D264B95F8484004F072
S2144452000102C4F302101A60C4F34002224B1A602F
S214445210C4F38002214B1A60C4F3C002204BE40955
S2144452201A600BF017FA1F4B1F4A18601F4BA86CE6
S2144452301C6095F84930C0F3473003F00F01C3F3C0
S2144452400013323811601A4A13600BF007FA194BF0
S2144452501860B5F84A00C0F3471032380BF0FEF930
S214445260154B1860B5F84C00A0F500400BF0F6F965
S214445270124B1860B5F84E000BF0F0F910490BF0DD
S21444528041FA10490BF034F90F4B186038BD00BF93
S214445290E8834020981E4020941E4020901E4020C4
S2144452A08C1E4020881E4020801E4020841E4020A5
S2144452B07C1E4020781E4020741E4020701E4020D5
S2144452C00AD7233C000048436C1E40207047304BAE
S2144452D0304A10B593F85940C4F381011170C4F3B1
S2144452E001112D4A1170C4F301012C4AA40911700E
S2144452F093F858202A49C2F381100870C2F301106B
S21444530028490870C2F381002749C2F30102087095
S21444531026490A7093F85D202549C2F38100C2F3FA
S2144453200102087023490A7093F85E202249C2F3AA
S21444533003120A7093F85F202049C2F301020A70F0
S21444534093F85A201E4902F003000860C2F3810015
S2144453501C490860C2F301101B49920908601B49A6
S2144453600A6093F85B201A4902F00300C2F38102F4
S2144453700860184993F85C000A700BF06FF91649F8
S2144453800BF0C0F9154B1860154B1C6010BD00BFE0
S214445390E8834020681E4020671E4020661E40204A
S2144453A0651E4020641E4020631E4020621E40202E
S2144453B0611E4020601E402070184020281E402059
S2144453C0581E4020541E4020501E40204C1E402054
S2144453D0481E402069184020CDCCCC3D401E40207D
S2144453E05C1E4020264A274992F8603003F00700A6
S2144453F00860C3F3C00024490860C3F3001023497F
S2144454000870C3F340102249C3F38013087021493F
S2144454100B70B2F860302049C3F3C7130B60136EA9
S2144454201E49C3F3C7330B60B2F862301C49C3F35A
S214445430C1130B6092F863301A49C3F34100086005
S214445440C3F3C1001849C3F34113086017490B60FE
S21444545092F86430164A03F003011160C3F38001E6
S214445460144A1160C3F3C001134A1160C3F3001118
S214445470124AC3F340131160114A1360704700BFC9
S214445480E8834020241E4020201E40201E1E40202C
S2144454901D1E40201C1E4020181E4020141E402066
S2144454A0101E40200C1E4020081E4020041E402093
S2144454B0001E4020FC1D4020F81D4020F41D4020C6
S2144454C0F01D402010B5194C194A94F8683094F8E9
S2144454D06A00C3F38101C3F301131170154A1370B4
S2144454E094F86930144AC3F301011170C3F381017F
S2144454F0124AC3F381131170114A13700BF0AAF8C1
S214445500104B186094F86B000BF0A4F80E4B94F80C
S2144455106C2018600D4B1A7094F86D200C4B1A7062
S21444552094F86E200B4B1A7010BD00BFE8834020E1
S214445530E61D4020D51D4020E51D4020D41D4020BA
S214445540E41D4020E01D4020DC1D4020D81D4020A6
S214445550D71D4020D61D402010B50C4CB4F8720020
S2144455600BF07CF80A490BF0CDF80A4B1860B4F8F7
S21444557070000BF073F806490BF0C4F8064BB4F809
S21444558074201860054B1A8010BD00BFE883402085
S214445590CDCCCC3DD01D4020CC1D4020CA1D402043
S2144455A0084B0949B3F87A20C2F387020A709A6F07
S2144455B00649C2F309220A8093F87820044B1A70ED
S2144455C0704700BFE8834020C81D4020C61D4020C9
S2144455D0C41D402010B5124C124B94F88020B4F8E9
S2144455E081001A600BF03AF80F490BF08BF80F491C
S2144455F00AF07EFF0E4B1860B4F884000BF02EF8C9
S2144456000C490BF07FF80C4B0C4A186094F8863023
S21444561003F00F011B091160094A136010BD00BF57
S214445620E8834020C01D4020ACC52737ACC5A73E04
S214445630BC1D4020CDCCCC3DB81D4020B41D4020E0
S214445640B01D402010B5114CB4F888000BF006F895
S2144456500F490BF057F80F490AF04AFF0E4B1860F3
S214445660B4F88A000AF0FAFF09490BF04BF80949E6
S2144456700AF03EFF094B0A4A186094F88C3003F04F
S2144456800F011B091160074A136010BDE8834020D0
S2144456900AD7A33C00C02344AC1D4020A81D40208C
S2144456A0A41D4020A01D4020114A124992F8903073
S2144456B003F003000860C3F381000F490860C3F396
S2144456C001100E499B0908600D490B6092F8913011
S2144456D00C4903F00100C3F3430308600A490B6016
S2144456E0D2F89030094AC3F343331360704700BF7F
S2144456F0E88340209C1D4020981D4020941D402057
S214445700901D40208C1D4020881D4020841D402034
S214445710194A1A4992F8943003F003000860C3F318
S214445720810017490860C3F3011016499B090860B5
S21444573015490B6092F89530144903F0030008604D
S214445740C3F3810012490860C3F3011011499B0951
S214445750086011490B6092F89630104903F0030034
S214445760C3F3810308600E490B60D2F898300D4AA3
S214445770C3F3833313607047E8834020801D402082
S2144457807C1D4020781D4020741D4020701D402004
S2144457906C1D4020681D4020641D4020601D402034
S2144457A05C1D4020581D402010B50E4C0E4B94F8FE
S2144457B09F0094F89C2000F01F001A6000EB8000C5
S2144457C00AF04CFF094B1860B4F8A0000AF046FFF4
S2144457D007490AF097FF07490AF08AFE064B186005
S2144457E010BD00BFE8834020541D40203C1D40208F
S2144457F0CDCC4C3D00C0CC44381D402010B50C4C9C
S214445800B4F8A6000AF02AFF0A490AF07BFF0A49C0
S2144458100AF06EFE094B1860D4F8A800C0F34F0097
S214445820A0F5FF407F380AF019FF054B186010BDFD
S214445830E88340200AD7A33C00C02344281D4020C8
S214445840201D402010B50D4CB4F8AE00C0F30D003A
S2144458500AF004FF4FF07A510AF054FF084B1860E0
S214445860B4F8B000C0F30D000AF0F8FE4FF07A51D9
S2144458700AF048FF034B186010BD00BFE883402081
S214445880181D4020141D402070470B4A0B49B2F89F
S214445890C40008B5B2F8C030C0F30900C3F38703A8
S2144458A00B700AF0DBFE06490AF02CFF05490AF0A5
S2144458B01FFE054B186008BDE8834020101D40209D
S2144458C0CDCCCC3D9A994C420C1D402010B5174C7B
S2144458D0B4F8CA00C0F309000AF0C0FE14490AF03E
S2144458E011FF144B1860B4F8CC00C0F309000AF05A
S2144458F0B5FE0F490AF006FF0F4B1860D4F8CC00EB
S214445900C0F309300AF0AAFE09490AF0FBFE0B4B25
S2144459101860B4F8D000C0F309000AF09FFE0449AA
S2144459200AF0F0FE064B186010BD00BFE883402026
S214445930CDCCCC3D081D4020041D4020001D4020F9
S214445940FC1C402038B5154DB5F8D60080090AF041
S21444595085FE13490AF0D6FE12490AF0C9FDB5F889
S214445960D840114BC4F34904186020460AF076FE2A
S2144459700E490AF0C7FE0E4B1860D5F8D800C0F39F
S214445980CF200AF06BFE0B490AF0BCFE0A4B1860A7
S2144459900A4B1C600A4B1C6038BD00BFE88340209D
S2144459A0CDCC4C3D66667241F81C40209A99193E0F
S2144459B0F41C40200AD7233CF01C40207C1C40208A
S2144459C01C1B402010B5164CB4F8DE00C0F309008A
S2144459D00AF044FE13490AF095FE134B1860B4F8D7
S2144459E0E000C0F309000AF039FE0E490AF08AFEC8
S2144459F00E4B1860D4F8E000C0F3C9200AF02EFE1F
S214445A0008490AF07FFE0A4B1860B4F8E2008009A1
S214445A100AF024FE03490AF075FE064B186010BDD2
S214445A20E88340209A99193EEC1C4020E81C40200C
S214445A30E41C4020E01C402010B5134CB4F8EA00A7
S214445A40C0F3C5000AF00AFE10490AF05BFE10498E
S214445A500AF04EFD0F4B1860B4F8EC00C0F30B0090
S214445A600AF0FCFD0C490AF04DFE0C4B1860D4F8C5
S214445A70EC00C0F30A300AF0F1FD04490AF042FE95
S214445A80074B186010BD00BFE8834020CDCCCC3D0A
S214445A90CDCC4C40DC1C40200AD7233CD81C4020AC
S214445AA0D41C40207047704710B50E4C0E4B94F8EB
S214445AB00B0194F8082100F01F001A6000EB8000E8
S214445AC00AF0CCFD094B1860B4F80C010AF0C6FD88
S214445AD007490AF017FE07490AF00AFD064B186004
S214445AE010BD00BFE8834020D01C4020CC1C402082
S214445AF0CDCC4C3D00C0CC44C81C402010B50C4C0A
S214445B00B4F812010AF0AAFD0A490AF0FBFD0A4954
S214445B100AF0EEFC094B1860D4F81401C0F34F00A9
S214445B20A0F5FF407F380AF099FD054B186010BD7C
S214445B30E88340200AD7A33C00C02344C41C40202A
S214445B40C01C402070470B4A0B49B2F8280108B5E0
S214445B50B2F82431C0F30900C3F387030B700AF08C
S214445B607DFD06490AF0CEFD05490AF0C1FC054B09
S214445B70186008BDE88340209C1C4020CDCCCC3D1A
S214445B809A994C42981C402010B5174CB4F82E01F4
S214445B90C0F309000AF062FD14490AF0B3FD144B41
S214445BA01860B4F83001C0F309000AF057FD0F49F5
S214445BB00AF0A8FD0F4B1860D4F83001C0F3093042
S214445BC00AF04CFD09490AF09DFD0B4B1860B4F8E9
S214445BD03401C0F309000AF041FD04490AF092FD7D
S214445BE0064B186010BD00BFE8834020CDCCCC3DAA
S214445BF0941C4020901C40208C1C4020881C402034
S214445C0010B5134CB4F83A0180090AF027FD11493F
S214445C100AF078FD10490AF06BFC104B1860B4F893
S214445C203C01C0F349000AF019FD0D490AF06AFD2B
S214445C300AF02EFF0B4B1860D4F83C01C0F3C72083
S214445C400AF00CFD08490AF05DFD084B186010BDCB
S214445C50E8834020CDCC4C3D66667241BC1C402057
S214445C609A99193EB41C40200AD7233CB81C4020BD
S214445C7010B50C4CB4F84201C0F309000AF0EEFC2F
S214445C8009490AF03FFD094B1860B4F84401C0F3D3
S214445C9009000AF0E3FC04490AF034FD044B18609A
S214445CA010BD00BFE88340209A99193EB01C40209E
S214445CB0AC1C402008B5FFF71BF8FFF767F8FFF762
S214445CC0BEF8FFF7E5F9FFF795FAFFF700FBFFF795
S214445CD089FBFFF7F7FBFFF73FFCFFF761FCFFF795
S214445CE0F3F8FFF73FF9FFF78BF9FFF773FCFFF77D
S214445CF0A9FCFFF7D9FCFFF70BFDFFF7E7FDFFF71D
S214445D0021FEFFF75FFEFFF73FFFFFF779FFBDE891
S214445D100840FFF7ADBF10B5124CB4F84A01C0F3C3
S214445D20C5000AF09BFC10490AF0ECFC0F490AF047
S214445D30DFFB0F4B1860B4F84C01C0F30B000AF0BD
S214445D408DFC0C490AF0DEFC0B4B1860D4F84C0171
S214445D50C0F30A300AF082FC03490AF0D3FC074B2E
S214445D60186010BDE8834020CDCCCC3DCDCC4C4013
S214445D70A81C40200AD7233CA41C4020A01C40203A
S214445D8008B5FFF759FEBDE80840FFF7C4BF7047A3
S214445D90704708B5084BD3F86801C0F30F100AF0F3
S214445DA05DFC06490AF0AEFC05490AF0A1FB0AF080
S214445DB06FFE044B186008BDE8834020CDCC4C3DB4
S214445DC000C0CC44C41B402008B5084BB3F86C0153
S214445DD00AF044FC06490AF095FC06490AF088FB9A
S214445DE00AF056FE044B186008BD00BFE883402006
S214445DF00AD7A33C00C02344C81B402008B5094B1F
S214445E00D3F87001C0F30F100AF028FC06490AF0D4
S214445E1079FC06490AF06CFB0AF03AFE044B18601B
S214445E2008BD00BFE8834020CDCC4C3D00C0CC44E8
S214445E30B81B402008B5084BB3F874010AF00EFCB2
S214445E4006490AF05FFC06490AF052FB0AF020FEB7
S214445E50044B186008BD00BFE88340200AD7A33C23
S214445E6000C02344B81B402008B5FFF79DFCFFF74D
S214445E70C5FCFFF7E7FCFFF708FDFFF715FEFFF745
S214445E803DFEFFF760FEFFF784FFFFF79DFFFFF739
S214445E90B5FFBDE80840FFF7CDBF1A4B186810B5EC
S214445EA0C830194C0AF0D6FB18490AF0DFFC09F052
S214445EB07BFF0EF081FF0AF0A7FA154B1549A4F8AC
S214445EC0780118680AF016FB13490AF0CFFC09F06B
S214445ED06BFF0EF071FF0AF097FA104BA4F87A01A4
S214445EE01B68A4F87C310E4B186809F05DFF0EF071
S214445EF063FF0AF089FA0B4B84F87E011B6884F82A
S214445F007F3110BD841C4020E8834020CDCCCC3D5E
S214445F10801C402000C023440AD7A33C7C1C40205D
S214445F20781C4020741C4020324B334A10B5334C06
S214445F301B78126884F88431314B1202D4F88411E9
S214445F401B6802F440729B0203F4806313432D4A99
S214445F501268D20202F4C05213432B4A1268520308
S214445F6002F4C0421343294A1268D20302F4C032F0
S214445F701343274A1268520402F460221343254A04
S214445F80127802F0010243EA0253234A127802F0DE
S214445F90030243EA4253214A127802F0070243EAD4
S214445FA002631F4A0A401F491343C4F884311E4BF8
S214445FB018680AF09FFA1D490AF058FC09F0F4FEE6
S214445FC00EF0FAFE0AF020FA194BA4F88A01186873
S214445FD00AF040FB13490AF08DFA14490AF046FCCD
S214445FE009F0E2FE0EF0E8FE0AF00EFAA4F8880184
S214445FF010BD00BFD61D4020641C4020E8834020CE
S214446000601C40205C1C4020581C4020541C4020EF
S214446010241E40201E1E4020E91A4020E81A402034
S214446020FF0080F8ACC5A73E501C4020ACC52737BF
S2144460304C1C4020184B1949186810B50AF016FC39
S214446040174C09F0B1FE0EF0B7FE0AF0DDF9154B19
S2144460501249A4F88C0118680AF008FC09F0A4FE5A
S2144460600EF0AAFE0AF0D0F90F4B0C49A4F88E01A4
S21444607018680AF0FBFB09F097FE0EF09DFE0AF046
S214446080C3F90A4BA4F890011B7884F89331084B63
S2144460901B7884F8923110BDCC1D4020CDCCCC3D2D
S2144460A0E8834020D01D4020401E4020C81D40208C
S2144460B0C41D4020174B184A1B7812785B0002F028
S2144460C0010203F002031343144A1278920002F0CA
S2144460D004021343124A1278D20002F00802134311
S2144460E0104A1278120102F0100213430E4A127834
S2144460F0520102F0200213430C4A1278920102F035
S214446100400213430A4A127843EAC213094A82F801
S214446110E4317047291C40202A1C4020281C40207B
S214446120271C4020261C4020251C4020241C4020A0
S2144461307E174020E883402038B5254B254D196806
S214446140254B18680AF0D6F9244B044624491868A7
S2144461500AF0D0F923490AF089FB09F025FE0EF02F
S2144461602BFE0AF051F9204B2049A5F8E80118689F
S2144461700AF0C0F91E490AF079FB09F015FE0EF044
S2144461801BFE0AF041F91B49A5F8EA0120460AF02D
S2144461906DFB09F009FE0EF00FFE0AF035F9164BBA
S2144461A0A5F8EC0118880AF059FA14490AF05EFB7F
S2144461B009F0FAFD0EF000FE114B1C780AF024F9A3
S2144461C0C0F30D00A4030443A5F8EE4138BD00BF58
S2144461D0A0174020E8834020A41F4020A417402056
S2144461E0000048430AD7233C9C17402000C0234461
S2144461F00AD7A33CCDCCCC3D7C174020CDCC4C3EDE
S2144462007A1740201C4B1D49186810B50AF02EFB1F
S2144462101B4C09F0C9FD0EF0CFFD0AF0F5F8194BFA
S214446220A4F89401186809F0BFFD0EF0C5FD0AF005
S214446230EBF8154B1549A4F8960118680AF05AF974
S21444624013490AF013FB09F0AFFD0EF0B5FD0AF052
S214446250DBF8104B1049A4F8980118680AF04AF97C
S2144462600E490AF003FB09F09FFD0EF0A5FD0AF067
S214446270CBF8A4F89A0110BD9C1F4020CDCCCC3D51
S214446280E8834020B8194020A418402000C0234486
S2144462900AD7A33C5C1B4020000048430AD7233C53
S2144462A0114B1249186810B50AF0E0FA104C09F080
S2144462B07BFD0EF081FD0AF0A7F80E4B0E491B78C5
S2144462C0A4F89C01A4F89E310C4B18680AF012F905
S2144462D00B490AF0CBFA09F067FD0EF06DFD0AF0A3
S2144462E093F8A4F8A00110BD08194020CDCCCC3DAD
S2144462F0E88340201219402000C023448C184020D4
S2144463000AD7A33C184B1949186810B50AF0F2F896
S21444631017490AF0ABFA174C09F046FD0EF04CFD4F
S2144463200AF072F8144B1549A4F8A40118680AF048
S214446330E1F813490AF09AFA09F036FD0EF03CFDEE
S2144463400AF062F80F4BA4F8A6011B6884F8A8313B
S2144463500D4B1A680D4B1B6803F00F0343EA0213F8
S21444636084F8A93110BD00BF281D402000C0234436
S2144463700AD7A33CE8834020381D402000C0CC44C4
S214446380CDCC4C3D2C1C4020DC1B4020E01B402048
S214446390164B1749186810B50AF0ACF815490AF0B8
S2144463A065FA154C09F000FD0EF006FD0AF02CF8CF
S2144463B0124B1349A4F8AC0118680AF09BF811492B
S2144463C00AF054FA09F0F0FC0EF0F6FC0AF01CF859
S2144463D00D4BA4F8AE011A680C4B1B6803F00F0370
S2144463E043EA021384F8B03110BD00BFC41C4020F9
S2144463F000C023440AD7A33CE8834020C81C40205E
S21444640000C0CC44CDCC4C3DCC1B4020D01B4020BF
S214446410174B186810B500F28F20164C0AF01AF97C
S21444642015490AF023FA09F0BFFC0EF0C5FC09F042
S214446430EBFF124BA4F8B401186800F266600AF049
S21444644009F90F490AF012FA09F0AEFC0EF0B4FC52
S21444645009F0DAFF0B4BA4F8B6011A680A4B1B681E
S21444646003F00F0343EA021384F8B83110BD00BFAB
S214446470C81B4020E88340200AD7A33CC41B4020C6
S214446480CDCC4C3DBC1B4020C01B4020174B18684D
S21444649010B500F28F20164C0AF0DCF815490AF0C5
S2144464A0E5F909F081FC0EF087FC09F0ADFF124BCC
S2144464B0A4F8BC01186800F266600AF0CBF80F49ED
S2144464C00AF0D4F909F070FC0EF076FC09F09CFF53
S2144464D00B4BA4F8BE011A680A4B1B6803F00F0363
S2144464E043EA021384F8C03110BD00BFB81B4020F5
S2144464F0E88340200AD7A33CB41B4020CDCC4C3D77
S214446500AC1B4020B01B40200A4A0B4B126883F851
S214446510DC210A4A126883F8DD21094A126883F8A6
S214446520DE21084A126883F8DF21074A1268C3F856
S214446530E0217047A81B4020E8834020A41B40204D
S214446540A01B40209C1B4020981B40202B4B2C49D2
S21444655030B51D782B4B05F003051C782A4B04F008
S21444656003041878294B00F003001B8881F8C831CF
S214446570274B1A68274B92001B6802F00C0203F064
S21444658003031A43244B1B681B0103F030031A43CE
S214446590224B1B689B01DBB21A43214B1B681B0230
S2144465A003F440731A431F4B1B689B0203F4406377
S2144465B01A431D4B1B681B0303F440531A431B4BDF
S2144465C01B689B039BB21A43194B1B681B0403F4BA
S2144465D040331A43174B1B689B0403F4402313436E
S2144465E0D1F8C42143EA055302F07C4243EA84537B
S2144465F043EA00631343C1F8C43130BD2A1B40202C
S214446600E88340202B1B40202C1B4020281B402086
S214446610901B4020941B40208C1B4020881B40200D
S214446620841B4020801B40207C1B4020781B40203D
S214446630741B4020701B4020124B13491B7803F0F8
S2144466400302124B1B7803F0030343EA8203104A07
S214446650127802F0030243EA02130E4A127802F05A
S214446660030243EA82130C4A127802F0030243EA16
S2144466700223B1F8CC2102F47C421343A1F8CC3176
S214446680704700BF6B1B4020E88340206C1B4020B3
S2144466906A1B4020691B4020681B4020094B0A495E
S2144466A01A680A4B02F001021B6803F0030343EA2C
S2144466B0820391F8D82122F00702134381F8D83197
S2144466C0704700BF601B4020E8834020641B402086
S2144466D038B5344B344D1868C83009F0BBFF3349DD
S2144466E00AF0C4F809F060FB0EF066FB304B1C68F9
S2144466F0304B64001B6804F0020403F001031C439F
S2144467002D4B1B689B0003F004031C432B4B1B6858
S214446710DB0003F008031C43294B1B681B01DBB258
S2144467201C43284B1B681B0203F440731C43264B34
S2144467301B689B0203F4E0531C43244B1B685B0317
S21444674003F4C0431C4309F05FFE214B214903EA8E
S214446750C0331C43D5F8D03103F000431C431E4BD2
S214446760C5F8D041186809F0C5FE10490AF07EF80D
S21444677009F01AFB0EF020FB09F046FE174B1549AC
S214446780A5F8D401186809F0B5FE08490AF06EF871
S21444679009F00AFB0EF010FB09F036FEA5F8D60108
S2144467A038BD00BF341B4020E88340200AD7233C32
S2144467B0501B4020541B40204C1B4020481B40206C
S2144467C0441B4020401B40203C1B4020381B40209C
S2144467D00080FF7F00004843301B40205C1B402065
S2144467E0274B2849186810B509F084FE26490AF054
S2144467F03DF8264C09F0D8FA0EF0DEFA09F004FE0D
S214446800234B2449A4F84402186809F073FE22492D
S2144468100AF02CF809F0C8FA0EF0CEFA09F0F4FDA6
S2144468201E4BA4F846021B68A4F848321C4B1A6850
S2144468301C4B02F003021B6803F0010343EA4203C5
S214446840194A126802F0030243EAC203174A12685E
S21444685002F0010243EA4213154A126802F00F029C
S21444686043EA8213134A126802F00F0243EA822371
S214446870B4F84A2202F440421343A4F84A3210BD04
S2144468806C1E4020000048430AD7233CE88340203F
S214446890281D402000C023440AD7A33C1C1B40208C
S2144468A05C1C4020141B4020541C4020081B4020E5
S2144468B0041B4020001B4020314B4FF08E4110B546
S2144468C01B78304C03F00F022F4B1B7803F00F035A
S2144468D043EA02132D4A1268120202F4706213430A
S2144468E02B4A1268120302F480521343294A126850
S2144468F0520302F4C0421343274A1268D20302F4F6
S214446900C0321343254A1268520402F0FF721343FE
S214446910D4F84C2202F07E421343C4F84C32204B47
S214446920186809F0E7FD09F03FFA0EF045FA09F059
S2144469306BFD1C4BA4F850021B7803F003021A4B61
S2144469401B7803F0030343EA8203184A127802F0E2
S214446950070243EA0213164A126802F00F0243EA99
S214446960C213144A126802F00F0243EAC223B4F870
S214446970522202F400421343A4F8523210BD00BF20
S214446980FC1A4020E8834020FD1A4020F81A402094
S214446990F41A4020581C4020EC1A4020181E402070
S2144469A0701E4020E91A4020EA1A4020E81A402087
S2144469B0E41A4020E01A4020144B10B5186809F039
S2144469C0F3F9134C0EF0F8F909F01EFD114B84F858
S2144469D054021B6884F855320F4B1B68A4F8563291
S2144469E00E4B186809F0E0F90EF0E6F909F00CFDD4
S2144469F00B4BA4F858021A680A4B1B6803F00F03A3
S214446A0043EA021384F85A3210BD00BF781C402073
S214446A10E8834020741C40204C1C4020501C4020DE
S214446A20C81A4020CC1A40201C4A936CC3F3473300
S214446A3082F88C32B2F84A30C3F3471382F88D3268
S214446A40B2F84230C3F3C71382F88E3292F85C3001
S214446A5082F88F32124B1968124B01F007011B68FB
S214446A6003F0010343EA41030F49097801F00101A9
S214446A7043EA01130D49096801F00F0143EA411343
S214446A800B49096801F00F0143EA4123B2F890121A
S214446A9001F460410B43A2F890327047E8834020EB
S214446AA0241E4020F01D40201E1E4020C41A4020B4
S214446AB0C01A4020FFF7B8BF174B184A1B78127805
S214446AC05B0002F0010203F002031343144A1278F7
S214446AD0920002F004021343124A1278D20002F0E3
S214446AE008021343104A1278120102F010021343AC
S214446AF00E4A1278520102F0200213430C4A1278CE
S214446B00920102F0400213430A4A127843EAC2133F
S214446B10094A82F894327047291C40202A1C402097
S214446B20281C4020271C4020261C4020251C402092
S214446B30241C40207E174020E8834020174B1868CA
S214446B4010B500F28F20164C09F084FD154909F063
S214446B508DFE09F029F90EF02FF909F055FC124B79
S214446B60A4F82402186800F2666009F073FD0F4921
S214446B7009F07CFE09F018F90EF01EF909F044FC01
S214446B800B4BA4F826021A680A4B1B6803F00F0343
S214446B9043EA021384F8283210BD00BFBC1A4020D2
S214446BA0E88340200AD7A33CB81A4020CDCC4C3DBD
S214446BB0B01A4020B41A4020174B186810B500F29B
S214446BC08F20164C09F046FD154909F04FFE09F092
S214446BD0EBF80EF0F1F809F017FC124BA4F82C026F
S214446BE0186800F2666009F035FD0F4909F03EFE6C
S214446BF009F0DAF80EF0E0F809F006FC0B4BA4F8BE
S214446C002E021A680A4B1B6803F00F0343EA02136A
S214446C1084F8303210BD00BFAC1A4020E8834020D0
S214446C200AD7A33CA81A4020CDCC4C3DA01A4020FD
S214446C30A41A402038B5184B184C1D6805F28F200E
S214446C4009F008FD164909F011FE09F0ADF80EF0FA
S214446C50B3F809F0D9FB134BA4F83402186800F2D1
S214446C60666009F0F7FC104909F000FE09F09CF84C
S214446C700EF0A2F809F0C8FB0C4BA4F836021A68CA
S214446C800B4B1B6803F00F0343EA021384F83832B5
S214446C90084B1D6038BD00BF9C1A4020E883402046
S214446CA00AD7A33C981A4020CDCC4C3D901A40209D
S214446CB0941A4020C81B402038B5184B184C1D6801
S214446CC005F28F2009F0C6FC164909F0CFFD09F0FD
S214446CD06BF80EF071F809F097FB134BA4F83C02DE
S214446CE0186800F2666009F0B5FC104909F0BEFD6C
S214446CF009F05AF80EF060F809F086FB0C4BA4F83D
S214446D003E021A680B4B1B6803F00F0343EA021358
S214446D1084F84032084B1D6038BD00BF8C1A4020B2
S214446D20E88340200AD7A33C881A4020CDCC4C3D6B
S214446D30801A4020841A4020B81B40204C4B4FF009
S214446D4084412DE9F04FDFF864A187B01B788AF8B8
S214446D50B832484B1B788AF8B932474B186809F062
S214446D60C9FB4FF0834109F0CDFC09F01DF80EF045
S214446D7023F8424B8046894618684FF0844109F010
S214446D80B9FB4FF0834109F0BDFC09F00DF80EF055
S214446D9013F83B4B06460F4693F800B0394B3A4936
S214446DA00BF0010B186809F0A5FB384909F05EFDA5
S214446DB008F0FAFF0EF000F8354B364A1B78CDE95A
S214446DC0000110683449059309F094FB334909F0EF
S214446DD04DFD08F0E9FF0DF0EFFF314A1478314AD3
S214446DE004F001041578240305F00105CDE90201F9
S214446DF04946404609F008FBC0F30900AD0239464F
S214446E000543BAF8BA0200F4784005433046AAF877
S214446E10BA524FEA8B2509F0F7FAC0F3090BDDE9BD
S214446E20000109F0F1FA204A059B45EA0B0B02EAF9
S214446E30C02203F001034BEA020BDAF8BC224BEA09
S214446E40C35302F07F421343DDE90201CAF8BC3261
S214446E5009F0DAFAC0F30B000443BAF8C00200F4AF
S214446E6060400443AAF8C04207B0BDE8F08F00BFB4
S214446E705D1940205C194020581940205019402084
S214446E804C1940204819402033336F410AD7233CDD
S214446E904419402040194020CDCCCC42CDCC4C3D6A
S214446EA03C1940205419402000F87F00E8834020D5
S214446EB0124B1A8DC3F85C22114A1168114A01F02C
S214446EC00F01126802F00F0242EA011293F82B10E7
S214446ED042EA0122A3F860229A8DC3F864220A4A41
S214446EE011680A4A126802F00F0242EA011283F855
S214446EF06822074A126883F869227047E88340206C
S214446F00481F40204C1F4020381F40203C1F402034
S214446F10341F4020114B1A8EC3F86C22104A116855
S214446F20104A126802F00F0242EA011283F87022F5
S214446F300D4A126883F871229A8EC3F874220B4A5B
S214446F4011680B4A126802F00F0242EA011283F8F3
S214446F507822084A126883F879227047E8834020EA
S214446F60281F40202C1F4020241F4020181F40204C
S214446F701C1F4020141F40200F4B1A8FC3F87C223E
S214446F800E4A11680E4A126802F00F0242EA0112D3
S214446F9083F880229A8FC3F884220A4A11680A4AE0
S214446FA0126802F00F0242EA011283F88822074A66
S214446FB0126883F889227047E8834020081F4020DF
S214446FC00C1F4020FC1E4020001F4020F81E40207E
S214446FD0334B3449F0B51E78334B06F0030691F82C
S214446FE05C201D78314B42EA062205F003051C68F6
S214446FF02F4B42EA8522240318682E4BA4B2000481
S2144470001B78224300F4702003F003072A4B1043F6
S2144470101B7803F0030343EA8703284F3F7807F0BF
S214447020030743EA0713264F3F7807F0030743EA6C
S2144470308713244F3F7807F0030743EA0723224F7A
S2144470403F7807F0030743EA8723204F3F7807F04B
S214447050030743EA07331E4F3F68BF03BFB23B43B1
S2144470601C4F43EA06433F7843EA864307F0030748
S21444707043EA065343EA865343EA066343EA87638E
S214447080D1F8007207F070473B43C1F80032D1F89C
S21444709004321B0D1B051843C1F80402F0BD00BFA3
S2144470A0601E4020E8834020611E4020101A402085
S2144470B00C1A4020631E4020621E4020641E40205E
S2144470C0651E4020661E4020681E4020671E4020E5
S2144470D05C1E402069184020204B214A70B51C682D
S2144470E0204BB2F8605004F00F04186892F86030F1
S2144470F005F4FF4592F8641000F00F0003F07F0398
S2144471002B43156E05F4FF052B43B2F86250C5F3C6
S214447110C11543EAC55392F86350C5F3410643EAA2
S2144471204663C5F3C106C5F3411543EAC66343EA5D
S2144471304573D2F8085205F000452B43C2F808328E
S21444714001F03F03B2F80C1243EA841301F44041C1
S21444715043EA80230B43A2F80C3270BDEC1D40205A
S214447160E8834020E81D40201D4B1E4A1B681268D9
S2144471709B001D4902F0030203F00C0313431B4A11
S2144471801268120102F030021343194A126892013F
S214447190D2B21343174A1268120202F440721343DF
S2144471A0154A1268920202F440621343134A126864
S2144471B0120302F440521343114A1268920302F433
S2144471C0703213430F4A1268920402F47012134347
S2144471D0D1F82022920D92051343C1F8203270470D
S2144471E0FC194020001A4020E8834020F81940202B
S2144471F0F4194020F0194020EC194020E8194020AA
S214447200E4194020E01940201A4B1B49186810B571
S21444721009F02CFB194C08F0C7FD0DF0CDFD09F024
S214447220F3F8174B1449A4F81002186809F01EFB2B
S21444723008F0BAFD0DF0C0FD09F0E6F8114BA4F8CD
S2144472401202188809F00AFA0B4909F00FFB08F0F5
S214447250ABFD0DF0B1FD09F0D7F80B4BA4F81402C2
S2144472601A680A4B1B6803F00F0343EA021384F8B8
S214447270163210BDCC1D4020CDCCCC3DE8834020FA
S214447280D01D4020CA1D4020301E4020341E4020C1
S214447290124A92F8783010B582F81832104BD2F869
S2144472A018421878B2F87A30C3F38701936FC3F361
S2144472B009231B0243EA81430A49097801F00F0176
S2144472C043EA8163084921400B43C2F8183292F8D6
S2144472D01C3260F3030382F81C3210BDE88340205E
S2144472E0DA194020DB194020FF0000C0094B0A4948
S2144472F01A680A4B02F007021B6803F0030343EACA
S214447300820391F8982222F01F02134381F89832A0
S214447310704700BF5C1C4020E8834020501B402040
S214447320064B10B5064C186809F0B2FBB4F89C320C
S21444733060F30903A4F89C3210BD00BF781C4020BB
S214447340E8834020094B0A4A1B7812789B00094977
S21444735002F0030203F00C03134391F8A02222F038
S2144473600F02134381F8A032704700BFD61940205D
S214447370D7194020E8834020044B054993F8A422BB
S214447380097861F3020283F8A4227047E883402018
S214447390D5194020044B054993F8A822097861F38F
S2144473A0030283F8A8227047E8834020D41940207B
S2144473B0F8B53D4B3D4D1B783D4985F8AC323D4BC9
S2144473C0186809F053FA08F0EFFC0DF0F5FC09F0E4
S2144473D01BF8394A394B03EA40231068D5F8AC22E7
S2144473E0000200F480700343354810400343C5F858
S2144473F0AC32344B1B7885F8B032334B1C68334B75
S21444740004F003041F68324B07F001071E68314B33
S21444741044EA870406F00106186809F01BF94FF0A1
S214447420814109F06FF909F033FB2B4A2B4B44EAB0
S214447430C606D5F8B01203EA00231068284A800529
S21444744095F8B44200F4800024F00F040343106817
S214447450244A2643C005126800F4000085F8B46246
S2144474601206034302F0407213431F4A1268920600
S21444747002F0406213431D4A1268120702F080521B
S21444748013431B4A1268520702F000521343194A28
S2144474901268920702F080421343174A0A40134385
S2144474A0C5F8B032F8BD00BF7C194020E8834020C0
S2144474B0CDCCCC3DAC194020B019402000FEFF0195
S2144474C0FF0000FE7D194020881940208419402082
S2144474D080194020A8194020A419402000FF3F00EE
S2144474E0A01940205C1C4020981940209419402044
S2144474F0901940208C194020FF000080084A094B10
S2144475001278094983F8C422084A0978127883F81D
S214447510C52293F8C62261F3000283F8C622704758
S214447520C6194020E8834020C4194020C51940208D
S214447530114B12491B6810B5114C84F8E032114BBC
S2144475401B6884F8E132104B186808F0D3FF0F49E3
S21444755009F08CF908F028FC0DF02EFC08F054FFD6
S2144475600B4A94F8E4321278A4F8E20262F3000379
S21444757084F8E43210BD00BFC019402000C0234444
S214447580E8834020BC194020B81940200AD7A33CC1
S214447590B4194020F8B5204B204D186809F05AF825
S2144475A04FF0814109F0AEF809F072FA1C4B0446DC
S2144475B01F681C4BC4F30D0407F001071E681A4BE2
S2144475C044EA8734186844EAC63409F043F84FF06E
S2144475D0814109F097F809F05BFA144AC0F30D03A9
S2144475E0A5F8DC421068124A800300F48040034346
S2144475F01068104AC003126800F4FF00D205034323
S21444760002F0FF421343D5F8D82202F00042134357
S214447610C5F8D832F8BD00BF68194020E88340203A
S214447620641940206019402078194020741940207D
S214447630701940206C1940200D4B0E4A1B780E4999
S21444764082F8EC320D4B09781B7801F0010182F880
S214447650ED320B4B1B785B0003F002030B4392F8AE
S214447660EE1221F003010B4382F8EE32704700BF5E
S2144476703B194020E8834020391940203A194020DD
S214447680381940200C4B0D4A1B680D4982F8E832E5
S2144476900C4B09781B6801F0030182F8E9320A4B67
S2144476A01B789B0003F00C030B430849097843EA14
S2144476B0011382F8EA32704734194020E8834020A8
S2144476C02F194020301940202E1940202D194020D3
S2144476D0F8B5254B254C1B78254F84F8F032254BBE
S2144476E01B7884F8F132244B1878323008F0B6FF11
S2144476F0014608F0FFFE09F0CBF9204984F8F2026F
S2144477000E781F493F780D781E4907F001071E4B37
S21444771008781E491A78303009781D4B49001B7882
S21444772001F03E01394394F8F37227F03F0739439A
S21444773084F8F31203F03F0102F01F0306F00F0231
S21444774043EA411343EAC22305F03F0243EAC23305
S21444775000F03F0243EA4253D4F8F42202F078425F
S2144477601343C4F8F432F8BD2C194020E883402073
S214447770291940202B1940202A1940202519402039
S2144477802419402023194020271940202819402036
S2144477902619402038B50C4B0C4C5D68284608F03A
S2144477A003FB0DF009FB08F02FFE0949C4F8D40288
S2144477B0284609F05BF808F0F7FA0DF0FDFA08F0F1
S2144477C023FEC4F8D00238BD48464020E883402013
S2144477D0000008422DE9F74F374D384E686809F0E7
S2144477E057F986F8F802A86809F052F9344986F839
S2144477F0F902686908F07EFE324909F037F809F064
S21444780047F98346A86909F043F92D490446E869CF
S21444781008F070FE2B4909F029F8CBF3090B09F060
S21444782037F98246286A09F033F925498146686A59
S21444783008F060FE234909F019F809F029F9804652
S214447840A86A09F025F91E4900F00107E86808F01F
S21444785051FE1C4909F00AF809F01AF9C0F3090365
S2144478602869019309F014F9019B00F0010043EAEA
S2144478708023B6F8FA0200F4784003431248A6F888
S214447880FA32A30200EACA2A03F480634FEA495054
S21444789043EA0B0300F4001043EA0A03034343EAB3
S2144478A08853C6F8FC3296F8003367F3000386F82C
S2144478B0003303B0BDE8F08F48464020E8834020BC
S2144478C066667241CDCC4C3D00F81F00084A094B11
S2144478D01278094983F82823084A0978127883F8E5
S2144478E0292393F82A2361F3000283F82A23704756
S2144478F022194020E88340202019402021194020A6
S214447900114B124A1B68124910B5124C127884F86F
S2144479101833114B1B6884F8193394F81C3362F3FC
S214447920000384F81C330D4B186808F0E3FD0C493B
S21444793008F09CFF08F038FA0DF03EFA08F064FDB3
S214447940A4F81A0310BD00BF1C1940201219402089
S21444795000C02344E88340201819402014194020CE
S2144479600AD7A33C284B294910B5294C1B7884F8E0
S2144479701033284B186808F079FF08F015FA0DF014
S2144479801BFA08F041FD244A244B03EA40231068BE
S214447990D4F81023000200F48070034320481040BB
S2144479A0204A03431268C4F8103312021E4B02F4F2
S2144479B080721B7884F814331C4B1B685B0203F4F8
S2144479C0C06313431A4A1268D20202F4C0521343E5
S2144479D0184A1268520302F400521343164A1268B5
S2144479E0920302F480421343144A1268D20302F408
S2144479F0C0321343D4F8142322F4FF3222F48072A4
S214447A001343C4F8143310BD10194020CDCCCC3DDC
S214447A10E8834020081940200C19402000FEFF014E
S214447A20FF0000FE04194020111940200019402090
S214447A30FC184020F8184020F4184020F018402045
S214447A403A4B4FF084412DE9F047394E1B7886F87F
S214447A500433384B1B7886F80533374B186808F0E0
S214447A6049FD4FF0834108F04DFE09F011F8334BC1
S214447A700446334993F800A0324B0AF0010A1868CA
S214447A8008F038FD304908F0F1FE09F001F82F4BB4
S214447A9081462F4993F800802E4B08F00108186859
S214447AA008F028FD2C4908F0E1FE08F0F1FF2B4BC6
S214447AB005464FF084411F78294BC5F30B0507F064
S214447AC00107186808F016FD4FF0834108F01AFEC7
S214447AD008F0DEFF234BC0F3090245EA0735187861
S214447AE0C4F3090300F0010043EA8A2342EA8022F1
S214447AF0B6F8060300F4784002431B4800EAC92956
S214447B00A6F80623D6F8082343EA090302F07F4280
S214447B1043EAC8531343C6F80833B6F80C3303F4A1
S214447B2060431D43A6F80C53BDE8F087ED1840208B
S214447B30E8834020EC184020E0184020DC18402021
S214447B4033336F41D81840200AD7233CD4184020FA
S214447B50CDCCCC42D0184020CDCC4C3DCC18402087
S214447B60E8184020E418402000F87F002DE9F74F3D
S214447B70374D384E686808F08BFF86F84803A86887
S214447B8008F086FF344986F84903686908F0B2FC71
S214447B90324908F06BFE08F07BFF8346A86908F07C
S214447BA077FF2D490446E86908F0A4FC2B4908F001
S214447BB05DFECBF3090B08F06BFF8246286A08F09B
S214447BC067FF25498146686A08F094FC234908F013
S214447BD04DFE08F05DFF8046A86A08F059FF1E492E
S214447BE000F00107E86808F085FC1C4908F03EFEF2
S214447BF008F04EFFC0F309032869019308F048FFD4
S214447C00019B00F0010043EA8023B6F84A0300F4DF
S214447C10784003431248A6F84A33A30200EACA2A25
S214447C2003F480634FEA495043EA0B0300F4001020
S214447C3043EA0A03034343EA8853C6F84C3396F8A8
S214447C40503367F3000386F8503303B0BDE8F08F33
S214447C5048464020E883402066667241CDCC4C3D81
S214447C6000F81F000D4B0E4A1B780E4982F8243349
S214447C700D4B09781B7801F0010182F825330B4B34
S214447C801B785B0003F002030B4392F8261321F0A3
S214447C9003010B4382F82633704700BFCB184020BD
S214447CA0E8834020C9184020CA184020C8184020FD
S214447CB00C4B0D4A1B680D4982F820330C4B09784F
S214447CC01B6801F0030182F821330A4B1B789B00A2
S214447CD003F00C030B430849097843EA011382F87E
S214447CE022337047C4184020E8834020BC18402004
S214447CF0C0184020BB184020BA184020F8B5254B81
S214447D00254C1B78254F84F84033254B1B7884F844
S214447D104133244B1878323008F0A0FC014608F072
S214447D20E9FB08F0B5FE204984F842030E781F4963
S214447D303F780D781E4907F001071E4B08781E4908
S214447D401A78303009781D4B49001B7801F03E0103
S214447D50394394F8437327F03F07394384F8431371
S214447D6003F03F0102F01F0306F00F0243EA4113FB
S214447D7043EAC22305F03F0243EAC23300F03F021F
S214447D8043EA4253D4F8442302F078421343C4F8F7
S214447D904433F8BDB9184020E8834020B618402044
S214447DA0B8184020B7184020B2184020B1184020D8
S214447DB0B0184020B4184020B5184020B3184020CE
S214447DC008B5FFF785FCBDE80840FFF797BF38B510
S214447DD00C4B0D4C5D68284607F0E6FF0CF0ECFFB4
S214447DE008F012FB0949C4F83C03284608F03EFD57
S214447DF007F0DAFF0CF0E0FF08F006FBC4F838039F
S214447E0038BD00BF48464020E88340200000084272
S214447E1008B5FEF742F8FEF787F8FEF70BF9FEF7CB
S214447E2049F9FEF789F9FEF76DFAFEF7B1FAFEF75F
S214447E30EFFAFEF72BFBFEF767FBFEF787FBFEF732
S214447E40FBFBFEF72BFCFEF743FCFEF7C9FCFEF7F4
S214447E5033FDFEF7B1FDFEF72FFEFEF76FFEFEF78D
S214447E60ABFEFEF7E7FEFEF727FFFFF721F8FFF726
S214447E7051F8FFF781F8FFF7ABF8FFF72DF9FFF756
S214447E80C3F9FFF705FAFFF76FF9FFF72FFAFFF785
S214447E9047FAFFF757FAFFF76FFAFFF77BFAFEF752
S214447EA04DFFFFF777FCFFF7CBFDBDE80840FFF733
S214447EB08EBF114B11491B6810B5114C84F85433CE
S214447EC0104B1B6884F855330F4B186808F012FBA8
S214447ED00E4908F0CBFC07F067FF0CF06DFF08F086
S214447EE093FA0B4A94F858331278A4F8560362F37C
S214447EF0000384F8583310BDAC18402000C0234417
S214447F00E8834020A8184020A41840200AD7A33C61
S214447F10A11840200D4B0E4A1B780E4982F8603358
S214447F200D4B09781B7801F0010182F861330B4B45
S214447F301B785B0003F002030B4392F8621321F0B4
S214447F4003010B4382F86233704700BFA0184020F9
S214447F50E88340209E1840209F1840209D184020CB
S214447F600C4B0D4A1B780D4982F85C330C4B097850
S214447F701B7801F0030182F85D330A4B1B789B00A3
S214447F8003F00C030B430849097843EA011382F8CB
S214447F905E3370479C184020E88340209A1840205F
S214447FA09B1840209918402098184020114B12499D
S214447FB01B6810B5114C84F86433114B1B6884F865
S214447FC06533104B186808F095FA0F4908F04EFCD4
S214447FD007F0EAFE0CF0F0FE08F016FA0B4A94F8A6
S214447FE068331278A4F8660362F3000384F86833AF
S214447FF010BD00BF9418402000C02344E8834020AE
S214448000901840208C1840200AD7A33C881840205B
S2144480100D4B0E4A1B780E4982F86C330D4B09788B
S2144480201B7801F0010182F86D330B4B1B785B0023
S21444803003F002030B4392F86E1321F003010B4343
S21444804082F86E33704700BF87184020E88340208C
S2144480508518402086184020841840200C4B0D4A32
S2144480601B680D4982F870330C4B09781B6801F085
S214448070030182F871330A4B1B789B0003F00C0310
S2144480800B430849097843EA011382F87233704770
S21444809080184020E8834020791840207C184020EF
S2144480A0781840207718402008B5FFF727FAFFF7DE
S2144480B03FFAFFF77DF9FFF76DFAFFF78BFBFFF703
S2144480C0BBFAFFF7DFFAFFF701FCFFF719FCFFF7EF
S2144480D049FCFFF74BFDFFF7C5FDFFF7E9FDFFF74A
S2144480E0E8FEFFF717FFFFF73BFFFFF75FFFFFF7DB
S2144480F08FFFBDE80840FFF7B1BF074A0020074B93
S214448100D2F87811D2F87C219962DA62044B93E86B
S2144481100600FBF779BC00BFE88340206087402018
S21444812094844600194A1A4892F8843130B492F836
S214448130854180F82830C4F3010104F01C03C4F3DD
S21444814041140B4392F8861180F82930D2F88431D2
S214448150C3F3C135C1F30013C1F34111DB0143EA54
S2144481608503234380F82A3092F8873103F00703C7
S21444817041EA8301D2F88831C362064B80F82B105B
S214448180002093E8060030BCFBF73EBCE883402062
S214448190608740209C8446000B4A00200B4BD2F854
S2144481A08C119962B2F8901183F82C1092F89211BF
S2144481B092F8932183F82D1083F82E20044B93E8ED
S2144481C00600FBF721BC00BFE883402060874020C0
S2144481D0A4844600084B002093F8E431C3F300021D
S2144481E003F0FE031343054A82F82830044B93E811
S2144481F00600FBF709BC00BFE883402060874020A8
S214448200AC8446000D480E4AD0F8E8319362B0F884
S214448210EC319385B0F8EE31C3F30D0190F8EF31AD
S214448220002003F0C00382F82E1043EA112382F89C
S2144482302F30044B93E80600FBF7E6BBE883402068
S21444824060874020DC84460008B50A4B50200A4A22
S214448250D3F8A41193F8A831283211600821137179
S21444826004F066F8054B002093E80600BDE8084095
S214448270FBF7CABBE883402060874020B4844600AE
S214448280094B00200949D3F8AC2193F8B0318A62EF
S21444829003F0F002C3F30303134381F82F30044B77
S2144482A093E80600FBF7B0BBE88340206087402095
S2144482B0BC844600094B00200949D3F8B42193F8FE
S2144482C0B8318A6203F0F002C3F30303134381F820
S2144482D02F30044B93E80600FBF796BBE883402018
S2144482E060874020C4844600094B00200949D3F8DF
S2144482F0BC2193F8C0318A6203F0F002C3F303034F
S214448300134381F82F30044B93E80600FBF77CBBFD
S214448310E883402060874020CC8446000A4A0020F8
S2144483200A4BD2F8DC1192F8E021996283F82C20AB
S21444833083F82D2083F82E2083F82F20044B93E8CF
S2144483400600FBF761BB00BFE883402060874020FF
S214448350D4844600254A264992F8C431C3F3010022
S21444836003F0FC03034310B481F8283092F8C53177
S214448370C3F3010003F0FC03034392F8C60181F8FB
S2144483802930C0F3010400F00C0323438409C0F3EE
S214448390011081F82A3092F8C73103F003039B0199
S2144483A043EA8403034381F82B3092F8C83181F8BA
S2144483B02C3092F8C93103F03800C3F30203034368
S2144483C081F82D3092F8CA31C3F38300D2F8C8310D
S2144483D0C3F3833343EA0013002081F82F30054B60
S2144483E010BC93E80600FBF70FBB00BFE8834020B1
S2144483F060874020E48446000B490C4A91F8CC310F
S214448400C3F3010003F0FC030343002082F8283042
S21444841091F8CD31C3F3010382F82930044B93E835
S2144484200600FBF7F1BA00BFE8834020608740208F
S214448430EC844600084B002093F8D83103F004023D
S214448440C3F301031343054A82F82830044B93E8E8
S2144484500600FBF7D9BA00BFE88340206087402077
S214448460F48446001049114A91F8D031C3F3000011
S21444847003F0FE03034382F8283091F8D13103F029
S2144484807C00C3F301030343002082F82930D1F86B
S214448490D031C3F3CF335385D1F8D431D362044BB0
S2144484A093E80600FBF7B0BAE88340206087402094
S2144484B0FC84460019491A48D1F8442200F5FE5374
S2144484C010B41A6041F6C473B1F84822C25291F807
S2144484D04A22C2F3C103C2F341041B0143EA8403A4
S2144484E0C2F30004C2F34012234343EA821341F624
S2144484F0C672835491F84B32C3F38302B1F84A32BE
S214448500C3F3831343EA021341F6C772835401202C
S214448510044B10BC93E80600FBF776BAE883402089
S2144485206087402024854600264B274993F84C0212
S21444853001F5FE5210B500F0F004C0F303002043EA
S214448540107093F84D0200F07004C0F3030020430B
S21444855041F6C174085541F6C274D3F84C02C0F3D0
S214448560C130085541F6C374B3F84E02C0F3470011
S214448570085541F6C470B3F850420C5293F8520270
S21444858000F07C04C0F30100204341F6C67408554D
S21444859093F85302B3F85232C0F3C300C3F3C31381
S2144485A043EA001341F6C7700B540821142004F024
S2144485B028F8064B012093E80600BDE81040FBF778
S2144485C023BA00BFE8834020608740202C854600BD
S2144485D01149124B01F5FE52D3F8540210B5B3F8C4
S2144485E05842106041F6C47093F85A320C5203F065
S2144485F0F000C3F30303034341F6C7700B5408214A
S214448600152003F0FEFF064B012093E80600BDE864
S2144486101040FBF7F9B900BF60874020E88340204C
S2144486203485460015491648D1F88C3200F5FE527A
S21444863010B5136091F8903203F01E04C3F30003A0
S214448640234341F6C474035591F89132C3F343046B
S214448650B1F8903241F6C771C3F3431343EA0413A7
S21444866043540821162003F0CCFF064B012093E820
S2144486700600BDE81040FBF7C7B900BFE8834020BA
S214448680608740203C854600FFF7CCBF08B5FDF721
S21444869077FBF9F7E2F8FEF7C7F9BDE80840FFF7BD
S2144486A0C1BF084B012093F89432C3F3000203F091
S2144486B0FE031343044A1370044B93E80600FBF787
S2144486C0A3B900BFE883402020A740204485460045
S2144486D008B50E480E4B00F5FE52D3F8241293F814
S2144486E02832116003F0F001C3F303030B4341F651
S2144486F0C77143540821502003F083FF054B0120E3
S21444870093E80600BDE80840FBF77EB96087402042
S214448710E88340200485460008B50E480E4B00F515
S214448720FE52D3F82C1293F83032116003F0F00165
S214448730C3F303030B4341F6C77143540821512046
S21444874003F05FFF054B012093E80600BDE80840B0
S214448750FBF75AB960874020E88340200C854600E2
S21444876008B50E480E4B00F5FE52D3F8341293F873
S2144487703832116003F0F001C3F303030B4341F6B0
S214448780C77143540821602003F03BFF054B01208A
S21444879093E80600BDE80840FBF736B960874020FA
S2144487A0E88340201485460008B50E480E4B00F575
S2144487B0FE52D3F83C1293F84032116003F0F001B5
S2144487C0C3F303030B4341F6C771435408216120A6
S2144487D003F017FF054B012093E80600BDE8084068
S2144487E0FBF712B960874020E88340201C8546008A
S2144487F0174B184A03F5FE51B2F85C02088092F80B
S214448800601201F0F000C1F30301014341F6C27067
S214448810195441F6C37192F86102585441F6C47132
S214448820B2F86402585292F8681201F0F000C1F3AC
S2144488300301014341F6C6701954012092F86912A7
S21444884041F6C7729954044B93E80600FBF7DCB82C
S21444885060874020E88340204C854600174B184AE2
S21444886003F5FE51B2F86C02088092F8701201F0DB
S214448870F000C1F30301014341F6C270195441F6B6
S214448880C37192F87102585441F6C471B2F8740236
S214448890585292F8781201F0F000C1F303010143F4
S2144488A041F6C6701954012092F8791241F6C772FF
S2144488B09954044B93E80600FBF7A6B8608740201B
S2144488C0E883402054854600174B184A03F5FE516A
S2144488D0B2F87C02088092F8801201F0F000C1F3EE
S2144488E00301014341F6C270195441F6C370D2F8ED
S2144488F084121954090A41F6C470195492F888121D
S21444890001F0F000C1F30301014341F6C670195467
S214448910012092F8891241F6C7729954044B93E8A1
S2144489200600FBF771B800BF60874020E88340200C
S2144489305C8546002848294990F8003201F5FE52E5
S21444894070B5C3F3010403F0FC032343137090F89B
S2144489500132C3F3010403F0FC03234341F6C1741C
S2144489600B5541F6C27390F802422501A609C4F39A
S2144489700114CD5490F8035205F00303C5F3810562
S2144489801B0143EA8603234341F6C37443EA851333
S2144489900B5541F6C47390F80442CC5441F6C57462
S2144489A090F8053290F806021D01C3F3031300F055
S2144489B00F000D5543EA001341F6C7700B540821C7
S2144489C04FF4AE6003F01DFE054B012093E806000D
S2144489D0BDE87040FBF718B8E88340206087402025
S2144489E0848546002D4991F8080238B5C0F3001531
S2144489F000F008032A4C43EA4513C0F3020504F585
S214448A00FE522B43C0F34015C0F3801043EA85134F
S214448A1043EAC01341F6C1701370B1F80832C3F389
S214448A20C713235441F6C270D1F80832C3F3C73390
S214448A30235491F80B02C0F3C103C0F34105C0F3BD
S214448A4041101B0143EA8503B1F80A52C5F3C11528
S214448A502B4343EA801341F6C370235441F6C47053
S214448A6091F80C329B00235491F80D32C3F38300E3
S214448A70B1F80C3241F6C771C3F3831343EA0013CB
S214448A804FF4B0606354082103F0BBFD054B01204E
S214448A9093E80600BDE83840FAF7B6BFE8834020BE
S214448AA0608740208C8546001849194891F8203242
S214448AB000F5FE5210B5C3F3010403F0FC03234350
S214448AC0137091F8213203F03C04C3F301032343AB
S214448AD041F6C174035591F82232C3F38304D1F8A6
S214448AE0203241F6C771C3F3833343EA0413435435
S214448AF0082140F2855003F084FD064B012093E89C
S214448B000600BDE81040FAF77FBF00BFE883402068
S214448B1060874020948546001149124B01F5FE5269
S214448B20D3F8100210B5B3F81442106041F6C4707E
S214448B3093F816320C5203F0F000C3F303030343D6
S214448B4041F6C7700B5408214FF4B26003F059FD48
S214448B50054B012093E80600BDE81040FAF754BFE1
S214448B6060874020E8834020A4854600104810B51E
S214448B70104C90F8183204F5FE52137090F81C32DC
S214448B8003F00F0190F81B3240F29550C3F3830371
S214448B9043EA011341F6C7716354082103F031FDDB
S214448BA0054B012093E80600BDE81040FAF72CBFB9
S214448BB0E883402060874020AC854600084B01206F
S214448BC0084993F8983203F01C02C3F30103134395
S214448BD041F6C3728B54044B93E80600FAF714BF6D
S214448BE0E88340206087402064854600084B41F671
S214448BF0C271B3F89C22074BC2F30120585441F685
S214448C00C37101205A54044B93E80600FAF7FCBE9D
S214448C10E8834020608740206C854600054B012051
S214448C20054A93F8A0321B011370044B93E80600E0
S214448C30FAF7EABEE883402020A740207485460021
S214448C40074B41F6C1720749012093F8A43203F05A
S214448C5007039B008B54044B93E80600FAF7D4BEF4
S214448C60E8834020608740207C854600074B41F6D9
S214448C70C1720749012093F8A832C3F303038B5407
S214448C80044B93E80600FAF7BFBE00BFE8834020D3
S214448C90608740209C8546000D4843F65872B0F8DD
S214448CA0C41208B549BA0B4B99521A4490F8C612E6
S214448CB043F65A70C90119540321322003F038FB95
S214448CC0054B022093E80600BDE80840FAF79CBE30
S214448CD0E883402060874020B4854600114B43F625
S214448CE05870114AB3F8E01249BA10B5115243F617
S214448CF05A74B3F8E21293F8E43249BA03F0010323
S214448D00115343F65C719B015354024405214020A1
S214448D1003F097F9054B022093E80600BDE810409F
S214448D20FAF772BEE883402060874020BC85460040
S214448D303048314A90F8B03290F8AC1270B543F6E9
S214448D40587590F8B342535543F65973D15443F685
S214448D505A71D0F8AC32C3F34F235BBA5352C4F3C0
S214448D60801304F0100141EAC301C4F3010319431C
S214448D7090F8AD3203F0010341EA4311C4F3810392
S214448D8004F0200441EA831143F65C73D15490F80E
S214448D90B412C1F3800601F00803C1F3010143EAAB
S214448DA006130B4390F8B212D0F8B0022343CC0912
S214448DB0C1F3801143EA841343F65D741355C0F33C
S214448DC00D2343F65E74C0F305409B0010556420A3
S214448DD043EA410343F65F7153542A44082103F09F
S214448DE0A7FA064B022093E80600BDE87040FAF75F
S214448DF00BBE00BFE883402060874020C485460001
S214448E001F4843F658721F4BB0F8DA12C1F3C71125
S214448E1070B5995443F65974D0F8D8121A44B0F839
S214448E20D852C1F3C731C5F30526195590F8DD422B
S214448E3004F08001C4F38014314343F65A769955BE
S214448E4043F65B715D54B0F8DC5290F8D912C5F322
S214448E50052001F04001014343F65C7041EAC41129
S214448E60195443F65D716A205D54062103F060FA96
S214448E70054B022093E80600BDE87040FAF7C4BDEF
S214448E80E883402060874020CC85460038B52C4B8C
S214448E9043F658702B4AB3F8B812B3F8C05249BADE
S214448EA0115293F8BE12CC09C5F3032141EA0411CA
S214448EB093F8C142C4F3001441EA441193F8BB4208
S214448EC0C4F3800441EA841193F8BD42C4F3800499
S214448ED041EAC41143F65A74115543F65B71B3F82C
S214448EE0BA42555443F65C71C4F30905C4F3870487
S214448EF05454B3F8BC12D3F8BC32C1F30904C1F3DA
S214448F00051141EA851143F65D755155C3F3CB21EE
S214448F10C3F3C34343EA041343F65E74135543F65C
S214448F205F73D15402440821702003F001FA064BC3
S214448F30022093E80600BDE83840FAF765BD00BF56
S214448F40E883402060874020D4854600284A43F67C
S214448F5058702849B2F8F8325BBA30B40B5243F62C
S214448F605A73B2F8FA02B2F8FC52C0F30904C0F3DA
S214448F708700C854C5F3012092F8FB3203F004037B
S214448F80034392F8FD02C0F3800043EAC00392F81C
S214448F90FE02C0F3401043EA001392F8000300F0C8
S214448FA0010043EA401343F65B7043EA841343F6F6
S214448FB05D740B5443F65C73D2F8FC02CD54C0F394
S214448FC0C923B2F8FE22C0F347309B0108559009E6
S214448FD043EA923343F65E728B5443F65F73C85447
S214448FE00220054B30BC93E80600FAF70DBD00BFDF
S214448FF0E883402060874020DC854600104843F6DE
S2144490005871104A08B5B0F8EC325BBA535290F82F
S214449010EE3203F00100C3F3400343EA400343F651
S2144490205A7013540A444FF44470032103F009F869
S214449030054B022093E80600BDE80840FAF7E4BC76
S214449040E883402060874020E4854600134843F682
S2144490505872134BB0F8E81249BA10B599521A44EC
S21444906090F8EA1243F65A70C1F301041C54C1F353
S214449070031443F65B70C1F381011C5443F65C70E1
S214449080195405214FF4547002F0DBFF054B0220BF
S21444909093E80600BDE81040FAF7B6BCE8834020E3
S2144490A060874020EC854600254943F65872B1F85F
S2144490B0F00238B540BA234B91F8F34298521A441A
S2144490C0D1F8F40204F00105C4F34404C0F3C530F7
S2144490D040EAC51043F65A75585543F65B75B1F8E1
S2144490E0F402C0F34510585543F65C7591F8F40203
S2144490F0C0F304005855B1F8F602C0F3022500F454
S214449100FC6045EAC40443F65D755C5591F8F54247
S214449110C4F3C304204343F65E74185591F8F20230
S21444912043F65F71585408214FF4617003F000F918
S214449130054B022093E80600BDE83840FAF764BCC5
S214449140E883402060874020F4854600094943F67A
S2144491505870094AD1F8D0321BBA13500220D1F8BD
S214449160D43243F65C711BBA5350044B93E8060062
S214449170FAF74ABCE883402060874020FC854600D6
S2144491800E4845F6F062B0F8281308B549BA0C4BB9
S21444919099521A4490F82A1345F6F260C1F3000136
S2144491A019540321332003F0C3F8064B032093E8F5
S2144491B00600BDE80840FAF727BC00BFE883402015
S2144491C06087402004864600114B45F6F060114AFD
S2144491D0B3F8181349BA10B5115245F6F264B3F809
S2144491E01A1393F81C3349BA03F00103115345F696
S2144491F0F4619B01535402440521402002F07EFF53
S214449200054B032093E80600BDE81040FAF7FCBB84
S214449210E8834020608740200C8646002248234A44
S21444922090F8101338B590F8143345F6F064135597
S21444923045F6F163D15445F6F261D0F81033C3F3E2
S2144492404F235BBA535290F81513C1F34013C1F33E
S21444925080151B0143EAC503C1F341052B4390F82F
S214449260115305F0010543EA4513C1F3C10501F066
S214449270010143EA851345F6F4655355D0F8143393
S2144492806520C3F3C13343EA811145F6F563D154EF
S2144492902244082103F04CF8054B032093E80600CB
S2144492A0BDE83840FAF7B0BBE883402060874020EA
S2144492B01486460038B52C4B45F6F0602B4AB3F876
S2144492C00413B3F80C5349BA115293F80A13CC0951
S2144492D0C5F3032141EA041193F80D43C4F3001483
S2144492E041EA441193F80743C4F3800441EA8411E5
S2144492F093F80943C4F3800441EAC41145F6F26482
S214449300115545F6F361B3F80643555445F6F461F2
S214449310C4F30905C4F387045454B3F80813D3F8C4
S2144493200833C1F30904C1F3051141EA851145F632
S214449330F5655155C3F3CB21C3F3C34343EA041342
S21444934045F6F664135545F6F763D15402440821AE
S214449350712002F0EDFF064B032093E80600BDE8BB
S2144493603840FAF751BB00BFE8834020608740206E
S2144493701C86460008B5FEF7C0FEFEF7D3FEFEF791
S2144493800BFFFEF727FFFEF75FFFFEF779FFFEF7BA
S214449390C5FFFEF7DFFFFFF72FF8FFF74BF8FFF7A1
S2144493A061F8FEF72FFFFFF785F8FFF7BDF8FFF7E4
S2144493B00FF9FFF776F9FFF7AFF9FFF7D1F9FFF7A3
S2144493C0F3F9FFF785F9FFF713FAFFF747FAFFF7C4
S2144493D07BFAFFF7AFFAFFF705FBFFF79DFBFFF7B6
S2144493E063FBFFF7C3FBFFF7E9FBFFF7FFFBFFF762
S2144493F015FCFFF725FCFFF739FCFFF747FDBDE8F2
S2144494000840FFF757BF284A45F6F0602749B2F8A8
S21444941048335BBA30B40B5245F6F263B2F84A03AB
S214449420B2F84C53C0F30904C0F38700C854C5F3DC
S214449430012092F84B3303F00403034392F84D03A0
S214449440C0F3800043EAC00392F84E03C0F34010D2
S21444945043EA001392F8500300F0010043EA401335
S21444946045F6F36043EA841345F6F5640B5445F633
S214449470F463D2F84C03CD54C0F3C923B2F84E2358
S214449480C0F347309B010855900943EA923345F6AA
S214449490F6628B5445F6F763C8540320044B30BC3D
S2144494A093E80600FAF7B0BAE88340206087402085
S2144494B024864600104845F6F061104A08B5B0F8D0
S2144494C024335BBA535290F8263303F00100C3F3B7
S2144494D0400343EA400345F6F26013540A444FF40B
S2144494E04470032102F00AFE054B032093E806006D
S2144494F0BDE80840FAF788BAE883402060874020F1
S2144495002C864600134845F6F062134BB0F82013F9
S21444951049BA10B599521A4490F8221345F6F260A7
S214449520C1F301041C54C1F3031445F6F360C1F3BC
S21444953081011C5445F6F460195405214FF45470C7
S21444954002F0DCFD054B032093E80600BDE810401E
S214449550FAF75ABAE88340206087402034864600AB
S214449560254945F6F062B1F8400338B540BA234B76
S21444957091F8434398521A44D1F8440304F0010541
S214449580C4F34404C0F3C53040EAC51045F6F2655A
S214449590585545F6F365B1F84403C0F3451058559D
S2144495A045F6F46591F84403C0F304005855B1F801
S2144495B04603C0F3022500F4FC6045EAC40445F6BD
S2144495C0F5655C5591F84543C4F3C304204345F61A
S2144495D0F664185591F8420345F6F7615854082145
S2144495E040F2853002F0A4FE054B032093E80600C3
S2144495F0BDE83840FAF708BAE88340206087402040
S2144496003C86460008B5FFF74FFDBDE80840FFF727
S214449610A7BF08B5F8F723F9FEF7D2FBBDE8084024
S214449620FFF7F0BF094945F6F060094AD1F83833E8
S2144496301BBA13500320D1F83C3345F6F4611BBAE9
S2144496405350044B93E80600FAF7DEB9E88340200B
S2144496506087402044864600114B47F68860114A8E
S214449660B3F8541349BA10B5115247F68A64B3F89E
S214449670561393F8583349BA03F00103115347F687
S2144496808C619B01535402440521402002F094FD12
S214449690054B042093E80600BDE81040FAF7B4B939
S2144496A0E8834020608740204C864600104847F6B2
S2144496B08861104A08B5B0F860335BBA535290F8E4
S2144496C0623303F00100C3F3400343EA400347F622
S2144496D08A6013540A444FF44470032102F06CFD2C
S2144496E0054B042093E80600BDE80840FAF78CB919
S2144496F0E88340206087402054864600134847F657
S2144497008862134BB0F85C1349BA10B599521A44A0
S21444971090F85E1347F68A60C1F301041C54C1F303
S214449720031447F68B60C1F381011C5447F68C60E2
S214449730195405214FF4547002F03EFD054B0420A5
S21444974093E80600BDE81040FAF75EB9E883402087
S214449750608740205C86460008B50A4B49F622627C
S21444976009494020B3F866335BBA8B520521074A51
S21444977002F080FD064B052093E80600BDE808404D
S214449780FAF742B9E883402060874020802541208C
S21444979064864600134849F62062134BB0F87013AB
S2144497A049BA10B599521A4490F8721349F6226091
S2144497B0C1F301041C54C1F3810449F62360C1F388
S2144497C003111C5449F62460195405214FF454706F
S2144497D002F050FD054B052093E80600BDE8104016
S2144497E0FAF712B9E8834020608740207486460022
S2144497F0104849F62061104A08B5B0F86C335BBA95
S214449800535290F86E3303F00100C3F3400343EA27
S214449810400349F6226013540A444FF4447003212B
S21444982002F028FD054B052093E80600BDE80840F5
S214449830FAF7EAB8E8834020608740206C86460002
S21444984008B5FFF729FAFFF749FAFFF771FAFFF769
S214449850D7FAFFF7D3FBFFF7F9FBFFF791FCFFF7C7
S214449860B3FCFFF7DBFCFFF725FEFFF74BFEFFF7E5
S214449870F3FEFFF71BFFFFF741FFFFF76DFFFFF710
S214449880B7FFBDE80840FFF785BF08B5FCF7ECFA1C
S214449890F7F7C1FFFEF708FCBDE80840FFF7D0BF66
S2144498A07047704770477047064AB2F82032B2F89D
S2144498B0681003F44043C1F30D010B43A2F8203271
S2144498C0704700BFE8834020044BB3F81221A3F846
S2144498D02422B3F80C21A3F826227047E8834020BC
S2144498E0044BB3F8A620A3F82C22B3F8A020A3F880
S2144498F02E227047E883402070477047054BB3F8E4
S2144499006C21A3F83422D3F86821C2F30F12A3F8CB
S21444991036227047E8834020054BB3F87421A3F8F9
S2144499203C22D3F87021C2F30F12A3F83E227047AC
S214449930E8834020054BB3F86C21A3F8B421D3F850
S2144499406821C2F30F12A3F8B6217047E88340207B
S214449950054BB3F87421A3F8BC21D3F87021C2F3A5
S2144499600F12A3F8BE217047E883402008B5FFF7DE
S214449970E1FFFFF7EDFFFFF797FFFFF7A5FFFFF7C0
S214449980AFFFFFF7BBFFBDE80840FFF7C5BF08B50C
S214449990FCF790F9F7F740FFFEF73AFAFFF7E6FFD1
S2144499A0BDE80840FFF7E6BC70477047704770470D
S2144499B00B4AD2F8C431D2F894101B0DC1F31301EC
S2144499C01B050B43D2F89810C2F8C43101F47F113A
S2144499D0D2F8C83123F47F130B43C2F8C83170471A
S2144499E0E883402008B5F9F7ADF8BDE80840F8F735
S2144499F0D5BA7047F7F70DBFFFF747BFFFF7C7BFA6
S214449A00FBF716BA7047074A1378632B96BF0133A1
S214449A100023DBB21370044A136801331360FEF765
S214449A2035BE00BF70484120E820402008B5FAF70C
S214449A3007F8BDE8084002F0E5B808B503F0D4F9E5
S214449A40FFF7E7FD4CF24053044AD058B0FA80F092
S214449A50BDE808404009F9F7EFB800BF7448412014
S214449A60014900201EF0B0BB20AB460000201EF08B
S214449A70A3BB0022114610461EF0A2BB704700BF8F
S214449A802DE9F04FB84CD9B0D4E904230DF58078CD
S214449A90CDE92A23DDE92A01D4E9502306F026F845
S214449AA0A1A3D3E9002306F0D7F906460F46A0A3A0
S214449AB0D3E90023D4E9520106F0CEF902460B4618
S214449AC03046394606F012F89BA3D3E9002306F045
S214449AD0EDFA95A3D3E90023D4E94856D4E94AAB32
S214449AE0CDE94C23CDE9005695A3D3E90023D4E928
S214449AF04C45CDE91001CDE9522300200022002335
S214449B009A49CDE9024546AC0325CDE94601CDE95F
S214449B104823CDE94A23CDE94E01CDE95023CDE98A
S214449B205423CDE95601CDE90A01CDE90623A146E1
S214449B30504659460834D9E9062306F08DF90646B8
S214449B400F46D9E90023DDE9000106F085F902460F
S214449B500B463046394605F0C9FF06460F46D4E95B
S214449B600A23DDE9020106F077F902460B46304641
S214449B70394605F0BBFF013DE8E80201D7D17A4CEF
S214449B80236D0293636D0493DDE94223DDE940AB24
S214449B90CDE90023DDE94423CDE90823DDE90801C6
S214449BA00022002306F058F9002280468946002306
S214449BB0DDE9000106F050F952465B4605F096FF93
S214449BC042464B4605F092FF02460B4602980499DD
S214449BD005F08AFF002206460F46002350465946A3
S214449BE006F03AF9DDE9002305F080FF42464B468D
S214449BF005F07CFF02460B46DDE9100105F074FFD4
S214449C0002460B46CDE90C234FA3D3E9002306F0C6
S214449C1023F980468946304639464DA3D3E9002386
S214449C2006F01AF902460B464046494605F05EFFE2
S214449C3052465B4605F05AFF00220023C4E9480119
S214449C403046394606F008F98046894642A3D3E9A9
S214449C500023DDE90C0106F0FFF802460B464046B9
S214449C60494605F043FFDDE9002305F03FFF024681
S214449C700B46CDE91201C4E94A233046394638A397
S214449C80D3E9002306F0E8F806460F4600220023F0
S214449C90DDE90C0106F0E0F802460B46304639464C
S214449CA005F024FFDDE9082305F020FFD4E91A2354
S214449CB0D4E902ABC4E94C01CDE91823504600224E
S214449CC02B4B594606F04EFB002840F00182D4E95F
S214449CD01267D4E90C453046394622462B4606F0F0
S214449CE037FB08B926462F4600224FF08043DDE96D
S214449CF0180106F019FB0022002800F0EC8100232E
S214449D003046394606F0A8F802460B46CDE9082305
S214449D10154BD3E9A44522462B4605F0E5FE0646F8
S214449D200F4627E0AFF30080FCA9F1D24D62603FB6
S214449D30D9D6F61FCE4EE43F2DBA9CBB926FE43F75
S214449D4049DC63E9431794BF7B14AE47E17A843F0A
S214449D50E71DA7E8482ED33F386744696FF0EF3FC6
S214449D603CBD5296218EB5BFF80D42200000F03F10
S214449D7000004940ACA3D3E9002306F0FDFA0028CE
S214449D8000F0AB8120462946A7A3D3E9002305F07B
S214449D90ADFECDE90801DDE90834B74E0022C6E938
S214449DA0A434D6E95445B54B2046294606F0E4FA91
S214449DB0002840F0A4810022B14B2046294606F0F4
S214449DC0BDFA002840F09E8196F8EA320BB1C6E907
S214449DD05645A94B20462946D3E9566732463B4664
S214449DE005F082FE04460D4691A3D3E9002306F00F
S214449DF0C3FA002840F08981204629468EA3D3E939
S214449E00002306F09BFA002840F0838122462B4626
S214449E103046394605F06AFE02460B46CDE92E2307
S214449E2087A3D3E9002306F017F806460F460BF03F
S214449E300BF804460D46304639460AF077FF914BF8
S214449E4006460F4620462946D3E9002306F004F882
S214449E5004460D46304639467BA3D3E9002305F035
S214449E60FBFF0022002305F0F7FF02460B46204680
S214449E70294605F03BFE76A3D3E9002305F0ECFF24
S214449E8075A3D3E9002305F0E7FF00227E4B044682
S214449E900D4606F071FA002840F03F810022002368
S214449EA02046294606F04AFA08B100240025724B9B
S214449EB093F8EB220AB1C3E95845D3E958672046DC
S214449EC0294632463B4605F00FFE04460D4664A33B
S214449ED0D3E9002306F050FA002840F021812046BA
S214449EE0294661A3D3E9002306F028FA002840F067
S214449EF01B8122462B463046394605F0F7FD02467E
S214449F000B46CDE93A235AA3D3E9002305F0A4FF30
S214449F10594BCDE93001D3E90E45D3E95A122046D0
S214449F200023CDE900120022294606F0FDF9002858
S214449F3000F0FE80002200230298049906F008FAF6
S214449F4050B10022514B5046594606F00BFA18B110
S214449F5000230024CDE90034474CD4E90023CDE95E
S214449F600C2394F8E832002B40F0458140F201136C
S214449F70A4F8E832DFF800810022454DDDE90634D6
S214449F80DDE90001C8E9C434424B06F0CDF9031EAE
S214449F904FF00002594618BF0123504616933E4BD5
S214449FA006F0D6F9041E4FF000024FF0804318BF67
S214449FB00124DDE9080106F0CBF9169B00280CBF06
S214449FC02046601C0024184405F0DCFE0022334B77
S214449FD005F08CFDD8E9C62305F088FD0022304BF9
S214449FE006F0C0F90022D8E9B267002800F02481C0
S214449FF000233046394606F097F918B1DDE90623C2
S21444A000C8E9B8231C4EDDE90A23C6E9B445D6E9B7
S21444A010B845C6E9B223204600221E4B294606F020
S21444A0208DF900284BD03DE0FCA9F1D24D62703F3B
S21444A030FCA9F1D24D62603FFCA9F1D24D6260BFEB
S21444A040399D52A246DF913F407EFCF8F14B7B405F
S21444A050E3A59BC420B0D23F578C22C76075B53F5A
S21444A060FCA9F1D24D62903F7B14AE47E17AC4BF5F
S21444A0709A9999999999E93FF80D42200000204011
S21444A080000020C0C088460000004E4000005940F2
S21444A09000408F4000000840000034400000F03F7D
S21444A0A00000144020462946DDE93023C6E9B6239D
S21444A0B07DA3D3E9002305F019FDC6E9B801DDE91F
S21444A0C00A34C6E9C43400238B4CCDE90E342DE162
S21444A0D00026002708E6894B12E675A3D3E9002339
S21444A0E03046394606F02AF900283FF454AE204656
S21444A0F0294671A3D3E9002305F0F6FC49E600247B
S21444A1007F4D61E600247F4D5EE66DA5D5E90045AA
S21444A1107CE66DA5D5E9004578E600247A4DC6E68A
S21444A1206BA5D5E90045E4E66BA5D5E90045E0E630
S21444A130DDE9000106F040F903283FF60DAFDFE8FD
S21444A14000F002452845002200230298049906F0B0
S21444A150FFF800283FF400AF0022684B204629460B
S21444A16006F0E2F8002842D10022684B20462946F1
S21444A17006F0DAF800283AD100224FF08043204611
S21444A180294606F0D1F800283FF4E6AECDE900456E
S21444A190E2E6002200230298049906F0D9F8002843
S21444A1A03FF4DAAE00225A4B5046594606F0DAF8E7
S21444A1B000283FF4D1AE0022504B2046294606F0F4
S21444A1C0B3F80028E2D10022504BD8E700224FF0E3
S21444A1D080432046294606F0A7F800283FF4BCAE44
S21444A1E0002200230298049906F0B2F8CBE7002335
S21444A1F04FF08044AEE694F8E932012B0FD10022AA
S21444A200444BDDE90C0106F099F818B1022384F8B2
S21444A210E932AFE6DDE90623C4E9C623AAE630A35D
S21444A220D3E90023DDE90C0106F0A6F808B10123C2
S21444A230EDE7DDE90A23EFE7304B3046394606F0D2
S21444A24073F8002801F03F81D8E9B623D8E9100115
S21444A25006F088F8002861D0D8E9B44522A3D3E9AB
S21444A26000232046294605F0F7FD02460B462046C5
S21444A270294605F039FC04460D461DA3D3E90023C0
S21444A28006F05CF828B9C8E9B445234BD3E9B4349E
S21444A2901BE7DDE90634C8E9B434C8E9B234C8E992
S21444A2A0B634C8E9B834F0E77B14AE47E17A743F75
S21444A2B0FCA9F1D24D6280BFFCA9F1D24D62803F29
S21444A2C0FCA9F1D24D62603FFCA9F1D24D6260BF59
S21444A2D0FCA9F1D24D62903F7B14AE47E17AC4BFED
S21444A2E00000000000C062409A9999999999A93F44
S21444A2F07B14AE47E17A843F00408F400000F03F35
S21444A30000002040000020C000004E4000000840EE
S21444A31000005940000049C0F80D4220DDE90A23F8
S21444A320C8E9B445C8E9C423CDE90E45049C02985F
S21444A33024F000410024B6A3D3E9002305F0FEFF31
S21444A340002841F0C480C24DDFF80C83B2A3D3E9A1
S21444A3500023DDE9100105F07FFD02460B46002090
S21444A360002105F0C1FB22462B4605F075FD02464A
S21444A3700B46CDE92C230022B64B05F06DFDA8A371
S21444A380D3E90023CDE93201D8E95C0105F064FD48
S21444A39006460F46A4A3D3E90023DDE92C0105F0C5
S21444A3A05BFD02460B463046394605F09FFB0646A3
S21444A3B00F46D8E95E23DDE9320105F095FB00221D
S21444A3C0002305F049FD02460B463046394605F063
S21444A3D08DFB02460B46CDE91A2395A3D3E9002309
S21444A3E005F0CAFF002841F0758093A3D3E9002303
S21444A3F0DDE91A0105F0A2FF002841F07080DDE98E
S21444A4001A23CDE91423DDE914232046294605F012
S21444A41023FD914B04460D46D3E9A66732463B4698
S21444A42005F062FB00224FF080438046894605F0E3
S21444A430A3FF0022002801F057804FF080433046A7
S21444A440394605F053FB04460D46834B0022C3E9C8
S21444A450A645DDE90001814B05F066FF002801F0C2
S21444A460558000207A4922462B4605F0F5FC0246E4
S21444A4700B46CDE90A230022002305F073FF18B9E2
S21444A48000230024CDE90A3473490022744BD1E9F1
S21444A490600105F0E1FC0022724B05F0DDFC002271
S21444A4A004460D466A4BDDE9000105F03DFF169B68
S21444A4B000284FF000022046294608BF1E466A4B35
S21444A4C018BF4FF0FF3605F057FF002841F02280B2
S21444A4D0002200232046294605F030FF08B1002418
S21444A4E00025304605F04EFC22462B4605F0B4FCCB
S21444A4F0594B80468946D3E9A84522462B4605F063
S21444A500F3FA0022554B06460F4605F035FF002267
S21444A510002801F00380514B2046294605F0E6FA10
S21444A520804689464C4B002240464946C3E9A889A2
S21444A5304D4B05F021FF002841F000800022002307
S21444A5404046494605F0FAFE18B14FF000084FF071
S21444A550000900224FF08043DDE9180105F0E4FECF
S21444A560002800F0F1870022404B0298049905F039
S21444A57073FC06460F4632A3D3E9002305F0FCFEDF
S21444A580002840F0E987002200233046394605F08B
S21444A590D5FE08B10026002700222D4BDFF8B8A0D0
S21444A5A0DDE9080105F0DEFE48B927A3D3E9002318
S21444A5B0DAE9320105F0D6FE002800F0E7870022EB
S21444A5C02B4BDAE910452046294605F0CBFE0028F9
S21444A5D000F0DC8712A3D3E90023DDE9100105F07F
S21444A5E0C1FE002800F0D2870022224B029804992C
S21444A5F005F0B8FE002800F0C98700221C4B304600
S21444A600394605F0A5FE002800F0C08734E000BFB8
S21444A6109A9999999999B93F00000000007097401B
S21444A6209A9999999999C93FEC51B81E85EBB13FCF
S21444A63000000000008AAB40000000000088A3C071
S21444A640000000000088A3407B14AE47E17A843FB4
S21444A6500000F03F00407F40F80D422000000840D4
S21444A6600000B03F000054C000408F4000005940F6
S21444A670000024400000F83FDAE9B023DAE9080194
S21444A680CDE90623ACA3D3E9002305F0E5FBDDE9D9
S21444A690122305F02BFAAAA3D3E9002305F0DCFB2A
S21444A6A002460B462046294605F000FD04460D4664
S21444A6B00022C14BCAE94E4505F05EFE002800F074
S21444A6C05B870022BD4B2046294605F037FE00280E
S21444A6D000F0528720462946DDE9062305F004FAB1
S21444A6E021F0004CDDE90623614605F0DFFC96A325
S21444A6F0D3E9002305F022FE002800F03D8794A30A
S21444A700D3E90023DDE9060105F0A6FB92A3D3E9CD
S21444A7100023CDE912012946204605F09DFB02465A
S21444A7200B46DDE9120105F0E1F902460B46CAE99B
S21444A730B023DDE9062305F0D7F921F000450022D1
S21444A7409F4B294605F0FAFD002800F00A870123AE
S21444A7508AF8EE329B4B00204FF08041C3E9E0017B
S21444A760984CD4E9B023C4E9BC67C4E9DE23C4E901
S21444A770DA677BA3D3E90023DDE90A01C4E9CC897F
S21444A78005F06AFB78A3D3E9002305F08FFC00228A
S21444A7900023C4E9CE01DDE9000105F0C5FD064607
S21444A7A0002840F0FA8600224FF08043DDE900019D
S21444A7B005F0BAFD58B9844B0022DDE9000105F0E6
S21444A7C0B3FD169B00280CBF1E464FF0FF360022F2
S21444A7D07E4BDDE9080105F03FFB65A3D3E9002382
S21444A7E005F064FC60A3D3E9002305F035FB0022A2
S21444A7F0774B05F031FB60A3D3E9002305F056FC04
S21444A80004460D46304605F0BDFA02460B46204641
S21444A810294605F021FB02460B46CDE90A23694B3F
S21444A820D3E9AA4522462B4605F05EF906460F466E
S21444A83053A3D3E9002305F09FFD002800F0B0861B
S21444A840204629464EA3D3E9002305F04FF9CDE927
S21444A8500A015C4CDDE90A23DDE90A01C4E9AA23BE
S21444A860D4E9622305F042F947A3D3E9002305F06F
S21444A870F3FA06460F4646A3D3E90023D4E9640117
S21444A88005F0EAFA02460B463046394605F02EF9FC
S21444A89041A3D3E9002305F009FC02460B46CDE963
S21444A8A00623D4E9662305F01FF90022474B05F03A
S21444A8B0D3FAD4E9682305F017F902460B46CDE9E6
S21444A8C01C23D4E96A2305F00FF900223F4B05F018
S21444A8D0C3FAD4E96C2305F007F902460B46CDE9E2
S21444A8E01E23D4E96E2305F0FFF80022374B05F00B
S21444A8F0B3FAD4E9702305F0F7F829A3D3E9002383
S21444A900CDE93401DDE9060105F0A6FA804689461C
S21444A91025A3D3E90023DDE91C0105F09DFA424650
S21444A9204B4605F0E3F806460F4621A3D3E9002339
S21444A93050E000BFAFF300807B14AE47E17A843F1B
S21444A9408462BF15623E973F9A9999999999C93FEF
S21444A9505C8FC2F5285CEF3F7B14AE47E17A943FA8
S21444A9600E9F7422C154D13F5C8FC2F528DC274029
S21444A970000000000020AC40B46155D0CC38FB3F0A
S21444A9809A9999999999D93FFCA9F1D24D62603F19
S21444A990B428207983A6BA3F54434F56A8ACBB3F4D
S21444A9A09A999999999963409A99999999996A40E3
S21444A9B0CDCCCCCCCCCC354000407F4000409F40F2
S21444A9C000001440F80D42200000F03F00408F4045
S21444A9D000004E40DDE91E0105F03EFA02460B46F5
S21444A9E03046394605F082F8DDE9342305F07EF832
S21444A9F0BFA3D3E9002305F02FFAD4E97223CDE9A7
S21444AA0020011046194605F071F8DDE9202305F0CB
S21444AA106DF8D4E9382305F069F8B7A3D3E90023E1
S21444AA2005F01AFA06460F46B5A3D3E90023D4E93F
S21444AA30740105F011FA02460B463046394605F0D5
S21444AA4055F806460F46B0A3D3E90023D4E93C01A3
S21444AA5005F002FA02460B463046394605F044F8FD
S21444AA60ABA3D3E9002305F021FB02460B46CDE910
S21444AA702223D4E9762305F039F8A7A3D3E90023A3
S21444AA8005F0EAF906460F46A5A3D3E90023D4E920
S21444AA90780105F0E1F902460B463046394605F0A2
S21444AAA025F8A1A3D3E9002305F000FBDDE90C2338
S21444AAB0CDE93601DDE9060105F016F80022B44B6F
S21444AAC004460D4605F058FC002840F07C85204698
S21444AAD0294697A3D3E9002305F030FC002840F02C
S21444AAE085850022AB4B2046294605F045FC0028C8
S21444AAF000F06D850022A74B2046294604F0F4FF5B
S21444AB0082468B46A44CDDE90601D4E97A2304F058
S21444AB10EBFF0022A14B05F09FF9D4E97C2304F017
S21444AB20E3FF02460B46CDE92423D4E97E2304F012
S21444AB30DBFF0022994B05F08FF9D4E9802304F01B
S21444AB40D3FF02460B46CDE92623D4E9822304F0FC
S21444AB50CBFF0022914B05F07FF9D4E9842304F01F
S21444AB60C3FF75A3D3E90023CDE93801DDE9240109
S21444AB7005F072F942464B4604F0B8FF06460F46C7
S21444AB806FA3D3E90023DDE9260105F065F9024603
S21444AB900B463046394604F0A9FFDDE9382304F075
S21444ABA0A5FF53A3D3E9002305F056F9D4E9AC2313
S21444ABB004F09AFF02460B46CDE93C23D4E98623AB
S21444ABC004F094FF54A3D3E9002305F045F9064660
S21444ABD00F465DA3D3E90023D4E9880105F03CF988
S21444ABE002460B463046394604F080FF58A3D3E964
S21444ABF0002305F05BFAD4E98A23CDE91201104616
S21444AC00194604F073FFDDE9122304F06FFFD4E91C
S21444AC10402304F06BFF50A3D3E9002305F01CF94E
S21444AC2006460F464EA3D3E90023D4E98C0105F02B
S21444AC3013F902460B463046394604F057FF06469B
S21444AC400F4649A3D3E90023D4E9440105F004F9A7
S21444AC5002460B463046394604F046FF44A3D3E941
S21444AC60002305F023FA00224D4BCDE92801029833
S21444AC70049905F063FB002840F0C2840022484B48
S21444AC800298049904F030FF3BA3D3E9002305F06F
S21444AC90E3F80022434B04460D4605F063FB08B137
S21444ACA00024404D36A3D3E90023DDE9280105F00E
S21444ACB0D3F800223C4B8846064605F03FFB8146C7
S21444ACC0002840F0A1840022384B3046414605F027
S21444ACD053FB002840F09E84B14608F10048504695
S21444ACE0594629A3D3E9002305F0B6F860E000BF2F
S21444ACF0E3F36EFB79D0E33E277845D92444D93F25
S21444AD00FB50D7647BD71C403043BB3975F10440B5
S21444AD106D0D4BFEC9AF1840FCA9F1D24D62603FA1
S21444AD20EBF33CDE4AA2813FE9C8B5C771D3893FFD
S21444AD300000000000409FC09A99999999996A40EA
S21444AD40CDCCCCCCCCCC35405ED817C2038C9E3F01
S21444AD506F216A9B4B52A13F2ED7D19C0A49373F5D
S21444AD607119ABB745FF1F40ECBC164D8E930F4090
S21444AD701988C921F33610409A9999999999C93FE7
S21444AD80CDCCCCCCCCCCEC3F3B08AA2A23DCA63F8B
S21444AD9000409F4000004940F80D422000408F404C
S21444ADA0000014400000F03F00003EC000003E405B
S21444ADB0DDE9362304F09AFE06460F4622462B4625
S21444ADC04846414605F048F832463B4604F08EFE77
S21444ADD002460B46CDE90C230022B74B05F0CCFACD
S21444ADE0002840F01B840022B44BDDE90C0105F03A
S21444ADF0A5FA18B10023B14CCDE90C3400224FF02B
S21444AE008043DDE9180105F08FFA0446002800F077
S21444AE100984AB4C0022AB4BD4E9200105F084FAFC
S21444AE20002800F02A840022A64BD4E9220105F02B
S21444AE307BFA002800F0218402980026049994A303
S21444AE40D3E9002305F032F900229F4B05F094FA2B
S21444AE50002800F01384994F994C0022994BD4E96A
S21444AE601E0105F061FA002840F00F8432463B4646
S21444AE70C4E9DC67C4E9C223DDE91A01DDE9142329
S21444AE8004F032FEDDE90E23CDE93E01C4E9CA23CF
S21444AE90DDE90023DDE92A01C4E9D423DDE93023D2
S21444AEA0C4E9C023DDE92E23C4E9C823D4E98E23AC
S21444AEB004F01CFE78A3D3E9002304F0CDFF064635
S21444AEC00F4677A3D3E90023D4E9900104F0C4FFE6
S21444AED002460B463046394604F008FE72A3D3E9D0
S21444AEE0002305F0E3F8D4E99223CDE91801D4E928
S21444AEF0060104F0FBFD68A3D3E9002304F0ACFF8D
S21444AF0006460F4666A3D3E90023D4E9940104F029
S21444AF10A3FF02460B463046394604F0E7FD62A3DB
S21444AF20D3E9002305F0C2F8D4E99623CDE9040119
S21444AF30D4E9080104F0DAFD57A3D3E9002304F06A
S21444AF408BFF06460F4656A3D3E90023D4E998015F
S21444AF5004F082FF02460B463046394604F0C6FDEE
S21444AF6051A3D3E9002305F0A1F8CDE90E01DDE9AC
S21444AF7004231046194604F06FFF04460D46DDE9E7
S21444AF800E231046194604F067FF02460B46204639
S21444AF90294604F0ABFD09F09DFF00220023044639
S21444AFA00D4605F0C1F948B922462B46DDE918019D
S21444AFB005F07CF809F030FD04460D46404E204628
S21444AFC02946424FD6E95423CDE9142338A3D3E97E
S21444AFD0002304F041FF02460B46DDE9140104F069
S21444AFE083FDD6E90A34CDE91A01CDE91634DDE904
S21444AFF01601D6E99C2304F079FD27A3D3E9002360
S21444B00004F02AFF04460D4625A3D3E90023D6E9D7
S21444B0109E0104F021FF02460B462046294604F0D2
S21444B02065FD21A3D3E9002305F040F8D6E914458D
S21444B030CDE92A0122462B46DDE9080104F054FDF9
S21444B0400022234BCDE930012046294604F004FF74
S21444B05002460B4600201F4904F046FD00221B4BC7
S21444B0600C46054605F06AF9002808BF28460AA398
S21444B070D3E9002316BF00202146394604F0ECFEEF
S21444B08096F8EC3282468B4626E000BFAFF300804B
S21444B090CDCCCCCCCCCC0C40FCA9F1D24D62603F9C
S21444B0A0FEF2469F2892AF3F1F94D22C39CFB03F32
S21444B0B0F8C1631ADCA54C4000005440000054C05C
S21444B0C0F80D42200000F03F0000E03F0080614061
S21444B0D000001A4000007940D6E916010BB1C6E9D3
S21444B0E0A001D6E9A08942464B4604F0FDFC002266
S21444B0F006460F46A04B2846214605F01FF9002871
S21444B10040F0C78204F1004432463B465046594616
S21444B11005F014F9002840F0BF822846214694A33F
S21444B120D3E9002304F098FE02460B46CDE902011B
S21444B1303046394605F002F908B1DDE90267324681
S21444B1403B464046494604F0D1FC8C4B0A46CDE982
S21444B15002010146C3E9BE12C3E9D81293F8ED22B0
S21444B160D3E918010AB1C3E9A201D3E9A289424648
S21444B1704B4604F0B9FC06460F4602460B4650467C
S21444B180594605F0DBF878B92846214678A3D3E932
S21444B190002304F061FE32463B4682468B4605F069
S21444B1A0EBF808B9B246BB4652465B46404649466B
S21444B1B004F09CFC714C02460B46C4E9D0230022A2
S21444B1C00023CDE90801C4E9D623D4E91C010022B2
S21444B1D06B4B05F0A9F868B90022694BD4E91E0107
S21444B1E005F0A2F830B90022654BD4E9280105F0F1
S21444B1F09BF818B10022624BC4E9D6235F4C002268
S21444B2005F4BD4E92A0105F08FF8A0B900225C4BC5
S21444B210D4E92C0105F088F868B90022584BD4E9E3
S21444B2202E0105F081F830B90022554BD4E930019F
S21444B23005F07AF8A8B1514E00220023D6E91A4503
S21444B2402046294605F070F838B900224FF080436E
S21444B2502046294605F068F818B10023484CC6E94C
S21444B260D634464C0022464BD4E9200105F05CF81F
S21444B27040B90022424BD4E9220105F055F8002893
S21444B28000F00D823D4B00213D4AC3E9D612DFF85B
S21444B290ECA00022DAE99A67DDE91034DAE9048999
S21444B2A0CAE952343046374B3946CAE9508904F025
S21444B2B0D3FD04460D460022334BDDE91A0104F063
S21444B2C0CBFD02460B462046294604F00FFC0246B8
S21444B2D00B46DDE92A0104F007FC25A3D3E9002345
S21444B2E004F0BAFDDDE9142304F000FCDDE92E3455
S21444B2F0CAE95401CAE95634DDE93A34DDE92C0199
S21444B300CAE95834DDE90034CAE95A34DAE9AE23E6
S21444B31004F0EAFB16A3D3E9002304F09DFDDAE922
S21444B3205C2304F0E3FB0022DDE93234CAE95C0125
S21444B330CAE95E34DAE96001144B04F08DFDDDE9B8
S21444B340302304F0D3FBDDE90A34CAE96001CAE9D4
S21444B3506234DDE90634CAE96434CAE96634DDE9B0
S21444B3601C34CAE96834CAE96A34DDE91E340FE09D
S21444B370FCA9F1D24D62603F00806140F80D422046
S21444B3800000F03F00001440000059400000EE3F2B
S21444B390CAE96C34CAE96E34DDE93434CAE9703437
S21444B3A0DDE92034CAE97234DAE93A23CAE93823B3
S21444B3B0DDE92034CAE93A34DDE92234CAE9743492
S21444B3C0DAE93E23CAE93C23DDE92234CAE93E34BD
S21444B3D0CAE97634DDE93634CAE97834DDE90C3432
S21444B3E0CAE9AC34DDE90634CAE97A34DDE9243402
S21444B3F0CAE97C34CAE97E34DDE92634CAE98034B5
S21444B400CAE98234DDE93834DDE91A01CAE984340C
S21444B410DDE93C34CAE98E89CAE98634DDE912346A
S21444B420CAE98834CAE98A34DAE94223CAE94023B5
S21444B430DDE91234CAE94234DDE92834CAE98C34F9
S21444B440DAE94623CAE94423DDE92834CAE946341E
S21444B450DDE93E34CAE9AE34DDE91834CAE990344D
S21444B460DAE90623CAE99223DDE90434CAE99434C6
S21444B470DAE90823CAE99623DDE90E34CAE99834A2
S21444B48091A3D3E9002304F0E7FC3B46324604F09C
S21444B4902DFBDDE91634CAE99A01CAE99C34DDE994
S21444B4A02A34CAE99E34DDE90234CAE9A0340023CA
S21444B4B0AAF8EA32AAF8EC32DDE90834CAE9A2343A
S21444B4C059B0BDE8F08F00230024FEF7FEBD0025EA
S21444B4D0FEF73ABF7EA3D3E90023FEF792BF7EA3CE
S21444B4E0D3E90023FEF78DBF4FF04043404649461C
S21444B4F004F024FF00283EF4A8AF00224FF0804317
S21444B5003046394604F0F0FAFEF79DBF002000218D
S21444B510FEF7A9BF00247A4DFEF7E3BF794B3046C9
S21444B520394604F00BFF00283EF4FCAF0022764B6D
S21444B5302046294604F0D8FAFEF7F2BF4FF000083A
S21444B540DFF8BC91FFF705B842464B46DDE90E01ED
S21444B55004F0CCFAFFF70DB861A7D7E90067FFF708
S21444B5601BB89AF8EE32002B7FF4F4A80023674CFD
S21444B570CAE9E034FFF7F4B80022654B002183F8AB
S21444B580EE22624AC3E9E012FFF7EAB80022604BB3
S21444B59083F8EE22DDE90612F4E70026FFF717B932
S21444B5A051A3D3E900233046394604F0C7FE0028A9
S21444B5B03FF44FA9204629464DA3D3E9002304F07F
S21444B5C093FAFFF744B90024524DFFF793BA00228A
S21444B5D0514B2046294604F0C5FE58B900224F4B2D
S21444B5E02046294604F082FAFFF78ABA42A5D5E9EE
S21444B5F00045F3E74FF0000A4FF0000BFFF782BA1E
S21444B60000240025FFF74EBB4FF00009DFF81881F1
S21444B610FFF765BBDFF81481FFF761BB0023404C9E
S21444B620FFF7EABB00220023DDE9000104F07CFEBC
S21444B630054630BB00224FF08043DDE9000104F0AC
S21444B64073FE00BB314B0022DDE9000104F06CFEC2
S21444B6500028169B18BF4FF0FF33184604F092FBA1
S21444B660DDE90C2304F0F8FB0022002306460F46CF
S21444B67004F064FE00283FF4EFAB00260027FFF7F3
S21444B680EBBB2046EAE72846E8E700220023FFF71C
S21444B690EFBB0025234C37E556465F464FE5002270
S21444B6A01A4BD4E9240104F03FFE00283FF4EFADE2
S21444B6B00022164BD4E9260104F036FE00287FF417
S21444B6C0E1ADE4E5AFF30080FCA9F1D24D62603F02
S21444B6D000000000008AAB40000000000088A3C0C1
S21444B6E0000000000088A3409A9999999999E9BF67
S21444B6F09A9999999999E93F0000000000409FC0A3
S21444B70000408F40000008C0000008400000F03FA2
S21444B710F80D422000409F40000049C000004940C8
S21444B72000005440008061C000003E4000003EC01F
S21444B730094B40F2011206A1D1E90001A3F8EA221E
S21444B740A3F8EC22C3E9B001704700BFAFF3008012
S21444B7500000000000709740F80D4220F8B56B4B8F
S21444B76000266B4C0027186804F01EFB694B1D68C6
S21444B770C4E90001284604F0F5FA674BC4E91A0107
S21444B780186804F011FB654BC4E91401186804F00A
S21444B7900BFB634BC4E90401186804F005FB614BDA
S21444B7A0C4E90601186804F0FFFA5F4BC4E90801CF
S21444B7B0186804F0F9FA5D4BC4E90A01186804F005
S21444B7C0F3FA5B4BC4E93201186804F0EDFA594BBE
S21444B7D0C4E93601186804F0E7FA574BC4E9020195
S21444B7E0186804F0E1FA554BC4E91001C4E934671B
S21444B7F0187804F0B7FA524BC4E92A01187804F0D2
S21444B800B1FA504BC4E92C01187804F0ABFA4E4B0D
S21444B810C4E92E01187804F0A5FA4C4BC4E930016B
S21444B820187804F09FFA4A4BC4E91C01187804F0CF
S21444B83099FA484BC4E91E01187804F093FA464B2B
S21444B840C4E92001187804F08DFA444BC4E9220177
S21444B850187804F087FA424BC4E92401187804F0B7
S21444B86081FA404BC4E92601187804F07BFAC4E90F
S21444B870280125BB3C4B186804F096FA3B4BC4E9B8
S21444B8800201186804F06EFA0022394BC4E9122308
S21444B890384BC4E90C01C4E93267186804F062FA0C
S21444B8A0354BC4E90E01186804F07EFA334BC4E9FC
S21444B8B01601186804F078FAC4E91801F8BD012D99
S21444B8C01CD12F4B186804F04DFA2E4BC4E90C01DA
S21444B8D0C4E93267186804F045FA2B4BC4E91201F0
S21444B8E0186804F03FFA294BC4E90E01186804F0BE
S21444B8F05BFAC4E91601C4E91867DFE7023D012D87
S21444B900DCD8C4E90C67C4E91667F4E7701E402027
S21444B910F80D4220581C4020781C4020201F402010
S21444B920401F4020041F4020101F4020901F4020EE
S21444B930501C4020A41F40206C1E402082174020EC
S21444B94081174020801740207F174020561F4020F4
S21444B950551F4020281C4020271C4020261C4020E1
S21444B960251C4020541F4020B81D4020C01D4020A8
S21444B97000004440901D4020AC1D4020A81D40209F
S21444B9808C1F4020581F4020741F4020981F402082
S21444B9902DE9F04F7D4C85B07D4EDFF85CA2DFF894
S21444B9A05CB2D4E9000104F04FFD7A4B804618603F
S21444B9B0D4E9060104F048FD3060D4E9040104F0FB
S21444B9C043FD754B1860D4E9020104F03DFD734A0B
S21444B9D0734B074610601860D4E9140104F034FD34
S21444B9E0CBF80000CAF800008146D4E9180104F0F8
S21444B9F00BFD6C4905460860D4E9220104F004FDB9
S21444BA0069490880D4E9240104F0FEFC67490870BB
S21444BA10D4E91A0104F0F8FC65490870D4E9200119
S21444BA2004F012FD63490860D4E91E0104F00CFDDD
S21444BA3061490860D4E91C0104F006FD5F490860CA
S21444BA4038465F490968039105F018F8534A544B41
S21444BA50029616461C460399CDF804A060B11160C0
S21444BA601960584F4846394605F008F8B8B1019B66
S21444BA70CBF800701F6019E001F1004A3846514681
S21444BA8004F0DEFF20B1C6F800A0C4F800A0E8E742
S21444BA905146384604F0D4FF0028E2D0F5E74A4F32
S21444BAA04846394604F0CCFF0028E0D1474B484F7F
S21444BAB01B6853B9474B25F002051968012D08D178
S21444BAC0404604F017FD386004E0012B4ED1424B4B
S21444BAD0F1E73960414D3868294604F0C5FF00B1A6
S21444BAE03D603B680022DFF818813D4F3D4DC8F865
S21444BAF000303B603C4BD5E9200104F015FC10B106
S21444BB000023C8F800300022374BD5E9220104F060
S21444BB100BFC08B100233B60344B0022344FD3F86F
S21444BB200080314BC7F80080D5E9240104F0FCFBC3
S21444BB3020B1002333602F4B1B683B6000222A4B06
S21444BB40D5E9260104F0F0FB18B10023C7F80080BD
S21444BB5023600022244BD5E9280104F0E5FB10B10C
S21444BB6000233360236005B0BDE8F08F022B03D179
S21444BB70194B41461868A4E7032BABD10023029A1D
S21444BB801360154B1B683B60A4E700BFE8104220D7
S21444BB905C1B4020941F4020B4174020B819402016
S21444BBA0141940205C1C40207C1740207A17402003
S21444BBB0A8174020A4174020A01740209C174020D8
S21444BBC0AC17402000004843000048C3581C40209F
S21444BBD09C1F4020B81D4020A41F402000401C4508
S21444BBE008194020F80D42200000F03F281D402050
S21444BBF0801C4020C41C40208C184020A4184020A0
S21444BC00AC194020F8B5174B174C1E68174D66B153
S21444BC10012E19D000210020F5F760FE00210120F6
S21444BC20F5F75CFE00232B700CE02678002EF1D14D
S21444BC3000213046F5F752FE0D490120F5F74EFE39
S21444BC4001232E702370F8BD2F78002FE2D10849C7
S21444BC503846F5F743FE00213046F5F73FFE2E7092
S21444BC602770F0E7581C4020E8174020E91740208A
S21444BC700000C8420A4B1B685A1E53425341094AA5
S21444BC801360094B1B68012B03D0084B1B68012B20
S21444BC9005D1074B00221A600122064B1A607047F2
S21444BCA05C1C4020801B40208C1B4020881B40206E
S21444BCB0741B4020781B4020104B1A68104B1A60A7
S21444BCC0104B1A68104B1A60104B1A68104B1A60C7
S21444BCD0104B1A68104B1A60104B1A68104B1A60B7
S21444BCE0104B1A68104B1A60104B1A68104B1A60A7
S21444BCF0104B1A68104B1A60FFF7BCBF5C1A402002
S21444BD00741B4020741A40208C1B4020701A40201C
S21444BD10881B4020601A4020781B4020781A402018
S21444BD20901B40206C1A4020841B4020641A4020FC
S21444BD307C1B4020581A4020701B4020104B1A6829
S21444BD40104B1A60104B1A68104B1A60104B1A6846
S21444BD50104B1A60104B1A68104B1A60104B1A6836
S21444BD60104B1A60104B1A68104B1A60104B1A6826
S21444BD70104B1A60104B1A68104B1A60FFF77ABFC4
S21444BD80601D4020741B4020781D40208C1B4020A2
S21444BD90741D4020881B4020641D4020781B402092
S21444BDA07C1D4020901B4020701D4020841B40205A
S21444BDB0681D40207C1B40205C1D4020701B40209A
S21444BDC000230B4A012113600A4A13600A4A13608F
S21444BDD00A4A13600A4A13600A4A13600A4A1360FE
S21444BDE00A4A13600A4A11600A4A1360704700BF41
S21444BDF0941B4020901B40208C1B4020881B4020D6
S21444BE00841B4020801B40207C1B4020781B402005
S21444BE10741B4020701B402002230B4A13600B4ABD
S21444BE20136000230A4A13600A4A13600A4A1360DE
S21444BE300A4A13600A4A13600A4A13600A4A13609D
S21444BE400A4A1360704700BF941B4020901B402052
S21444BE508C1B4020881B4020841B4020801B402095
S21444BE607C1B4020781B4020741B4020701B4020C5
S21444BE702A4B2B491A6810B542B90A68012A05D1DB
S21444BE80284802602848026028480260284A502011
S21444BE901060284A28481060284A12681A60284BBE
S21444BEA01B780B60274B1C688CB9274B00211868FD
S21444BEB004F0BCFDB0B1254B07221A600122244B86
S21444BEC01C60244B1A600222234B1A600AE0012CA1
S21444BED009D102231D4A13601D4A13601D4A13608C
S21444BEE01D4B1C6010BD022C0AD1184B03221A604D
S21444BEF00022174B1A600122164B1C60164BE4E7CF
S21444BF00032CEFD1114B042202211A600123104A5C
S21444BF101360104A1160104A1360E3E73C1B40204C
S21444BF20381B4020481B40204C1B4020541B4020BC
S21444BF30341B4020301B4020000048C2FC194020DF
S21444BF401E1E40205C1C4020781C4020441B402081
S21444BF50401B4020641B40209819402000000000ED
S21444BF6038B5174B00211C68204604F069FD08B11B
S21444BF7004F10044134D20462C6003F015FF0CA337
S21444BF80D3E9002304F092F80BA3D3E9002303F08B
S21444BF9063FF00220C4B03F05FFF0C4B002204F0BF
S21444BFA085F804F051FA0A4B6860186038BD00BF43
S21444BFB05C8FC2F528DC2740B4A766033D39FB3FB7
S21444BFC0701E4020F020402000004E4000408F402D
S21444BFD0781C402008B5074B186804F03BFB064B1A
S21444BFE00649186004F036FD10B1054B01221A705C
S21444BFF008BD00BF181E4020501840200000F041E5
S21444C00054184020FE28D4BF01300020704770B535
S21444C0100022FF23064ED4B2551C8C4202D3D8438A
S21444C020C0B270BD025D53402A46F35CF3E700BFDE
S21444C030D08846000721013008B5FFF7E8FFC0B2B4
S21444C04008BDB0F5447F38B5144617D1244D204674
S21444C05095F8EC32FF2B14BF01330023DBB285F88E
S21444C060EC3253701F4A1370FFF7E4FF1E4BC0B206
S21444C07085F8ED0220701870012038BD402818D08D
S21444C080B0F5547FF8D1164D204695F8E832FF2B8C
S21444C09014BF01330023DAB285F8E8226270134AEB
S21444C0A01360FFF7C7FFC0B2114B85F8E902207052
S21444C0B014E00B4D204695F8E032FF2B14BF0133B5
S21444C0C00023DAB285F8E02262700A4A1360FFF76A
S21444C0D0B1FF094BC0B285F8E10220701860CBE787
S21444C0E0E88340203B1940203A1940203419402028
S21444C0F030194020C0194020BC194020402838B58B
S21444C100144616D1254D204695F81833FF2B14BFF8
S21444C11001330023DAB285F818236270204A13608C
S21444C120FFF788FF1F4BC0B285F8190320701860CC
S21444C13005E0B0F5547F04D0B0F5447F17D0012015
S21444C14038BD164D204695F82033FF2B14BF0133D7
S21444C1500023DAB285F820236270134A1360FFF78F
S21444C16069FFC0B2114B85F821032070DFE70B4D01
S21444C170204695F82433FF2B14BF01330023DBB24B
S21444C18085F8243353700A4A1370FFF753FF094B5C
S21444C190C0B285F8250320701870D0E7E8834020A5
S21444C1A01C19402018194020C4184020C0184020AC
S21444C1B0CB184020CA184020402838B5144617D11A
S21444C1C0254D204695F81833FF2B14BF0133002322
S21444C1D0DAB285F854236270204A1360FFF72AFFC8
S21444C1E01F4BC0B285F8550320701860012038BD37
S21444C1F0B0F5547F18D0B0F5447FF7D1164D20469D
S21444C20095F86033FF2B14BF01330023DBB285F867
S21444C21060335370134A1370FFF70CFFC0B2124BCF
S21444C22085F86103207014E00B4D204695F85C3386
S21444C230FF2B14BF01330023DBB285F85C33537005
S21444C2400A4A1370FFF7F6FE094BC0B285F85D0341
S21444C25020701870CAE700BFE8834020AC1840201E
S21444C260A8184020A01840209F1840209C18402022
S21444C2709B184020402838B5144616D1254D2046F4
S21444C28095F86433FF2B14BF01330023DAB285F8E4
S21444C29064236270204A1360FFF7CCFE1F4BC0B283
S21444C2A085F865032070186005E0B0F5547F04D027
S21444C2B0B0F5447F17D0012038BD164D204695F87A
S21444C2C07033FF2B14BF01330023DAB285F8702392
S21444C2D06270134A1360FFF7ADFEC0B2114B85F887
S21444C2E071032070DFE70B4D204695F86C33FF2B27
S21444C2F014BF01330023DBB285F86C3353700A4A0B
S21444C3001370FFF797FE094BC0B285F86D03207093
S21444C3101870D0E7E88340209418402090184020B6
S21444C320801840207C1840208718402086184020DB
S21444C330502870B50546144616D18C4A92F8A83152
S21444C340FF2B14BF01330023D9B282F8A811884AC0
S21444C3502171136040F285339D4200F0DD80162D36
S21444C36000F0F080012070BD642826D065283BD0BC
S21444C37032284FD0702863D0712877D0332800F005
S21444C3808C806A2800F09F80B0F5617FE2D1774DBB
S21444C390204695F8F032FF2B14BF01330023DBB25E
S21444C3A085F8F0325370734A1370FFF743FEC0B2F9
S21444C3B0714B85F8F10220706DE06C4E204696F87D
S21444C3C0AC32FF2B14BF01330023DBB286F8AC3209
S21444C3D053706A4A1370FFF72DFE694BC0B286F855
S21444C3E0B00220701870B5E7604E204696F81033B9
S21444C3F0FF2B14BF01330023DBB286F8103353708F
S21444C400604A1370FFF716FEC0B25F4B86F81403FB
S21444C4102070E7E7554E204696F8C432FF2B14BFEB
S21444C42001330023DBB286F8C4325370574A137084
S21444C430FFF700FEC0B2564B86F8C5022070D1E71F
S21444C4404A4E204696F8B832FF2B14BF01330023D9
S21444C450DBB286F8B83253704E4A1370FFF7EAFDE3
S21444C460C0B24D4B86F8B9022070BBE73F4D20461C
S21444C47095F80433FF2B14BF01330023DBB285F851
S21444C48004335370454A1370FFF7D4FD444BC0B28F
S21444C49085F805032070187064E7344D204695F8F7
S21444C4A02833FF2B14BF01330023DBB285F828332F
S21444C4B053703C4A1370FFF7BDFDC0B23A4B85F843
S21444C4C029032070E7E7294D2046D5F8D832D5F819
S21444C4D0D822C3F3C733FF2B14BF01330023DBB288
S21444C4E063F3D632C5F8D8226370D5F8D8322F4ACB
S21444C4F0C3F3C7331360FFF79DFDB5F8DA32C0B215
S21444C5002B4A60F3CE13A5F8DA322070B5F8DA3247
S21444C510C3F3C713136025E7144D2046254A95F800
S21444C5204033FF2B14BF01330023DBB285F840337E
S21444C53063701370FFF77EFDC0B21F4B85F841034E
S21444C5402070A8E70949B1F89022C2F34313013397
S21444C55003F00F0363F34812A1F890226370B1F816
S21444C5609032164AC3F34313D4E700BFE88340200F
S21444C5702C1C40202C1940202B1940207C1940208C
S21444C5807D1940201019402011194020C61940201A
S21444C590C51940205D1940205C194020ED18402004
S21444C5A0EC184020221940202119402070194020C0
S21444C5B06C194020B9184020B8184020C41A4020AE
S21444C5C00F28D4BF01300020704770B50022FF23E7
S21444C5D0074ED4B2551C8C4205D3DB4383EA13136F
S21444C5E003F00F0070BD025D53402A46F35CF0E74B
S21444C5F0D08946000721013008B5FFF7E6FFC0B2F0
S21444C60008BDB0F5AE6F70B5054614461AD1C04D98
S21444C610204695F805221309013363F3071203F005
S21444C6200F0385F80522BB4A1360FFF7E3FF95F82E
S21444C630063260F3030300F00F0085F80632B64B6B
S21444C6401860C0E0B0F5B06F1DD0B0F5B26F35D10C
S21444C650AF4D204695F8162202F00F03013363F3DC
S21444C660030203F00F0385F81622AC4A1360FFF763
S21444C670C1FF95F8163260F3071300F00F0085F8F3
S21444C6801632A74BDCE7A24D2046B5F80C22C2F37F
S21444C6908313013363F3891203F00F03A5F80C22C6
S21444C6A0A04A1360FFF7A6FF95F80D3260F38503A2
S21444C6B000F00F0085F80D329B4BC1E740F29553CE
S21444C6C0984222D040F28553984258D050287CD085
S21444C6D0512835D18E4D204695F8302202F00F036E
S21444C6E0013363F3030203F00F0385F830228F4AC5
S21444C6F01360FFF77FFF95F8303260F3071300F0BE
S21444C7000F0085F830328A4B9AE7814E204696F8D9
S21444C7101B22C2F38303013303F00F0363F3850242
S21444C72086F81B22834A1370FFF764FF96F81C3280
S21444C73000F00F0060F3030386F81C327E4B18703B
S21444C740602D5DD0612D35D1714D204695F840223F
S21444C75002F00F03013363F3030203F00F0385F87B
S21444C7604022764A1360FFF745FF95F8403260F35F
S21444C770071300F00F0085F84032714B60E7644EB3
S21444C7802046D6F82022C2F38333013363F3913232
S21444C79003F00F03C6F820226A4A1360FFF72AFF05
S21444C7A096F8223260F3850300F00F0086F82232B2
S21444C7B0654B1860132D3ED0142D57D0152D70D0D0
S21444C7C0162D00F08980012070BD514D204695F805
S21444C7D0282202F00F03013363F3030203F00F032E
S21444C7E085F82822594A1360FFF704FF95F8283243
S21444C7F060F3071300F00F0085F82832544B1FE708
S21444C800434D204695F8382202F00F03013363F374
S21444C810030203F00F0385F838224E4A1360FFF7ED
S21444C820E9FE95F8383260F3071300F00F0085F8F8
S21444C8303832494B04E7364D2046B5F84A22C2F30F
S21444C8408313013363F3891203F00F03A5F84A22D6
S21444C850424A1360FFF7CEFE95F84B3260F38503E9
S21444C86000F00F0085F84B323D4BE9E6284D204654
S21444C870B5F85222C2F3C313013363F3CA1203F06A
S21444C8800F03A5F85222374A1360FFF7B3FE95F814
S21444C890533260F3C60300F00F0085F85332324B30
S21444C8A0CEE61B4D204695F85A2202F00F0301337C
S21444C8B063F3030203F00F0385F85A222B4A1360EE
S21444C8C0FFF798FE95F85A3260F3071300F00F000E
S21444C8D085F85A32264BB3E60D4D2046B5F89022DD
S21444C8E0C2F34313013363F3481203F00F03A5F86E
S21444C8F09022204A1360FFF77DFE95F8913260F34C
S21444C900440300F00F0085F891321B4B98E600BFB5
S21444C910E8834020101A40200C1A4020341E402041
S21444C920301E4020EC1D4020E81D4020A41A402024
S21444C930A01A4020DB194020DA194020841A4020EF
S21444C940801A4020E4194020E0194020B41A4020C0
S21444C950B01A4020941A4020901A4020041B4020CD
S21444C960001B4020E41A4020E01A4020CC1A402005
S21444C970C81A4020C41A4020C01A40200D4B0E4905
S21444C9800E4810B51C680E4B1A78A2421A460BD1B4
S21444C9900B8801339BB2312B0B8008D932230B8092
S21444C9A001230370147010BD00230B80F9E70023A5
S21444C9B0F7E700BF581D40209A17402082174020B2
S21444C9C08A1740200D4B0E490E4810B51C680E4B76
S21444C9D01A78A2421A460BD10B8801339BB2312BEC
S21444C9E00B8008D932230B8001230370147010BDCA
S21444C9F000230B80F9E70023F7E700BFB41D40206F
S21444CA009817402081174020891740200D4B0E4927
S21444CA100E4810B51C680E4B1A78A2421A460BD123
S21444CA200B8801339BB2312B0B8008D932230B8001
S21444CA3001230370147010BD00230B80F9E7002314
S21444CA40F7E700BFA41D40209617402080174020DB
S21444CA50881740200D4B0E490E4810B51C680E4BE7
S21444CA601A78A2421A460BD10B8801339BB2312B5B
S21444CA700B8008D932230B8001230370147010BD39
S21444CA8000230B80F9E70023F7E700BF881D40200A
S21444CA90941740207F1740208717402008B5FFF79B
S21444CAA06DFFFFF78FFFFFF7B1FFBDE80840FFF7C4
S21444CAB0D1BF0D4B0D490E4810B51C780D4B1A7856
S21444CAC0A2421A460BD10B8801339BB2312B0B8002
S21444CAD008D932230B8001230370147010BD002341
S21444CAE00B80F9E70023F7E7101D402092174020FB
S21444CAF0281C4020861740200D4B0E490E4810B582
S21444CB001C780E4B1A78A2421A460BD10B88013376
S21444CB109BB2312B0B8008D932230B800123037040
S21444CB20147010BD00230B80F9E70023F7E700BF1D
S21444CB309C1C402090174020271C402085174020EE
S21444CB400D4B0E490E4810B51C680E4B1A78A2427F
S21444CB501A460BD10B8801339BB2312B0B8008D974
S21444CB6032230B8001230370147010BD00230B8006
S21444CB70F9E70023F7E700BF541D40208E174020F6
S21444CB80261C4020841740200D4B0E490E4810B5F5
S21444CB901C680E4B1A78A2421A460BD10B880133F6
S21444CBA09BB2312B0B8008D932230B8001230370B0
S21444CBB0147010BD00230B80F9E70023F7E700BF8D
S21444CBC0D01C40208C174020251C40208317402032
S21444CBD0554B70B51B78012B40F09780534B1B7810
S21444CBE0003B18BF0123524A1370524B1B78012B4B
S21444CBF040F08D804D4B1B781A1E18BF01224E4BB9
S21444CC001A704E4B1B78012B40F08380474B1978A3
S21444CC10003918BF01214A4B19704A4B1B78012B27
S21444CC200FD0494B1B78012B0BD0484B1B78012B5C
S21444CC3007D0474B1B7803F1FF3CDCF1000343EB82
S21444CC400C03444803704448006828B1022805D1C0
S21444CC5042480078032801D1012B13D0404B1B785F
S21444CC60012B0FD03F4B1B78012B0BD03E4B1B7830
S21444CC70012B07D03D4B1B78012B03D0012914BF51
S21444CC801346012303F0010239490A70394A1478DD
S21444CC90394A601E414241411170384A1068384A48
S21444CCA000F1FF3CDCF1000141EB0C011170354A08
S21444CCB01268511E4D424D4133490D70334909881F
S21444CCC04D1E6E426E41324D2E7083B9012C22D0D9
S21444CCD0012822D0012922D0012A22D02D4B1B68BC
S21444CCE0012B04D0114B1B785A1E5342534103F078
S21444CCF00103294A1370294B294A1B68013B022B1E
S21444CD008CBF00230123137070BD00236BE7002201
S21444CD1075E700217FE72346E9E70346E7E70B4646
S21444CD20E5E71346E3E700BF561F4020A817402018
S21444CD302A1C4020551F4020291C4020541F4020B8
S21444CD40241C402082174020811740208017402012
S21444CD507F1740207E174020581C4020E81A402069
S21444CD60281C4020271C4020261C4020251C4020F0
S21444CD704546402078174020464640206C1F4020B9
S21444CD80444640208C1D4020434640200418402002
S21444CD90424640207C1F402041464020241E4020DE
S21444CDA0404640200B4B1B68012B09D10A4A1168A8
S21444CDB00A4A106888420ABF094A116013607047DD
S21444CDC0022B06D1074B1B68012B02BF044B0022E3
S21444CDD01A607047581C4020601F4020841F402023
S21444CDE07C1F40206C1F4020044A1368013313F50F
S21444CDF0807F28BF00231360704700BFF820402080
S21444CE00034B18B11A790AB91A689A6018717047B0
S21444CE10F8204020054A107930B113689068834260
S21444CE2038BFA3F58073181A704700BFF820402017
S21444CE30034B18B11A7B0AB91A681A6118737047FB
S21444CE40F8204020054A107B30B1136810698342AD
S21444CE5038BFA3F58073181A704700BFF8204020E7
S21444CE601F4B10B51C681F4B012C03D11A780AB906
S21444CE7002225A701C4A1178012903D19A780AB9B9
S21444CE8003225A70194800220129027021D1012C2C
S21444CE901BD1174A174C1268022A0CD12278032A4F
S21444CEA009D10222DA705A7001221A704A1E51427F
S21444CEB05141997010BD5A78032A18BF0222DA707D
S21444CEC00122027006202070EFE70320D8705870C5
S21444CED0EBE7012CE5D05878033818BF0120F5E776
S21444CEE0781F40200C214020641F402078174020A3
S21444CEF0581C4020E81A40209C4B2DE9F0471D78EA
S21444CF009B4CDFF8B89225716571FFF7A9FF994BE2
S21444CF101B784BB3984A022317786371A37177B191
S21444CF20964A13700027E3786279012B40F05D81BE
S21444CF30D31E18BF0123384689F800307CE0904B56
S21444CF401B781BB18D4B03221A70ECE78D4A177879
S21444CF501FB18A4A04211170E4E78B4B1B78002BDF
S21444CF60E0D0864B0122EFE7884ADFF81082177834
S21444CF705FB10322002188F800306271844A13703E
S21444CF80844A1160844A1370CCE7E379E678EBB1BF
S21444CF90E5B9824B8249186803F05CFD18B1814BB1
S21444CFA01B68052B12D9804B1B68012B0ED002231D
S21444CFB0002089F800606371A371062388F8003066
S21444CFC0FFF71EFF0023E371BDE8F087237AFBB129
S21444CFD0012D1DD1714B7249186803F03BFD18B101
S21444CFE0724B1B68052B13D9714B93F800A0BAF10A
S21444CFF0000F0DD10223504689F800606371A37177
S21444D000062388F80030FFF7FBFE84F808A0DBE729
S21444D010022E15D100232372022D40F00A8198F87F
S21444D0200030052B40F0FB80022E00F002810020E9
S21444D0306571A57189F80060BDE8F047FFF7E0BE6A
S21444D0400023032EE371E7D0E4E7002D40F0D880B8
S21444D050554B4FF07E511D68504B012D18680BD030
S21444D06003F0EEFC70B902236371A371052388F8BC
S21444D070003058E7657156E703F0E2FC10B9012327
S21444D080A37150E70323012DA37140F0E18049E7E3
S21444D090C5B9424B4249186803F0DCFC18B1414B11
S21444D0A01B68052B02D90123E371E9E70323A37127
S21444D0B03D4B1B68012B3FF435AF0123A571E57149
S21444D0C0637130E7032D09D1344B4FF07E51186815
S21444D0D003F0B6FC0028D2D00123BAE0012DCED10D
S21444D0E0FAE74DB9304B1B68012B00F0B38002239E
S21444D0F0A37163710623BAE7012D2ED12D4B1B680D
S21444D100002B40F0A7802A4D2A78012A0CD1234BC5
S21444D1102349186803F09EFC18B1244B1B68052B62
S21444D12002D901232372ABE72B78012B40F092807F
S21444D13023720323A3711C4B1B68012B04D10023C9
S21444D1406371A3712372EEE6FFF764FE1D284FF069
S21444D150010784BF0223A371E5E6032D7AD1164B5B
S21444D1601B78022B2CD165718AE700BF581C4020DF
S21444D1700C2140204146402044464020E81A4020A6
S21444D18043464020424640204546402040464020B4
S21444D190251840205C1B402024184020781C402042
S21444D1A00000A0408C1F40209C1D4020C01D4020F5
S21444D1B0641F4020781F4020E91A4020EA1A402085
S21444D1C0A379022B46D0244B4FF07E51186803F0C7
S21444D1D037FC00283ED0214BA5711B68012BB3D1E8
S21444D1E084F805A084F806A09DE6022B03D1012A04
S21444D1F008BF00239FE6032B7FF49DAE002AF7E783
S21444D200022D3FF437AF012D22D1134B4FF07E5100
S21444D210186803F015FC00283FF484AE18E0062B8B
S21444D22007D1731E012B3FF602AF012E01D0022E0A
S21444D23010D14FF0000A022E88F800A03FF428AF21
S21444D240032E3FF44EAF012E04D1032D7FF4FDAEE2
S21444D25003236371002313E7781C40209C1D402061
S21444D260184B1A78184B1B781343184B14BF0122DB
S21444D27000221A70164B174A1B68003B18BF01233E
S21444D2801370154B1A78154B1B781343144B14BF65
S21444D290012200221A70134B134A1B78013B18BF15
S21444D2A001231370114B124A1B78003B18BF01230D
S21444D2B01370104B104A1B78003B18BF01231370A1
S21444D2C0704700BFE61D4020E51D402067184020FB
S21444D2D0901E402064184020D51D4020D41D402078
S21444D2E0651840201D1E4020661840201E1E402003
S21444D2F063184020281E40206218402038B52A4B28
S21444D3002A4D1B68012B30D1294B1C68294B012C14
S21444D3101B6814D1002B42D1274B4FF07E5118681E
S21444D32003F098FB00283AD0244B0021186803F0F9
S21444D3307DFB002833D02C60214B1C7038BD1C4329
S21444D3402DD11D4B4FF07E51186803F083FB30B34C
S21444D3501A4B0021186803F069FB00B32C60194B84
S21444D3601C68003C18BF0124E6E7C3B9164B1C688A
S21444D370164B012C1B6810D18BB90F4B4FF07E51C6
S21444D380186803F067FB50B1114B0021186803F08E
S21444D3904DFB20B10B4B1C6001E01C43EDD02B68C9
S21444D3A0002BDCD00124C7E7581C4020641C4020D6
S21444D3B0681F40208C1F4020781C4020901F40202F
S21444D3C079174020141B4020981D4020C01D402043
S21444D3D0BC1D402038B50124204B00251C70204B32
S21444D3E01C70204B1C70204B1C70204B1D70204B17
S21444D3F01D70204B1C70204B1C70204B1D70204B06
S21444D4001D70204B186803F043FB1F4B18601F4BDE
S21444D4101C601F4B1C601F4B1C601F4B1A681F4B25
S21444D4201A6015221E4B1C701E4B1C701E4B1C7023
S21444D4301E4B1C701E4B1D701E4B1D701E4B1A70CF
S21444D44006221E4B1D701E4B1D701E4B1A70182252
S21444D4501D4B1D701D4B1A7038BD00BFC4194020AB
S21444D460201940203919402038194020C918402036
S21444D470C81840209D1840209E18402084184020FC
S21444D480851840205C1B4020A8194020A419402041
S21444D49094194020F81840205C1C40200019402075
S21444D4A0B419402012194020A11840208818402062
S21444D4B02A1940202919402028194020271940209D
S21444D4C0261940202519402024194020231940209D
S21444D4D0064B01221A70064B1B78934204D1054A28
S21444D4E013707822044B1A80704700BF2B1B4020D1
S21444D4F0631840202A1B4020281B402008B5FFF70D
S21444D500E7FFFEF71BFC044B1B68012B1EBF034BB7
S21444D51000221A6008BD00BF8C1D4020081B402016
S21444D52008B5FFF7D5FFFEF7C7FB064B1B68012B74
S21444D5301EBF054B00221A60044B1A68044B1A603F
S21444D54008BD00BF6C1F4020601C4020581F402070
S21444D550741C40200C4B1A780C4B32B90C4A127887
S21444D560012A02BF1A8801321A801A88B2F5FA7F55
S21444D57021BF00221A80064B1A700023054A1370F6
S21444D580054A1380704700BF621840201A1840208E
S21444D5902B1B40202A1B4020281B402008B5FFF7A1
S21444D5A0D9FFFEF70DFC0023024A1360024A1360BB
S21444D5B008BD00BF601C4020081B4020F8B52B4B1C
S21444D5C02B4918682B4D03F04FFA2B4C10B102230D
S21444D5D02B6003E0637ABBB1286060720123274F57
S21444D5E0274E3B603360FFF7B5FFFEF715FC254B2F
S21444D5F01B7833B9244B1B78052B0CD1E378022BCC
S21444D6000FD002236371F8BD204A126832F002013B
S21444D61008BF1346DCE7062B03D1E378013B012B16
S21444D620EFD81B4A194B12781B6882B9E278022A53
S21444D63004D10BB12A680AB90123E3E7E278012A48
S21444D64005D113B12B68002BDBD10323DAE7002B7B
S21444D650D7D1104A3B6013600F4A336013600122EF
S21444D660A371627203226271CDE700BF781C40202A
S21444D670CDCCCC3D5C1C40200C214020601C40207E
S21444D680081B402041464020E81A4020741F402092
S21444D69045464020941B4020901B402010B5134C18
S21444D6A0FFF798FEFFF7FAF9FFF726FCFEF756F861
S21444D6B0FCF7E6F9FEF76CF92268032A05D8DFE89A
S21444D6C002F0020B0E11FFF719FF094B5A7922603C
S21444D6D09A79084B1A7010BDFFF722FFF5E7FFF75B
S21444D6E06DFFF2E7FFF75AFFEFE700BF581C4020F4
S21444D6F00C214020E91A402010B52F4CFFF7B0FD0E
S21444D7002378052B56D8DFE803F0031638474F53E3
S21444D71000F072F8FEF75EFC284B1B78012B3AD1DA
S21444D720274A1178274A12780A4334D1264A136086
S21444D730264A137018E0254B1A78511E4B424B412B
S21444D74023490B7023490B7023490B7023490B70F4
S21444D750234B1B78012B234B08D1012A06D11A7080
S21444D7600022214B1A700223237014E000221A7000
S21444D770124B1B787BB90323F6E7FFF78FFFFEF7C0
S21444D78077FBFEF7EDFB0D4B1B7823B9174B1B6855
S21444D790023B012BEFD910BD154B00221A80012203
S21444D7A0144B1A700423DFE7FFF7D4FE0523DBE7A8
S21444D7B00023BDE70023D7E76818402069184020B7
S21444D7C06718402063184020501B40202C1B4020E4
S21444D7D06E1840206D1840206C1840206B1840206E
S21444D7E0701840207518402072184020581C40205D
S21444D7F01A18402074184020074B1A221A60032235
S21444D800064B1A601322064B1A600122054B1A6017
S21444D810054B064A1A607047A81B4020A41B4020AC
S21444D820A01B40209C1B4020981B4020EFAB0300CD
S21444D8307047704730B53D4C85B03D48237801A9C4
S21444D8400193019B1B020193019A6378134401934D
S21444D850019B1B020193019AA37813440193019BF5
S21444D8601B020193019AE3781344019323790293AC
S21444D870029B1B020293029A637913440293029B0F
S21444D8801B020293029AA37913440293029B1B023F
S21444D8900293029AE37913440293237A0193019BF9
S21444D8A01B020193019A637A13440193019B1B0262
S21444D8B00193019AA37A13440193019B1B0201939B
S21444D8C0019AE37A13440193237B0293029B1B023F
S21444D8D00293029A637B13440293029B1B020293B5
S21444D8E0029AA37B13440293029B1B020293029A5E
S21444D8F0E37B1344029342F21273019342F213738E
S21444D900029300F0B0FB04F1100004F1080104F1A6
S21444D9101802082314F8015B013B00F8015B11F878
S21444D920015B02F8015BF5D105B030BD841142209D
S21444D930808080000C4A0823002102F1280030B47D
S21444D94002F1080502F12004013B02F8011B05F828
S21444D950011B13F0FF0304F8011B00F8011BF3D16D
S21444D96030BCFFF767BF00BF841142204F4BF0B571
S21444D9701B688BB002934E4B1A6803925A68049203
S21444D9809B68059342F21273029A9A4200F0898089
S21444D990484800F013FBFFF7CDFF002346480AAA89
S21444D9A050F8231002EB83020133082B42F8201C64
S21444D9B0F5D1002340480AAA50F8231002EB83020C
S21444D9C00133082B42F8201CF5D102990025039A0E
S21444D9D0049B0598394C00903948264600F0EEFAE8
S21444D9E0029B38481B0E2370029B1B0C6370029BE1
S21444D9F01B0AA370029BE370039B1B0E2371039BBD
S21444DA001B0C6371039B1B0AA371039BE371049B6A
S21444DA101B0E2372049B1B0C6372049B1B0AA3728B
S21444DA20049BE372059B1B0E2373059B1B0C6373BD
S21444DA30059B1B0AA373059BE37300F0B6FA0135F6
S21444DA4016F8010B00F0DAFA082DF8D11E4D002620
S21444DA5000F0CBFA1D482F4600F0A7FA013617F817
S21444DA60010B00F0CBFA082EF8D100F0BEFA184BA2
S21444DA70002203F1080703F1100003F1180194464D
S21444DA80013214F8016B15F801EB082A03F8016B10
S21444DA9007F801EB00F8016B01F801CBF0D10BB0AD
S21444DAA0F0BD0C4800F08AFA77E700BF808080001B
S21444DAB0848080003290460010808000841142208A
S21444DAC056904600739046008C1142207D90460046
S21444DAD09411422048904600194A08211948F0B546
S21444DAE092F8A53100F1100C00F1080500F1180772
S21444DAF0012B9CBF002382F8D431002310F8014B3D
S21444DB0001391CF8016B17F801EBB4422E7818BFA4
S21444DB10013344EA060418BFDBB2764505F8014BE8
S21444DB201CBF0133DBB211F0FF01E7D133B1B2F8C9
S21444DB30BE301BB9BDE8F040FFF77CBEF0BD00BF69
S21444DB40C0114220841142201FB5144B01A953F83A
S21444DB5020305A1E073312F8010F9A4201F8010B7F
S21444DB60F9D19DF804300024502B8DF80C4007D092
S21444DB70432B0CD0422B0DD0552B08BF4FF44004FA
S21444DB800DF1050000F04CFA204404B010BD4FF4EB
S21444DB908004F5E74FF40004F2E700BF1821402064
S21444DBA02DE9F04F5C4D8DB082462B6805F1080890
S21444DBB006AC09A963F07C4340462E46A9462B6032
S21444DBC04246082316F8017B013B04F8017B9BB2CE
S21444DBD010F8017B01F8017B002BF3D1BAF10A0F50
S21444DBE00BD141464C4C0823FF20013B04F8010B63
S21444DBF001F8010B9BB2002BF7D1484BC8240021F7
S21444DC00013C03F8011BA4B2002CF9D12646444932
S21444DC10DFF808B104F1080380279BB200932B7801
S21444DC201F4203D198F800301F4248D051F82430A0
S21444DC300DF10C0C581E073310F801EF98420CF8FF
S21444DC4001EBF9D14FF000038DF814309DF80C30F9
S21444DC50502B59D0432B59D0422B5AD0552B34D124
S21444DC604FF440030DF10D00019300F0D9F9019BE8
S21444DC7095F800C0184498F800302A4A3B404FEACA
S21444DC80102E274918BF082317EA0C0F4FEA104CEA
S21444DC9018BF43F001030BF806C006F1010C1FFA47
S21444DCA08CFC0BF80CE006F1020C1FFA8CFC0BF80B
S21444DCB00C00F01C043680B2B6B20BF800300134C7
S21444DCC0009B7F08A4B2A342A9D1013508F10108FC
S21444DCD095429FD1BAF10A0F0FD19DF81A30BDF87C
S21444DCE0182089F80230A9F800209DF82630BDF89F
S21444DCF0242089F80A30A9F80820084B0022304628
S21444DD009A550DB0BDE8F08F0023ABE74FF480037F
S21444DD10A8E74FF40003A5E7841142204E22402092
S21444DD20182140208C114220F0B50D4C08220020CA
S21444DD3004F1080514F8016B082380210E4202D131
S21444DD402F78394201D0013080B2013B49089BB25A
S21444DD50002BF3D1013A013592B2002AEAD1F0BD44
S21444DD60841142202DE9F04FDFF8B480002685B0B8
S21444DD708346A8F1080A3446284B022E4FF0800901
S21444DD804FF0000234BF082703272744BFB29AF84F
S21444DD90001019EA010F04D198F8001019EA010F8F
S21444DDA02DD053F8241001AD481E073110F801CF8A
S21444DDB0814205F801CBF9D19DF804108DF80C206A
S21444DDC0502914D0432914D0422915D055291CD1A2
S21444DDD04FF440050DF1050000F022F905440F4BC1
S21444DDE000225D450BD1E0B205B0BDE8F08F0025BA
S21444DDF0F0E74FF48005EDE74FF40005EAE7013419
S21444DE004FEA5909A4B2A742C1D1013608F1010824
S21444DE100AF1010A082EB0D1FF20E5E71821402078
S21444DE208C1142202DE9FF4700240746204EA14688
S21444DE30022C4FF0000834BF4FF0080A4FF0030A94
S21444DE40336801A95A1E073312F8010F9A4201F8A3
S21444DE50010BF9D19DF804308DF80C90502B0DD061
S21444DE60432B15D0422B16D0552B17D001340436ED
S21444DE70082CDDD1FF2004B0BDE8F08700250DF165
S21444DE80050000F0CDF80544BD420AD1E0B2F2E701
S21444DE904FF48005F3E74FF40005F0E74FF44005F0
S21444DEA0EDE708F101081FFA88F39A45C8D8DDE77C
S21444DEB0182140202DE9F04FDFF8C490002585B0A6
S21444DEC08346A9F108082C462B4A022D4FF0800AB7
S21444DED04FF0000134BF082703272744BFB298F801
S21444DEE000001AEA000F04D199F800001AEA000F5D
S21444DEF032D052F824000DF1040C461E073016F8B2
S21444DF0001EFB0420CF801EBF9D19DF804008DF80E
S21444DF100C10502818D0432818D0422819D0552819
S21444DF2020D14FF440060DF1050000F079F8064480
S21444DF30124B00215E45104A0ED15955E0B21D449D
S21444DF40297205B0BDE8F08F0026ECE74FF4800652
S21444DF50E9E74FF40006E6E701344FEA5A0AA4B26A
S21444DF60A742BCD1013509F1010908F10108082D81
S21444DF70ABD1FF20E5E700BF1821402084114220A2
S21444DF808C1142207047092894BF30303730C0B2D5
S21444DF90704707B501220DF107018DF807000020F0
S21444DFA013F0CEFB03B05DF804FB10B5441E14F822
S21444DFB0010F00B910BDFFF7ECFFF8E70FB400B54A
S21444DFC0C3B044AA02A852F8041B019204F06CFCA5
S21444DFD0002302A88DF805318DF80631FFF7E5FFDA
S21444DFE043B05DF804EB04B070470D2008B5FFF766
S21444DFF0D0FF0A20BDE80840FFF7CBBF10B5044663
S21444E0000009FFF7C0FFFFF7C4FF04F00F00FFF757
S21444E010BAFFFFF7BEFF2C20BDE81040FFF7B9BF9C
S21444E020002330B51A46441E184614F8011F3929F1
S21444E03008D82F290AD95D1C01F00F0303EB001002
S21444E0402B4606E0A1F14105052D06D900B943B19A
S21444E05008220132072AE8D930BD5D1CA1F13703F6
S21444E060ECE71D46EAE7002070470000034A92F8B2
S21444E0709E30013382F89E30704700BFC011422064
S21444E08010B52A4C94F89A30642B94BF013300237D
S21444E09084F89A3094F8C63043B1013BDBB284F836
S21444E0A0C6301BB984F8C53084F88A3194F8C73032
S21444E0B053B1013BDBB284F8C7302BB994F88A21BC
S21444E0C0032A08BF84F88A31B4F8E4315BB1013BD3
S21444E0D09BB2A4F8E43133B9012284F8CF3184F8F2
S21444E0E0C13184F8A52194F8C231013384F8C23191
S21444E0F0FFF7F2FC94F8A13123B1002084F8A10183
S21444E10001F01FFCB4F8BE3073B1013B9BB2A4F8D7
S21444E110BE304BB984F88A3184F8C53084F8A331CC
S21444E12084F8C13184F8DC3110BD00BFC0114220F0
S21444E130034A92F89830013382F89830704700BF0B
S21444E140C011422070470323002010B5064CA4F8A3
S21444E150EC3104F154020823E16CF4F7F7FB002396
S21444E16084F8953010BD00BFC0114220024B0022F7
S21444E170C3E91522704700BFC011422030B5224B78
S21444E180002201244FF4FB604FF4FA61082583F81B
S21444E190A541A3F89820A3F8B420C3F8D420A3F844
S21444E1A0CA20A3F8CC2083F88121A3F8822183F8DF
S21444E1B08C2183F89C21C3F8A02183F8D62183F8C8
S21444E1C0DB2183F8DC21A3F8E42183F8EA21A3F8D1
S21444E1D0C220C3F8C420D864196083F89450A3F8C6
S21444E1E0C621C3F8D02183F8D421C3E972424FF440
S21444E1F00C14C3E92E22C3E96122C3F8C04183F854
S21444E200C421C3E92B1030BDC0114220144B002258
S21444E21093F88D1183F88A21E1B90322A3F8861175
S21444E22083F8542093F8882142F0400283F855201E
S21444E23093F89C21012A01BF7F2283F855200022AF
S21444E24083F89C21B3F8862152BAA3F856200022BC
S21444E2509A65704746F60362A3F85420E8E700BF81
S21444E260C0114220054B3022A3F854200A2283F8DA
S21444E27056200D2283F8C720704700BFC0114220A5
S21444E280034B012283F8C5200B2283F8C62070472F
S21444E290C011422008B5FFF783FC0330284B81B2F7
S21444E2A0284AC0B207291DD85921C3F8982183F8B3
S21444E2B0540083F8551093F89E1183F85610FF21A6
S21444E2C083F85710117883F85810517883F859100A
S21444E2D09178D27883F85A1083F85B200422A3F806
S21444E2E0CA2008BDA3F8CC10090AC3F8982141F007
S21444E2F0100183F8550083F85410592183F85610BA
S21444E30093F89E1183F85710FF2183F8581011781C
S21444E31083F859105178927883F85A1083F85B2022
S21444E3200322A3F8CA20012283F8C520022283F8D8
S21444E3308A21212283F88C21222283F88821D0E75F
S21444E340C01142204E224020024B002283F8542023
S21444E350704700BFC011422038B5CB1C40F6FF744E
S21444E3609BB2A34228BF2346174C1D0A84F8553057
S21444E3706223A4F8CC1045F0100584F8580084F8BD
S21444E3805630030A84F85450022163F00F03C4F84D
S21444E390982184F857300123A4F8CA301378A4F897
S21444E3A0CA1084F85930537884F85A300323A4F8B2
S21444E3B0CA30937884F85B30FFF762FF212384F8F1
S21444E3C08A1184F88C3138BDC0114220F0B5C84C4F
S21444E3D087B094F8C2310133DAB21B064ABF002331
S21444E3E084F8C22184F8C231B4F8C63113B1013B73
S21444E3F0A4F8C63194F8A03123B1002384F8A031A0
S21444E400FFF798FA94F88A51012D40F0288194F841
S21444E41088312E2B3DD146F60362A4F854206289F7
S21444E420A4F8562094F88D210D2A0BD1002384F8A5
S21444E4308A31012384F8953040F2F513A4F8BE30AF
S21444E44007B0F0BD0E2AF4D194F88911A948049176
S21444E450A9490391B4F8CA10CDE9012194F8C5201E
S21444E46029460092B4F88421FFF7A8FD94F8893130
S21444E470012B03D1002001F064FAD7E7022B03D125
S21444E480002001F079FAD1E7FF2BCFD184F8CB51A5
S21444E490CCE7222BCAD1B4F88431B3F5A06F6BD144
S21444E4A0964D0022964915F8010B134601321F2853
S21444E4B092B204D9322A01F8010BF4D11346E21879
S21444E4C02C213A2082F8E4105A1C422114FA82F293
S21444E4D082F8E4109A1C4F2114FA82F282F8E4106F
S21444E4E0DA1C14FA82F282F8E4101A1D542114FA43
S21444E4F082F282F8E4105A1D562114FA82F282F807
S21444E500E410991DDA1D14FA81F192B281F8E40000
S21444E5107C49087842281FD022444E2182F8E410D1
S21444E52003F10802302114FA82F282F8E41003F16F
S21444E5300A010933202289B214FA83F383F8E420CB
S21444E5406318002201314FF4A06083F8E42089B2B6
S21444E5506B4AFFF701FF6CE70B466B4D1878114684
S21444E56001321F2892B2EBD901332144AB4281F8E1
S21444E570E400F3D11146E3E7644EB4F8862106EB93
S21444E5804316B4F886C14FEA122E3789D0B29CFAA5
S21444E5909CFCF268FB1C99B2DBB207292FD984F89D
S21444E5A05530C1F30321622384F857E041F010014B
S21444E5B084F8580084F85630002384F85410022116
S21444E5C0A4F8CA30C4F89821A4F8CC701378A4F8F8
S21444E5D0CA5084F859305378A4F8CA1084F85A308C
S21444E5E0937884F85B300323A4F8CA30FFF748FED8
S21444E5F0322384F88A1184F8C630212374E06221D9
S21444E60084F85430A4F856C0013384F855100021D9
S21444E610C4F89821DBB2A4F8CA10A4F8CC701078D9
S21444E620A4F8CA5084F85800507884F85900022058
S21444E630A4F8CA00907884F85A000320A4F8CA00C4
S21444E640D27884F85B200422A4F8CA20DAB2082AD6
S21444E6503FF4ECAEE218013382F85410F6E7022D8C
S21444E6607FF4EEAE94F8C530002B7FF4E9AE94F810
S21444E6708831222B7FF4DDAE94F8C430012B06D9C2
S21444E680023BDBB284F8C430002B7FF4D9AE94F856
S21444E690C330072194F88C212E27B4F8CC50D4F8F4
S21444E6A09861134884F8C43084F85420B4F8CA30C7
S21444E6B001390130AB4238BF16F803C003F10103F9
S21444E6C02CBF80F8547080F854C09BB211F0FF0100
S21444E6D0A4F8CA30EAD19D4202F10103DBB298BFE6
S21444E6E084F88A112F2B88D884F88C31A1E600BF91
S21444E6F0C01142207693460058134220000144003D
S21444E700A41242202010400039104000D08A46000F
S21444E710FFF75CBE38B51B4C6389A4F89E31FFF7FF
S21444E72013FE94F89E5105F0F703022B05D10123FE
S21444E730002584F89D31284638BD012D0FD145F675
S21444E740061384F85650A4F8543094F89F3184F84D
S21444E7505730FFF7E9FA40BAA4F85800EBE7032D20
S21444E76012BF47F6027345F6021384F856504FF02C
S21444E77001051BBFA4F854301223A4F8543084F87F
S21444E7805630D8E7C011422008B5FFF7DDFD0B4BE5
S21444E7904CF20252A3F854209A7A012A83F856205F
S21444E7A004D1002283F8D421012008BD022A01D1D5
S21444E7B00122F7E77F2283F85520F5E7C01142206F
S21444E7C0064B47F60372A3F85420012283F85600FA
S21444E7D083F8571083F89C21704700BFC01142202D
S21444E7E0074B93F8D621132A09D093F8A521032A78
S21444E7F01FBF7F2283F8D621012283F89C217047CD
S21444E800C0114220002310B56B4C84F8D63194F8DE
S21444E810CE30222B07D194F8D531032B09D01323BD
S21444E82084F8D63105E0202B14D194F8D531022B48
S21444E830F5D894F8D63163B147F6037284F8573066
S21444E8400123A4F8542094F8CE2084F89C3184F80C
S21444E850562010BD102B0BD194F8D531022BDED1A7
S21444E860A37A03F07F03013B022BE2D91223D7E7B6
S21444E870852B12D1A37A013B012B84BF122384F843
S21444E880D63194F8D531022B02D0132384F8D631EE
S21444E89094F8D601FFF7A4FFCBE7272B05D194F8CD
S21444E8A0D53103F0FB03022BB8E7192B18D194F8A3
S21444E8B0D531012BB3D0A27A0A2AF4D0032AF2D057
S21444E8C0022AAAD0042A08D1062BA8D1A37B012B5E
S21444E8D0AFD0FF2BADD03123A2E7012AC6D19CE7A7
S21444E8E0282B1DD194F8D511A27A032902F07F0370
S21444E8F005D0002BC9D0032BC7D0022902D0591EFD
S21444E9000129C2D912F07C0F01D01223BEE7E27A65
S21444E910013A022ABCD90BB1032BB9D13123B5E74E
S21444E920142B1CD194F8D531042B7FF478AFE07ABD
S21444E930A37A00EB0323207B00EB03206FF07F4396
S21444E9409842C4F8D0013FF474AF1C4B98423FF44D
S21444E95070AFFFF767FAFF287FF46BAFBBE73E2B39
S21444E96011D194F8D531022B7FF459AFA37A13F022
S21444E9707F0F4FF4FA7318BF1222A4F8E43118BF7D
S21444E98084F8D62155E7312B09D194F8D531062B96
S21444E9903FF645AFA37A013B022B9CD849E72E2B82
S21444E9A005D194F8D531022B7FF639AF41E70F2BCA
S21444E9B03FF63FAF112333E7C0114220FF0040002B
S21444E9C04FF287139842134B0ED10A290AD10022DC
S21444E9D083F8D62193F8D621003A18BF012283F84B
S21444E9E0DB2170471322F3E74FF28B12904201D19A
S21444E9F00429EBE74FF29512904201D10329E5E74B
S21444EA004FF293129042F9D04FF28C129042DED1DC
S21444EA100729DBE7C01142200B4B024693F90A0054
S21444EA20997A0028B3BF01F07F02012083F855206D
S21444EA300020B8BF9A724FF00102A8BF83F8540072
S21444EA4083F8A521704700BFC0114220274B0146DA
S21444EA5010B593F90A009A7A0028BBBF02F07F02E9
S21444EA60002001209A729A7A541E022C31D8062429
S21444EA7083F85510022A4FF0000183F854404FF4AF
S21444EA80997483F85620A3F858404FF0F40483F85A
S21444EA90571083F85A404FF4FA7483F8A521A3F824
S21444EAA0E44112D1124A1278422A06D102F5800273
S21444EAB002F6DF7212784F2A03D0012283F89C2193
S21444EAC003E00122084683F8CA21002283F8CF21B6
S21444EAD010BD47F60372A3F8542093F8CE2083F86B
S21444EAE05620122283F85720E7E700BFC011422081
S21444EAF02010400010B5214CA37AE07A00EB0320A6
S21444EB0080B2B0F5754FA4F886010BD14FF4A063DC
S21444EB10A4F884310123002084F88A31222384F81F
S21444EB20883111E0B0F5704F12D300F0A9FD4FF6CE
S21444EB30FF73984209D10223012084F85430637A43
S21444EB4043F0400384F8553010BDA4F88401E1E74F
S21444EB5040F2DF73D4F8E001C01A47F60373A4F812
S21444EB60543018BF012094F8CE3084F85630312300
S21444EB7084F85730012384F89C31E5E7C0114220DD
S21444EB802DE9F0414E4C2E23A27AE07A84F888315F
S21444EB90130900EB0220217B0E2B84F88D3180B2C2
S21444EBA084F88911A4F886010DD10123002084F845
S21444EBB08A3194F8DB31012B71D1424A626584F87C
S21444EBC09C31BDE8F081B0F5704F13D300F0C3FD1F
S21444EBD00F230246A4F8840184F88D314FF6FF7360
S21444EBE0984204D0384E06EB4013D96921B9032322
S21444EBF084F8DB310120DCE794F8CF11012901D0F9
S21444EC000223F5E7002084F89C0194F8DB010028F1
S21444EC10F0D19B6894F8D5010333DBB2984207D011
S21444EC2013232A4884F8DB1184F8D631FFF7C6F953
S21444EC30B4F884310027DFF89C80042506EB4313A0
S21444EC40A4F8CA70DA689B68C4F89421A4F8CC3057
S21444EC50B4F8CA3018F8011BD4F89421D154B4F847
S21444EC60CA30B4F8CC2001339BB29A42A4F8CA30D6
S21444EC70C0D90020FFF7CAFA94F89C3184F8DB71B7
S21444EC8043B9B4F8843106EB4313DB69012B08BF60
S21444EC9084F8A131013D15F0FF05D9D1AAE7022B2E
S21444ECA003D10B4B6365012389E7032B01BF03F1B3
S21444ECB0445303F5391303F57C53636581E700BF7A
S21444ECC0C0114220037F2E13D08A4600C7934600C5
S21444ECD0037F2E33CC114220204B014630B593F9A6
S21444ECE00A009A7A0028BBBF02F07F020020012067
S21444ECF09A72DA7A02F0FD04012C22D19A7A02F052
S21444ED00FD05012D11D183F8DC5193F8A521012A84
S21444ED104FF0020283F854201AD87F225A722222D5
S21444ED209A72002283F8DC2130BD12B983F8DC21C4
S21444ED30EBE7022A06BF002083F8DC4183F89C41B7
S21444ED40E3E7022A1FBF7F225A7212229A72DCE736
S21444ED509A7A83F8551083F85620E5E7C011422086
S21444ED60704770477047704750B123230549013BAD
S21444ED7000284FEA40009BB2B8BF4840002BF6D16B
S21444ED80704700BF69696C6CF8B56C4B064693F8DF
S21444ED90A5211C46012A0BD847F60372A3F8542033
S21444EDA05A7A83F856207F2283F8572001253DE07F
S21444EDB0997A01F0FB05012D4AD1062384F85500C3
S21444EDC084F8561084F8543094F8CF31012B2FD160
S21444EDD001292DD10023A4F8A631A4F8A83194F82B
S21444EDE0A661012994F8A72194F8A83118BF0221F6
S21444EDF084F8582002EB062294F8A90184F8593086
S21444EE0003EB022384F85A0000EB032084F857608F
S21444EE10FFF7AAFF030E84F8A631030C40BA84F821
S21444EE20A7310123A4F8A80184F8C1312846F8BDC7
S21444EE3094F8C23103F1110284F8A63184F8A7216C
S21444EE4003F12202343384F8A82184F8A931C6E7B2
S21444EE50022DABD193F8C121012A4FF0000210D005
S21444EE6083F8C12147F603720125A3F8542093F88A
S21444EE70CE2083F89C5183F85620242283F85720CA
S21444EE80D4E783F8C121DA7A93F8A6319A420AD1B4
S21444EE90227B94F8A7319A4205D1B4F8A821B4F855
S21444EEA00D309A421DD047F603730629A4F8543011
S21444EEB094F8CE3084F856304FF0350384F8573003
S21444EEC04FF0010384F89C317FF470AF1C4B1B78E1
S21444EED0422B08D001231B4884F89C31FFF76EF878
S21444EEE001E00629F2D094F89C51002D7FF45EAFE1
S21444EEF0A37A022784F8556084F8563084F8547010
S21444EF00FFF721F9A37A062B0ED101230E4884F885
S21444EF10CF7184F8CA31FFF748F80B48FFF745F835
S21444EF200948FFF742F881E794F8A531023B012BE4
S21444EF309CBF012384F8CF3178E700BFC01142203C
S21444EF4020104000DB93460039944600114B0022C3
S21444EF5093F89C1183F8D621012904BF7F2183F8B6
S21444EF609C2193F8CE2008BF83F85510312A0DD142
S21444EF7093F8D511062903D9132283F8D62103E042
S21444EF80997A01390229F8D801207047342AFBD1EE
S21444EF901222F2E7C011422070B5674C0025637A0E
S21444EFA0264694F8DD2184F8CE30237A84F89C51A2
S21444EFB09A4284F8D53101D800200FE0013B062B55
S21444EFC0FAD8FFF71FFC94F89C31012B0FD1D4F8E4
S21444EFD0E02140F2DF739A4201D0012070BD94F8DC
S21444EFE0D631113B012BF8D884F89C51E4E7627A79
S21444EFF094F8CE30102A43F0400003D1BDE8704068
S21444F000FFF724BD202A03D1BDE87040FFF704BDB6
S21444F010852A03D1BDE87040FFF7B6BB2A2B0AD138
S21444F020E37A84F8C33146F60223A4F85430A37A2C
S21444F03084F85630D1E7222B04D16220BDE87040D4
S21444F040FFF758BD2E2B04D16E20BDE87040FFF765
S21444F05097BD282B04D16820BDE87040FFF73CBE1E
S21444F0602F2B0ED146F60673344AA4F854300623A2
S21444F070013B12F8011B13F0FF0382F84B10F7D143
S21444F080ABE7142B15D1FFF75FF9D4F8D0016FF036
S21444F0907F43984202D02A4B984207D1012386F8F0
S21444F0A0A03145F20143A6F8543096E7FEF702FF36
S21444F0B0F7E7272B04D16720BDE87040FFF764BE0E
S21444F0C0192B03D1BDE87040FFF724BB312B0BD17D
S21444F0D01C4A0723013B12F8011B13F0FF0382F876
S21444F0E0DA10F7D1712079E7112B0FD145F20213CC
S21444F0F0A4F85430A37A84F85630FFF724F812481C
S21444F100FEF753FF1148FEF750FF66E73E2B0FD13C
S21444F11094F90A10A37A0029FFF64EAF022142F072
S21444F120400284F8563084F8541084F8552054E746
S21444F130FEF79CFF40E700BFC0114220CA114220A0
S21444F140FF004000C9114220E5934600FA9346006A
S21444F15038B5424C0F2384F88D312546237A217BDB
S21444F16003F00F02637AE07A03EB022304F1E4022D
S21444F17001EB0020C4F8942142F2030280B2A4F8C2
S21444F180CC30A4F88A2194F8CE202F2A23D1033BEE
S21444F1902E22A4F87A019BB284F8882104F22F1216
S21444F1A0A4F88601A4F8CC3084F87931A37BC4F85B
S21444F1B0942184F831310423627BA4F8CA30E37B7B
S21444F1C084F87C2184F82F1184F8302184F8323175
S21444F1D0FFF748F814E0A4F8860100F051FA4FF619
S21444F1E0FF7398420ED147F603723123A5F8542094
S21444F1F095F8CE2085F8D63185F8562085F85730D0
S21444F200012038BD164B03EB4013DA69002AEAD0D6
S21444F2102E22A4F8840184F88821032284F88A21C3
S21444F220DA689B68C4F89421A4F8CC300123A4F887
S21444F230CA30637B1370B4F8CA30D4F89421591C8E
S21444F240A4F8CA10A17BD154B4F8CA30D4F8942197
S21444F250591CA4F8CA10E17BD154B9E7C011422026
S21444F260D08A460008B51A4B0022197A83F88D21B5
S21444F27001F00F00597AA3F8842101EB00219A7A11
S21444F280C82983F888211A7B88BFC82183F8E520DB
S21444F290A3F8CC10D97A02EB01205A7B83F8E41009
S21444F2A083F8E6209A7BA3F8860142F2030083F8AB
S21444F2B0E720DA7BA3F88A0183F8E820052205488C
S21444F2C0A3F8CA20C3F89401FEF7CCFF012008BD7A
S21444F2D0C01142204E224020184B0022987A83F8D0
S21444F2E0D62183F89C21A0F12E0283F8CE00D1B219
S21444F2F008291DD840F24912CA40D24312F00102EE
S21444F30016D12E2883F8DB2114D193F8A521012A9F
S21444F31002D993F8CF216AB97E2283F8D62102F126
S21444F3207E2202F5381285325A65012283F89C21E2
S21444F330012070470020FFF70BBF00BFC0114220DA
S21444F340002340F2F51210B5884C84F8983084F8BF
S21444F3509C31A4F8BE204FF4FA72C4E915332368EE
S21444F360A4F8E421B3F5FA6F17D1431E04F108025A
S21444F370073013F8011F984202F8011BF9D14FF4E5
S21444F380FA63C4F8E031227A12F0F0032BD1FFF787
S21444F39003FE002840F08B804CE040F2DF7293423C
S21444F3A020D1037813F0F00F1CD14278A2F1100359
S21444F3B0DBB2182B11D9852A01D03E2A12D140F24D
S21444F3C0DF736B4AC4F8E031431E073013F8011F5D
S21444F3D0834202F8011BF9D1D5E7664A22FA03F3C1
S21444F3E0DB07ECD410BD102B02D1FFF775FFD0E736
S21444F3F0202B40F08F8094F8CE302E3BD9B206298D
S21444F4005CD84923CB40DB4313F0010356D194F830
S21444F4108A1103290ED194F8DD11072910D8B4F8BF
S21444F420CA3001391944B4F8CC30994202D2002388
S21444F43084F88A31002384F89C3184F89830D1E7E4
S21444F44094F88B11914205D14B4884F88A31FEF7E3
S21444F450ACFDEFE784F88B210D2284F8C72094F89E
S21444F460DB2132B9E218D4F89411507AB4F8CA20A1
S21444F4708854B4F8CA20B4F8CC10013292B29142FF
S21444F480A4F8CA2042D894F8DB31012B1AD147F6A7
S21444F4900372A4F8542094F8CE2084F856201322FD
S21444F4A084F8572084F89C31002384F8DB3194F8A0
S21444F4B09C31012B04BF7F2384F85530012384F804
S21444F4C09530B7E7022B0CD147F60373A4F85430B3
S21444F4D094F8CE3084F85630332384F857300123DA
S21444F4E0E0E70020FEF792FEB4F88421234B94F81C
S21444F4F09C1103EB42132248DA69012A08BF84F8B8
S21444F500A12194F8A131FEF759FDCDE70133072B2D
S21444F510A5D18FE7302B8DD194F8DD31022B86D9D7
S21444F520312A03D10B2384F8C63083E794F8C530D8
S21444F5305BB9322A09D146F20323A4F85430B4F80E
S21444F54086315BBAA4F856304CE7A37A0021312AB8
S21444F55003F1030384F8C51084F8C610DBB284F8BC
S21444F560C33084F8C4303FF662AF63E7C01142202C
S21444F570C8114220130204010A944600D08A460069
S21444F580229446000A4810B5FEF718FD72B64FF0AE
S21444F590005308491022084C0848C3E90012FEF7F5
S21444F5A00DFDFAF766FA2046FEF708FDFBE700BFB6
S21444F5B0349446007154CA3D5B94460041944600D8
S21444F5C038B52C4B93F8C8211C4632B9FEF7D6FD05
S21444F5D02948BDE83840FEF7E8BC93F89820002A4E
S21444F5E03FD0002293F89D1183F8982081B193F878
S21444F5F09E0183F89D21FEF74DFE012384F8953045
S21444F60040F2F513A4F8BE30BDE83840FEF79BBD83
S21444F61093F89550002DF3D1184A13780133DBB292
S21444F620022B01D8137038BD1570FEF7CFFE94F840
S21444F630993094F8C22101330132DBB284F8C221F6
S21444F640042B84F899300CD984F89950FEF718FDA9
S21444F650B4F89C30C72B96BF0133A4F89C50A4F84A
S21444F6609C3094F8CA2194F8CB311343DBD0FFF78F
S21444F67089FF00BFC01142206A94460014224020ED
S21444F6804FF22803984218D84FF20F03984259D99C
S21444F690A0F57040113817280DD8DFE800F0562939
S21444F6A02B2D2F3131333537393B3D3F414345458B
S21444F6B047494B4D4F51042070474FF2931398429D
S21444F6C045D00CD84FF28713984242D04FF2881256
S21444F6D04FF6FF73904214BF1846012070474FF20E
S21444F6E095124FF6FF73904214BF18460220704797
S21444F6F00620704707207047082070470920704747
S21444F7000A2070470B2070470C2070470D20704726
S21444F7100E2070470F207047102070471120704706
S21444F72012207047132070471420704715207047E6
S21444F73016207047172070471820704719207047C6
S21444F7401A2070474FF6FF70704705207047032015
S21444F750704700207047FFF793BF1C280146F0B55A
S21444F76085B037D83F4B420103EB40169C584FF6C2
S21444F770FF739C422ED0F369012B2BD1756804F598
S21444F7800004B368AD082246009337482B46FEF77C
S21444F79015FCD6E903639A1E012A1DD8002315E0FA
S21444F7A036F82310023389B2029102990904029171
S21444F7B05088029901440291918889B20391039931
S21444F7C009040391D188039A0A4403929D4206EBA6
S21444F7D08302E5D805B0F0BD043B012B3FD9002792
S21444F7E0BD4206EB8701F5D916F827302046023786
S21444F7F00834DBB20293029B1B0602934A78029BB0
S21444F80003EB024302938A78029B03EB02230293A0
S21444F810CB78029A134402930B79DBB20393039B8F
S21444F8201B0603934A79039B03EB024303938A79AB
S21444F830039B03EB02230393CB7902A9039A134455
S21444F8400393FEF710FCCBE756F8231002330291DD
S21444F850526803929D4206EB8302F5D8BAE700232A
S21444F860F8E700BFD08A4600759446001C28014637
S21444F87030B403D92C4830BCFEF7A0BB42012B4B16
S21444F88003EB40109B584FF6FF7293421FD0C26959
S21444F890012A1CD10169072919D0826803F500039F
S21444F8A0C468881E012814D85208023400219142A4
S21444F8B00DD253F8040B050C24F8025C4D1C9542FB
S21444F8C005D2023180B28A4224F8040BEFD830BC09
S21444F8D070470439012925D822F003022244944271
S21444F8E0F5D053F8041B44F8041BF8E75858050EA3
S21444F8F025704D1CAA42EAD9C0F3074565708D1C95
S21444F900AA42E4D9C0F30725A570CD1CAA42DED985
S21444F9100431C0B204348A4204F8010CD7D9914267
S21444F920E4D3D4E70021FAE796944600D08A46000A
S21444F93010B50024A0B20134FFF798FF1D2CF9D16E
S21444F94010BD1FB50024A0B20134FFF706FF1D2CDE
S21444F950F9D1074B02A902934FF47C730393054BEA
S21444F96001930198FEF77FFB002004B010BD00BF52
S21444F97055EFCDAB1000800008B508B9FFF7D8FFA7
S21444F980002008BD124B00B51B688BB00293114B88
S21444F9901A6803925A6804929B6805930299039ADC
S21444F9A0049B059800900C48FEF708FB039BB3F5B0
S21444F9B07C7F06D10948FEF701FB01200BB05DF8B9
S21444F9C004FB0748FEF7FAFA4FF0FF30F6E700BFAD
S21444F9D01000800014008000A6944600BE944600A2
S21444F9E0C994460008B5FFF7CDFF012805D1FFF7B7
S21444F9F09FFFBDE80840FDF7B9BFFFF7C3FF0128E6
S21444FA00F5D00020FFF79DFFFFF7BCFFF1E700BFEE
S21444FA1010F8012B11F8013B012A28BF9A42F7D06F
S21444FA20D01A7047034613F8012B002AFBD1181A44
S21444FA30013870470000000000000000000000008D
S21444FA4001F0FF01102A2BDB10F0070F08D010F846
S21444FA50013B013A8B422DD010F0070F42B3F6D14A
S21444FA60F0B441EA012141EA014122F007047FF063
S21444FA7000070023F0E80256083C85EA010586EABA
S21444FA80010685FA47F5A3FA87F586FA47F6A5FAF6
S21444FA9087F68EB9EED1F0BC01F0FF0102F0070202
S21444FAA032B110F8013B013A83EA010313B1F8D1AD
S21444FAB00020704701387047002D06BF354603388E
S21444FAC0073815F0010F07D1013015F4807F02BFC7
S21444FAD0013015F4C03F0130F0BC0138704700BF18
S21444FAE081F0004102E000BF83F0004330B54FEAA6
S21444FAF041044FEA430594EA050F08BF90EA020F13
S21444FB001FBF54EA000C55EA020C7FEA645C7FEAA5
S21444FB10655C00F0E2804FEA5454D4EB5555B8BFC8
S21444FB206D420CDD2C4480EA020281EA030382EA39
S21444FB30000083EA010180EA020281EA0303362DCB
S21444FB4088BF30BD11F0004F4FEA01314FF4801C9E
S21444FB504CEA113102D0404261EB410113F0004FB0
S21444FB604FEA03334CEA133302D0524263EB430367
S21444FB7094EA050F00F0A780A4F10104D5F1200E05
S21444FB800DDB02FA0EFC22FA05F2801841F1000160
S21444FB9003FA0EF2801843FA05F359410EE0A5F134
S21444FBA020050EF1200E012A03FA0EFC28BF4CF065
S21444FBB0020C43FA05F3C01851EBE37101F000451B
S21444FBC007D54FF0000EDCF1000C7EEB00006EEB28
S21444FBD00101B1F5801F1BD3B1F5001F0CD34908B2
S21444FBE05FEA30004FEA3C0C04F101044FEA445209
S21444FBF012F5800F80F09A80BCF1004F08BF5FEA90
S21444FC00500C50F1000041EB045141EA050130BD6F
S21444FC105FEA4C0C404141EB0101013C28BFB1F581
S21444FC20801FE9D291F0000F04BF01460020B1FACC
S21444FC3081F308BF2033A3F10B03B3F120020CDA9F
S21444FC400C3208DD02F1140CC2F10C0201FA0CF07D
S21444FC5021FA02F10CE002F11402D8BFC2F1200CE2
S21444FC6001FA02F120FA0CFCDCBF41EA0C01904098
S21444FC70E41AA2BF01EB0451294330BD6FEA0404E1
S21444FC801F3C1CDA0C340EDC04F11404C4F12002CC
S21444FC9020FA04F001FA02F340EA030021FA04F3DE
S21444FCA045EA030130BDC4F10C04C4F1200220FA35
S21444FCB002F001FA04F340EA0300294630BD21FA73
S21444FCC004F0294630BD94F0000F83F4801306BF39
S21444FCD081F480110134013D4EE77FEA645C18BF2D
S21444FCE07FEA655C29D094EA050F08BF90EA020FC4
S21444FCF005D054EA000C04BF1946104630BD91EABC
S21444FD00030F1EBF0021002030BD5FEA545C05D1BE
S21444FD104000494128BF41F0004130BD14F58004FD
S21444FD203CBF01F5801130BD01F0004545F0FE4171
S21444FD3041F470014FF0000030BD7FEA645C1ABFA6
S21444FD40194610467FEA655C1CBF0B46024650EADD
S21444FD50013406BF52EA033591EA030F41F4002109
S21444FD6030BD00BF90F0000F04BF0021704730B58F
S21444FD704FF4806404F132044FF000054FF0000164
S21444FD8050E700BF90F0000F04BF0021704730B525
S21444FD904FF4806404F1320410F0004548BF4042FA
S21444FDA04FF000013EE700BF42004FEAE2014FEA4F
S21444FDB031014FEA02701FBF12F07F4393F07F4F2A
S21444FDC081F06051704732F07F4208BF704793F02D
S21444FDD07F4F04BF41F40021704730B54FF4607440
S21444FDE001F0004521F000411CE700BF50EA010243
S21444FDF008BF704730B54FF000050AE050EA0102EC
S21444FE0008BF704730B511F0004502D5404261EB5B
S21444FE1041014FF4806404F132045FEA915C3FF49C
S21444FE20D8AE4FF003025FEADC0C18BF03325FEA39
S21444FE30DC0C18BF033202EBDC02C2F1200300FAEA
S21444FE4003FC20FA02F001FA03FE40EA0E0021FA0F
S21444FE5002F11444BDE600BF70B54FF0FF0C4CF4FD
S21444FE60E06C1CEA11541DBF1CEA135594EA0C0FAF
S21444FE7095EA0C0F00F0DEF82C4481EA030621EAEA
S21444FE804C5123EA4C5350EA013518BF52EA033525
S21444FE9041F4801143F4801338D0A0FB02CE4FF0D7
S21444FEA00005E1FB02E506F00042E0FB03E54FF007
S21444FEB00006E1FB03569CF0000F18BF4EF0010EFF
S21444FEC0A4F1FF04B6F5007F64F5407404D25FEAFB
S21444FED04E0E6D4146EB060642EAC62141EA5551AE
S21444FEE04FEAC52040EA5E504FEACE2EB4F1FD0CF0
S21444FEF088BFBCF5E06F1ED8BEF1004F08BF5FEA6E
S21444FF00500E50F1000041EB045170BD06F000461F
S21444FF1046EA010140EA020081EA0301B4EB5C04CC
S21444FF20C2BFD4EB0C0541EA045170BD41F48011C4
S21444FF304FF0000E013C00F3AB8014F1360FDEBFE9
S21444FF40002001F0004170BDC4F10004203C35DAC5
S21444FF500C341BDC04F11404C4F1200500FA05F348
S21444FF6020FA04F001FA05F240EA020001F00042E9
S21444FF7021F0004110EBD37021FA04F642EB06015F
S21444FF805EEA430E08BF20EAD37070BDC4F10C0489
S21444FF90C4F1200500FA04F320FA05F001FA04F24D
S21444FFA040EA020001F0004110EBD37041F1000139
S21444FFB05EEA430E08BF20EAD37070BDC4F1200544
S21444FFC000FA05F24EEA020E20FA04F301FA05F2AC
S21444FFD043EA020321FA04F001F0004121FA04F254
S21444FFE020EA020000EBD3705EEA430E08BF20EA24
S21444FFF0D37070BD94F0000F0FD101F0004640005E
S21445000041EB010111F4801F08BF013CF7D041EADE
S214450010060195F0000F18BF704703F000465200E2
S21445002043EB030313F4801F08BF013DF7D043EAB3
S2144500300603704794EA0C0F0CEA135518BF95EA69
S2144500400C0F0CD050EA410618BF52EA4306D1D1F0
S21445005081EA030101F000414FF0000070BD50EA0F
S214450060410606BF1046194652EA430619D094EA99
S2144500700C0F02D150EA013613D195EA0C0F05D183
S21445008052EA03361CBF104619460AD181EA0301D7
S21445009001F0004141F0FE4141F470014FF000008F
S2144500A070BD41F0FE4141F4780170BD70B54FF02A
S2144500B0FF0C4CF4E06C1CEA11541DBF1CEA1355AA
S2144500C094EA0C0F95EA0C0F00F0A7F8A4EB05048C
S2144500D081EA030E52EA03354FEA013100F0888083
S2144500E04FEA03334FF0805545EA131343EA12634C
S2144500F04FEA022245EA111545EA10654FEA002601
S2144501000EF000419D4208BF964244F1FD0404F5B9
S214450110407402D25B084FEA3202B61A65EB030515
S2144501205B084FEA32024FF480104FF4002CB6EBD2
S214450130020E75EB030E22BFB61A754640EA0C0052
S2144501405B084FEA3202B6EB020E75EB030E22BF92
S214450150B61A754640EA5C005B084FEA3202B6EBD3
S214450160020E75EB030E22BFB61A754640EA9C0092
S2144501705B084FEA3202B6EB020E75EB030E22BF62
S214450180B61A754640EADC0055EA060E18D04FEA20
S214450190051545EA16754FEA06164FEAC30343EAC0
S2144501A052734FEAC2025FEA1C1CC0D111F4801F8D
S2144501B00BD141EA00014FF000004FF0004CB6E786
S2144501C011F4801F04BF01430020B4F1FD0C88BF25
S2144501D0BCF5E06F3FF6AFAEB5EB030C04BFB6EB30
S2144501E0020C5FEA500C50F1000041EB045170BD23
S2144501F00EF0004E4EEA113114EB5C04C2BFD4EB50
S2144502000C0541EA045170BD41F480114FF0000ED3
S214450210013C90E645EA060E8DE60CEA135594EA4F
S2144502200C0F08BF95EA0C0F3FF43BAF94EA0C0F52
S2144502300AD150EA01347FF434AF95EA0C0F7FF4C7
S21445024025AF104619462CE795EA0C0F06D152EA1B
S21445025003353FF4FDAE1046194622E750EA4106FF
S21445026018BF52EA43067FF4C5AE50EA41047FF410
S2144502700DAF52EA43057FF4EBAE12E74FF0FF3C75
S21445028006E000BF4FF0010C02E000BF4FF0010C46
S2144502904DF804CD4FEA410C7FEA6C5C4FEA430CBF
S2144502A018BF7FEA6C5C1BD001B050EA410C0CBF0E
S2144502B052EA430C91EA030F02BF90EA020F002070
S2144502C0704710F1000F91EA030F58BF994208BFD7
S2144502D090422CBFD8176FEAE37040F00100704794
S2144502E04FEA410C7FEA6C5C02D150EA013C07D1EB
S2144502F04FEA430C7FEA6C5CD6D152EA033CD3D036
S2144503005DF8040B704700BF8446104662468C462F
S2144503101946634600E000BF01B5FFF7B7FF002862
S21445032048BF10F1000F01BD4DF808EDFFF7F4FF8B
S2144503300CBF012000205DF808FB00BF4DF808ED16
S214450340FFF7EAFF34BF012000205DF808FB00BF39
S2144503504DF808EDFFF7E0FF94BF012000205DF85B
S21445036008FB00BF4DF808EDFFF7CEFF94BF012010
S21445037000205DF808FB00BF4DF808EDFFF7C4FF09
S21445038034BF012000205DF808FB00BF4FEA410C52
S2144503907FEA6C5C02D150EA013C0AD14FEA430C35
S2144503A07FEA6C5C02D152EA033C02D14FF0000072
S2144503B070474FF0010070474FEA410212F50012B0
S2144503C015D211D56FF47873B3EB625212D94FEA52
S2144503D0C12343F0004343EA505311F0004F23FA3C
S2144503E002F018BF404270474FF00000704750EA91
S2144503F0013005D111F0004008BF6FF0004070474E
S2144504004FF00000704700BF4A0011D212F50012A7
S21445041011D20DD56FF47873B3EB62520ED44FEA12
S214450420C12343F0004343EA505323FA02F0704792
S2144504304FF00000704750EA013002D14FF0FF30D0
S21445044070474FF0000070474FEA4102B2F1E04373
S21445045024BFB3F5001CDCF1FE5C0DD901F0004C61
S2144504604FEAC0024CEA5070B2F1004F40EB8300B1
S21445047008BF20F00100704711F0804F21D113F1DD
S2144504803872BCBF01F00040704741F480114FEA16
S2144504905252C2F11802C2F1200C10FA0CF320FA9F
S2144504A002F018BF40F001004FEAC1234FEAD323BC
S2144504B003FA0CFC40EA0C0023FA02F34FEA430326
S2144504C0CCE77FEA625307D150EA01331EBF4FF0AF
S2144504D0FE4040F44000704701F0004040F0FE40CA
S2144504E040F40000704700BF80F0004002E000BFC7
S2144504F081F0004142001FBF5FEA410392EA030FC5
S2144505007FEA226C7FEA236C6AD04FEA1262D2EB0E
S2144505101363C1BFD218414048404140B8BF5B4213
S214450520192B88BF704710F0004F40F4000020F0AC
S2144505307F4018BF404211F0004F41F4000121F0C2
S2144505407F4118BF494292EA030F3FD0A2F101020C
S21445055041FA03FC10EB0C00C3F1200301FA03F14A
S21445056000F0004302D5494260EB4000B0F5000F6D
S21445057013D3B0F1807F06D340084FEA310102F12C
S2144505800102FE2A51D2B1F1004F40EBC25008BFDE
S21445059020F0010040EA03007047490040EB0000A8
S2144505A0013A28BFB0F5000FEDD2B0FA80FCACF1A9
S2144505B0080CB2EB0C0200FA0CF0AABF00EBC250D6
S2144505C052421843BCBFD0401843704792F0000FC4
S2144505D081F4000106BF80F400000132013BB5E717
S2144505E04FEA41037FEA226C18BF7FEA236C21D08D
S2144505F092EA030F04D092F0000F08BF08467047F2
S21445060090EA010F1CBF0020704712F07F4F04D1BF
S214450610400028BF40F00040704712F100723CBFD2
S21445062000F50000704700F0004343F0FE4040F4FC
S214450630000070477FEA226216BF08467FEA2363BA
S2144506400146420206BF5FEA412390EA010F40F4A5
S214450650800070474FF0000304E000BF10F00043F1
S21445066048BF40425FEA000C08BF704743F09643D8
S21445067001464FF000001CE050EA010208BF7047F3
S2144506804FF000030AE000BF50EA010208BF70477A
S21445069011F0004302D5404261EB41015FEA010C8F
S2144506A002BF84460146002043F0B64308BFA3F187
S2144506B08053A3F50003BCFA8CF2083AA3EBC25369
S2144506C010DB01FA02FC634400FA02FCC2F1200288
S2144506D0BCF1004F20FA02F243EB020008BF20F0BF
S2144506E00100704702F1200201FA02FCC2F1200225
S2144506F050EA4C0021FA02F243EB020008BF20EA1A
S214450700DC7070474FF0FF0C1CEAD0521EBF1CEA47
S214450710D15392EA0C0F93EA0C0F6FD01A4480EA35
S214450720010C400218BF5FEA41211ED04FF000631E
S21445073043EA501043EA5111A0FB01310CF000404A
S214450740B1F5000F3EBF490041EAD3715B0040EA70
S214450750010062F17F02FD2A1DD8B3F1004F40EB40
S214450760C25008BF20F00100704790F0000F0CF013
S214450770004C08BF49024CEA502040EA51207F3AD7
S214450780C2BFD2F1FF0340EAC250704740F40000B2
S2144507904FF00003013A5DDC12F1190FDCBF00F0A3
S2144507A000407047C2F10002410021FA02F1C2F151
S2144507B0200200FA02FC5FEA310040F1000053EAED
S2144507C04C0308BF20EADC70704792F0000F00F03B
S2144507D0004C02BF400010F4000F013AF9D040EA41
S2144507E00C0093F0000F01F0004C02BF490011F4D5
S2144507F0000F013BF9D041EA0C018FE70CEAD153D3
S21445080092EA0C0F18BF93EA0C0F0AD030F0004C52
S21445081018BF31F0004CD8D180EA010000F0004006
S214450820704790F0000F17BF90F0004F084691F0C4
S214450830000F91F0004F14D092EA0C0F01D14202FE
S2144508400FD193EA0C0F03D14B0218BF084608D1C7
S21445085080EA010000F0004040F0FE4040F4000011
S214450860704740F0FE4040F4400070474FF0FF0CA4
S2144508701CEAD0521EBF1CEAD15392EA0C0F93EAEB
S2144508800C0F69D0A2EB030280EA010C49024FEA3D
S214450890402037D04FF0805343EA111143EA1013F6
S2144508A00CF000408B4238BF5B0042F17D024FF4AE
S2144508B0000C8B4224BF5B1A40EA0C00B3EB510F89
S2144508C024BFA3EB510340EA5C00B3EB910F24BF72
S2144508D0A3EB910340EA9C00B3EBD10F24BFA3EBF7
S2144508E0D10340EADC001B0118BF5FEA1C1CE0D1BF
S2144508F0FD2A3FF650AF8B4240EBC25008BF20F072
S214450900010070470CF0004C4CEA50207F32C2BFC5
S214450910D2F1FF0340EAC250704740F400004FF062
S2144509200003013A37E792F0000F00F0004C02BF93
S214450930400010F4000F013AF9D040EA0C0093F05D
S214450940000F01F0004C02BF490011F4000F013BB7
S214450950F9D041EA0C0195E70CEAD15392EA0C0F1F
S21445096008D142027FF47DAF93EA0C0F7FF470AF57
S214450970084676E793EA0C0F04D14B023FF44CAF9A
S21445098008466EE730F0004C18BF31F0004CCAD12F
S21445099030F000427FF45CAF31F000437FF43CAF6B
S2144509A05FE700BF4FF0FF3C06E000BF4FF0010C8D
S2144509B002E000BF4FF0010C4DF804CD4FEA40026F
S2144509C04FEA41037FEA226C18BF7FEA236C11D0B9
S2144509D001B052EA530C18BF90EA010F58BFB2EB6C
S2144509E0030088BFC81738BF6FEAE17018BF40F0EC
S2144509F0010070477FEA226C02D15FEA402C05D1A0
S214450A007FEA236CE4D15FEA412CE1D05DF8040B24
S214450A10704700BF844608466146FFE70FB5FFF7B7
S214450A20C9FF002848BF10F1000F0FBD4DF808ED6F
S214450A30FFF7F4FF0CBF012000205DF808FB00BF60
S214450A404DF808EDFFF7EAFF34BF012000205DF8BA
S214450A5008FB00BF4DF808EDFFF7E0FF94BF012007
S214450A6000205DF808FB00BF4DF808EDFFF7D2FF04
S214450A7094BF012000205DF808FB00BF4DF808ED47
S214450A80FFF7C8FF34BF012000205DF808FB00BF14
S214450A9042000ED2B2F1FE4F0BD34FF09E03B3EB9E
S214450AA0126209D44FEA002343F0004323FA02F0CA
S214450AB070474FF00000704712F1610F01D14202B6
S214450AC002D14FF0FF3070474FF00000704700BF2F
S214450AD053B94AB9002908BF00281CBF4FF0FF315B
S214450AE04FF0FF3000F0A6B9ADF1080C6DE904CE25
S214450AF000F03EF8DDF804E0DDE9022304B0704777
S214450B0038B505460C462846214600220023FFF701
S214450B1015FC28B928462146BDE8384000F00AB8F5
S214450B20284604F1004100F005F8404261EB4101DA
S214450B3038BD00BFD0B50C4B002206460F46FFF722
S214450B408BF9FFF761FC0446FFF70CF9074B0022CB
S214450B50FFF782F902460B4630463946FEF7C4FF94
S214450B60FFF752FC2146D0BD0000F03D0000F041A5
S214450B702DE9F047089D0E4604468C46002B40F06E
S214450B8081808A42174645D9B2FA82F24AB1C2F105
S214450B90200106FA02F320FA01F1974041EA030CD8
S214450BA094404FEA174E230CBCFBFEF6B9B20EFB3B
S214450BB016CC43EA0C4306FB01F0984209D9FB18CC
S214450BC006F1FF3C80F01581984240F21281023EC4
S214450BD03B441B1AA4B2B3FBFEF00EFB103344EAAB
S214450BE0034400FB01F1A14209D93C1900F1FF334A
S214450BF080F00181A14240F2FE8002383C44641AEE
S214450C0040EA064000211DB1D4400023C5E9004313
S214450C10BDE8F08702B9FFDEB2FA82F2002A4FD16C
S214450C20CB1B4FEA174E1FFA87F80121B3FBFEFC94
S214450C30260C0EFB1C3346EA034608FB0CF3B34270
S214450C4007D9BE190CF1FF3002D2B34200F2EB8051
S214450C508446F61AA3B2B6FBFEF00EFB106643EAD0
S214450C60064408FB00F8A04507D93C1900F1FF33B8
S214450C7002D2A04500F2D2801846A4EB080440EA0A
S214450C800C40C0E78B4208D9002D00F0AF8000210C
S214450C90C5E900060846BDE8F087B3FA83F10029A2
S214450CA049D1B34202D3824200F2BB80841A66EB36
S214450CB0030301209C46002DAAD0C5E9004CA7E7B2
S214450CC0C2F120039740D8409140DE404FEA174E88
S214450CD008434FEA104CB6FBFEF11FFA87F80EFBA9
S214450CE011664CEA064601FB08F3B34204FA02F4E1
S214450CF009D9BE1901F1FF3C80F08E80B34240F21F
S214450D008B8002393E44F31A86B2B3FBFEF00EFBE7
S214450D10103346EA034600FB08F3B34207D9BE192B
S214450D2000F1FF3C74D2B34272D902383E44F31AFE
S214450D3040EA01417AE7C1F1200703FA01F422FAB5
S214450D4007F31C4320FA07F906FA01F34FEA144C59
S214450D50FE4049EA03094FEA1943B6FBFCFE1FFA73
S214450D6084F80CFB1E6643EA06460EFB08FAB245B7
S214450D7002FA01F200FA01F308D9A6190EF1FF307E
S214450D8048D2B24546D9AEF1020E2644A6EB0A062F
S214450D901FFA89F9B6FBFCF00CFB106649EA0646D5
S214450DA000FB08F8B04507D9A61900F1FF3C2DD23F
S214450DB0B0452BD90238264440EA0E40A6EB080635
S214450DC0A0FB02894E45C446CE4618D315D075B30A
S214450DD0B3EB0C0266EB0E0606FA07F722FA01F3AA
S214450DE0CE401F43C5E90076002111E7294628462F
S214450DF00EE76646EDE6184601E74345E7D2B8EB0B
S214450E00020C69EB04040138A646E0E76046D3E7E2
S214450E1060468CE78646B9E7614674E702383C4447
S214450E202BE7084647E7ACF1020C3E4411E7294656
S214450E30EEE600BF704700BF2DE9F04788B0002BAF
S214450E401F461446B8BF03F10043129A109DDDF8BD
S214450E504CA0B6BF1F4600232D231370149B23F0CA
S214450E602008B8F1460F05D0B8F1450F00D1013539
S214450E70022300E0032307AA049206AACDE902A2AC
S214450E80CDE9003522463B4601F0A6FDB8F1470FB1
S214450E90064602D1119BDB0722D5B8F1460F06EB75
S214450EA0050910D13378302B0AD10022002320467D
S214450EB03946FFF739FA18B9C5F10105CAF80050A1
S214450EC0DAF8003099440022002320463946FFF7D9
S214450ED02BFA08B1CDF81C903022079B4B4507D31B
S214450EE0079B159A9B1B3046136008B0BDE8F087F4
S214450EF0591C07911A70F0E7F7B503460029B8BFA5
S214450F00494203F8022BB4BF2D222B2209294270F1
S214450F102ADD0DF10704A4460A27A6460A4691FB94
S214450F20F7F607FB16153035632A04F1FF340EF83D
S214450F30015C3146F1DC3031AEF1020504F8011CA6
S214450F40441C294661450AD30DF10902A2EB0E025F
S214450F50654588BF00221344181A03B0F0BD11F842
S214450F60012B04F8012FEDE7302330318370C17033
S214450F70031DF1E72DE9F04F91B00C46DDF868808A
S214450F8016461F46054602F04DFE03680993184669
S214450F90FEF748FD00230E93D8F800300A90073335
S214450FA023F0070303F1080294F81890D4F800B02C
S214450FB0C8F80020D3E90023C4E91223D4E9128AED
S214450FC02AF000430B930B999C4B4FF0FF3240465B
S214450FD0FFF7DCF970BB994B0B994FF0FF32404653
S214450FE0FFF7B6F930BB0022002340465146FFF7CF
S214450FF0A5F910B12D2384F84330914B9148B9F1AA
S214451000470F94BF98468046032323612BF004037D
S21445101023604FF0000A009733460FAA214628461C
S21445102000F0D2F9013040F08F804FF0FF3011B01C
S214451030BDE8F08F4246534640465146FFF7A6F96F
S21445104040B1BAF1000FBCBF2D2384F843307E482B
S2144510507E4BD4E763685A1C09F0DF0142D106236C
S2144510606360002206920EAACDE904920DAA4BF4BF
S214451070806303920DF13302CDE901322360636844
S21445108000934246534628460B91FFF7D5FE0B99EB
S214451090472980460D9908D1C81C02DB63689942EA
S2144510A040DDA9F102095FFA89F9B9F1650F1FD844
S2144510B001394A4604F150000D91FFF71DFF0E9A7F
S2144510C01318012A8246236102DC2268D20701D51D
S2144510D0013323619DF83330002B9CD02D2384F8B3
S2144510E0433098E74729BCD1002BBAD10123B7E74F
S2144510F0B9F1660F18D1002963680BDD216113B974
S2144511002268D00702D501330B442361A1654FF011
S214451110000ADFE713B92268D20701D50233F4E7A0
S2144511200123F2E74FF067090E9B994205DB2368DA
S2144511302161D807EAD54B1CE7E70029D4BFC1F1A2
S214451140020201221344E0E723685A0507D42369BF
S214451150424631462846B84701302BD165E7B9F1B6
S214451160650F40F2DC80D4E9120100220023FFF728
S214451170DBF8002833D0364A012331462846B8479F
S21445118001303FF452AFDDE90D239A4202DB236876
S214451190D8070FD5DDE9092331462846B84701303B
S2144511A03FF443AF4FF0000804F11A090E9B013B8C
S2144511B0434509DC23689B0700F10181E0680F9BE6
S2144511C09842B8BF184632E701234A463146284674
S2144511D0B84701303FF429AF08F10108E6E70D9B13
S2144511E0002B37DC1A4A012331462846B8470130DA
S2144511F03FF41BAFDDE90D23134302D12368D9071E
S214451200D8D5DDE9092331462846B84701303FF4AD
S2144512100CAF4FF0000904F11A0A0D9B5B424B4593
S21445122001DC0E9B94E70123524631462846B847D3
S21445123001303FF4FAAE09F10109EEE7FFFFEF7F13
S214451240D6944600DA944600E2944600DE9446007C
S214451250E69446000E9AA36D9A42A8BF1A46002AFF
S214451260914637DC4FF0000B29EAE97904F11A027A
S214451270D4F858A0AAEB09035B4533DCDDE90D231A
S2144512809A423BDB2368DA0738D40E9A0D99A2EBCF
S2144512900A03A2EB01099945A8BF9946B9F1000F83
S2144512A034DC4FF0000829EAE97904F11A0ADDE949
S2144512B00D239B1AA3EB090343457FF77BAF012319
S2144512C0524631462846B84701303FF4AEAE08F19F
S2144512D00108ECE71346314642462846B8470130F2
S2144512E0C0D1A2E60123314628460B92B8470130C5
S2144512F03FF49BAE0B9A0BF1010BB9E7DDE90923E9
S21445130031462846B8470130BFD18EE64B4608EBF6
S2144513100A0231462846B8470130C2D185E60E9ABC
S214451320012A01DCDB0737D50123424631462846EC
S214451330B84701303FF479AEDDE909233146284602
S214451340B84701303FF471AED4E9120100220023BC
S214451350FEF7EAFFD8B90E9B08F10102013B31467C
S2144513602846B84701300ED15FE601234A46314646
S2144513702846B84701303FF458AE08F101080E9BA1
S214451380013B4345F1DC534604F15002E1E64FF09C
S214451390000804F11A09F2E701234246DFE7012374
S2144513A04A4631462846B84701303FF43EAE08F136
S2144513B00108E3680F995B1A4345F0DCFEE64FF0FB
S2144513C0000804F11909F4E72DE9F0471646994651
S2144513D08A680B69DDF820809342B8BF13463360B0
S2144513E091F8432007460C460AB10133336023681B
S2144513F0990642BF336802333360256815F0060503
S21445140006D104F1190AE36832689B1AAB4226DC1A
S21445141094F84320131E226818BF012392062BD446
S21445142004F1430249463846C04701301ED023687A
S214451430E568326803F00603042B08BFAD1AA368B7
S21445144022690CBF25EAE57500259342C4BF9B1A61
S214451450ED1800261A34B5421AD1002008E00123BB
S214451460524649463846C047013003D14FF0FF3013
S214451470BDE8F0870135C6E7E1185A1C302081F8EB
S2144514804300224494F8451082F843100233C7E7D8
S2144514900123224649463846C0470130E6D0013644
S2144514A0D9E700002DE9FF470C469146277E0C9963
S2144514B0782F80469A4604F1430207D8622F0AD809
S2144514C0002F00F0D880582F00F0A38004F1420684
S2144514D084F842703AE0A7F16303152BF6D801A0CD
S2144514E050F823F03D15450051154500CD144500EF
S2144514F0CD144500CD144500CD1445005115450085
S214451500CD144500CD144500CD144500CD144500F9
S2144515105D164500811545003F164500CD1445002E
S214451520CD1445007F164500CD1445008115450070
S214451530CD144500CD144500471645000B681A1DC9
S2144515401B680A6004F1420684F842300123A3E092
S214451550256808682E0600F104030AD505680B6061
S214451560002D03DA2D236D4284F843305E480A2366
S21445157019E015F0400F05680B6018BF2DB2EFE770
S2144515800B682568181D0860280601D51D6802E009
S2144515906906FBD51D8854486F2F0CBF08230A23C0
S2144515A0002184F843106668A660002EA2BF216815
S2144515B021F0040121600DB9002E4DD01646B5FB2D
S2144515C0F3F103FB1157C75D06F8017D2F46BB4275
S2144515D00D46F4D9082B0BD12368DF0708D52369B8
S2144515E061689942DEBF302306F8013C06F1FF36B6
S2144515F0921B2261CDF800A04B4603AA21464046E1
S214451600FFF7E2FE01304CD14FF0FF3004B0BDE8A5
S214451610F087354884F8457023680E681F0656F8E7
S214451620045B0E6014D5D90744BF43F020032360FE
S2144516301DB9236823F0200323601023B0E72368F1
S21445164043F0200323607823284884F84530E3E7B1
S2144516505E0648BFADB2E6E71646BBE70B682668AA
S21445166060691D1D0D6035061B6801D5186002E0D2
S2144516707106FBD51880002323611646BAE70B682A
S2144516801A1D0A601E68626800213046FEF7D8F9C2
S21445169008B1801B606063682361002384F843308B
S2144516A0A8E72369324649464046D0470130ABD085
S2144516B023689B0713D4E068039B9842B8BF184637
S2144516C0A4E70123324649464046D04701309BD0E1
S2144516D00135E36803995B1AAB42F2DCEBE700257C
S2144516E004F11906F5E700BFE8944600F99446006C
S2144516F02DE9F04F87B0174603938B685A1EB2F50F
S214451700AE7F83BF6FF4AE755B190293002386BF29
S21445171040F25D138B6002930B688B46002543F4BD
S214451720F0634BF81C3BCDE9045580460C465E46B7
S214451730AA46A9460195A26852B13B681B784E2B2E
S21445174064D8402B3CD8A3F12B01C8B20E283AD911
S214451750B9F1000F03D0236823F4807323600AF1A0
S214451760FF3ABAF1010F00F213815E4500F205819A
S2144517700125284607B0BDE8F08FA3F161020D2A82
S214451780E6D801A151F822F0C71845005117450083
S214451790511745005117450027194500FF184500C4
S2144517A05117450051174500D518450051174500B6
S2144517B05117450051174500511745008D184500EE
S2144517C0A3F14102DBE70E29C2D801A050F821F06B
S2144517D07F184500511745007F18450013194500E9
S2144517E0511745002D1845006918450069184500EC
S2144517F06918450069184500691845006918450087
S2144518006918450069184500691845006E2B09D8C2
S214451810602BB2D8542B77D0592B99D1072D97D119
S214451820082529E0742B6FD0792BF6E72168C80583
S2144518301AD5029B21F08001216009F101091BB1EF
S214451840013B01320293A260A368013BA360236972
S214451850013323617B68013B002B7B6040F384802A
S2144518603B6801333B6066E71AEB050F7FF470AFC4
S214451870226822F4C072226006F8013BE4E722683B
S21445188010067FF565AF22F08002F4E7BAF1000F47
S2144518900ED1B9F1000F0ED1226802F4E061B1F520
S2144518A0E06F08D122F4F06222604FF0010AE3E7C8
S2144518B0BAF1020F55D0012D02D0042D7FF448AF62
S2144518C00135EDB2D8E7BAF1010F7FF441AF4FF0DD
S2144518D0020AD1E77DB9B9F1000F7FF43CAF226823
S2144518E002F4E061B1F5E06F7FF439AF22F4F062BF
S2144518F022600125C0E7032DE2D0052DDEE7022D47
S2144519007FF426AF0325B7E7062D7FF421AF0725DD
S214451910B2E7226891057FF51BAF22F4207222605C
S214451920CDF80490A8E7226802F4A061B1F5806F6F
S21445193006D050057FF50CAFB9F1000F3FF40FAF59
S214451940910558BF019922F4F06258BFA9EB0101F1
S21445195042F4C07258BFCDE9041622604FF0000924
S2144519608AE74FF0030A87E7D4F880313946404680
S214451970984700283FF4DFAEEAE6D4F87C3116F8FF
S214451980011D3A46404698472369013B2361ECE6EC
S2144519906B1E062B25D8022D36D85E457FF6E8AE5B
S2144519A0D4F87C3116F8011D3A46404698472369D7
S2144519B0013B2361F1E70298D4F87C3110F8011D0C
S2144519C002903A46404698472369013B23610AF10F
S2144519D0FF3A5FFA8AFABAF1020FECD1033DEDB24F
S2144519E0761B2368DA052FD55B0510D55E457FF651
S2144519F0BFAED4F87C3116F8011D3A4640469847A6
S214451A002369013B2361F1E7AA460296DFE716F80C
S214451A10011C2369652903F1FF3306F1FF35236170
S214451A200CD045290AD0D4F87C313A4640469847EA
S214451A30236916F8021C013BB51E2361D4F87C3198
S214451A403A46404698472E46256815F0100559D122
S214451A503570236803F4C063B3F5806F1CD1019BD2
S214451A604B45A3EB090224D100225946404600F0D7
S214451A7083FED4F800C0039B1CF0020F1B68064685
S214451A800F4621D003991A1D0A601B68C3E90067F3
S214451A90E3680133E3606CE6049B002BE4D00599CC
S214451AA00A232A460131404600F0E6FE049B059E81
S214451AB0C21A04F26F139E4228BF04F5B776124940
S214451AC0304600F029F8CFE71CF0040F03F1040E6A
S214451AD003D00399C1F800E0D7E7039AC2F800E0BF
S214451AE0D3F8008002460B46FEF750FC28B107485F
S214451AF000F00EF8C8F80000CAE730463946FEF74B
S214451B00A3FCF7E7002534E60A954600F48F460021
S214451B10004870470000C07F0EB400B59AB01BABB6
S214451B20019005906FF000410948069103910949D7
S214451B3053F8042B04910068009301A902F0E4FDD4
S214451B40019B00221A701AB05DF804EB03B070478B
S214451B50282340200802FFFF2DE9F0410F46904616
S214451B6002F084FB04460D46B8F1000F11D0C7F3CA
S214451B700A53C3F16B03002B0BDD1B0503F17F55A1
S214451B80002405F5401522462B46FEF765F9044622
S214451B900D4620462946BDE8F081000000000000BD
S214451BA02DE9F04FA1B09B4600231C939E4B179200
S214451BB01F68824638460E46FDF734FF4FF000084C
S214451BC004464FF000091B961B9B1A782B2A4CD0CF
S214451BD03AD80D2A33D8082A33D8002A3DD00023D0
S214451BE00C931B9D2B78302B40F0A9806B7803F027
S214451BF0DF03582B66D10C9B01931CAB00938B4A95
S214451C00CDF808B01DAB1BA9504601F01FFD10F0DE
S214451C100706044605D0062E29D1013500231B9517
S214451C200C93179B002B40F08E850C9BD3B14246F8
S214451C3009F100431046194621B0BDE8F08F202A29
S214451C40CDD101331B93BFE72D2AC8D101220C9273
S214451C505A1C1B925B78002BC3D1179B1B96002BF7
S214451C6040F06F8542464B46E4E70022EFE71C9A74
S214451C703AB135211EA802F0F0FB1C99504602F0F9
S214451C8031F8013E042E06D8DFE806F00A0314179D
S214451C900A00DDE91E892107C3D549F00049C0E79A
S214451CA0DDE91E831D9A23F4801302F2334243EA8C
S214451CB00259F0E7DFF87891EDE76FF000494FF00D
S214451CC0FF38E8E71B9B5A1C1B925B78302BF9D0F4
S214451CD0002BA6D0012307931B9B08930023CDE931
S214451CE005339B460A221B980578A5F13003D9B2E1
S214451CF0092926D92246394602F01CFE002832D04C
S214451D0000202B465C4604900246652B01D0452BA9
S214451D1013D11CB9079B03439FD000241B9E731CFD
S214451D201B9373782B2B78D02D2B7BD00027A3F1D4
S214451D303001092940F282801B9600259EE000234B
S214451D40C9E7BBF1080FD5BF0699059902FB0133D4
S214451D5002FB013300F10100D4BF069305930BF156
S214451D60010B1B90BFE71B9B1A191B921B5DBBF112
S214451D70000F36D004905C46A3F13002092A12D9EA
S214451D800122C2E71B9B5A1C1B925B780130302B05
S214451D90F8D0A3F13102082A00F2DA841B9A04909F
S214451DA0002008920446303B00F1010213D0049906
S214451DB011440491224605190A21954213D1221849
S214451DC0082A04F1010404441BDC06990A2202FB96
S214451DD00133069300221B9B591C1B915B781046CA
S214451DE0CAE75846D3E7082A04DC069F4F430697BA
S214451DF00132E2E7571C102FDEBF059F4F4305977C
S214451E00F6E7102CDFBF05990A2202FB013305933E
S214451E10E0E70023049301227CE70027B31C1B93CD
S214451E20B37884E70127F9E7709646001095460093
S214451E300000F07F1B9B591C1B915B78302BF9D01B
S214451E40A3F1310108293FF678AFA3F1300C1B9B6F
S214451E5009934FF00A0E1B9B591C1B915B78A3F107
S214451E603005092D35D9099D491B082944F61F65B6
S214451E7002DC6545A8BF654607B16D42002C4CD1CE
S214451E80079901437FF4CDAE002A7FF4E6AE692B71
S214451E9026D023DC492B23D04E2B7FF4DEAE9C493F
S214451EA01BA801F00FFE00283FF4D7AE1B9B1B78FE
S214451EB0282B2CD197491EAA1BA801F017FE0528EA
S214451EC025D11F9BDDF8788043F0FF4949F4E009AA
S214451ED0A7E60EFB0C3CACF1300CBCE76E2BDCE702
S214451EE08D491BA801F0EEFD00283FF4B6AE1B9BBE
S214451EF08A49013B1BA81B9301F0E4FD10B91B9BC7
S214451F0001331B93DFF824924FF0000889E6844896
S214451F1002F00AFD8046894683E6049B0698EB1A3E
S214451F20BBF1000F08BFA346102C07932646A8BF53
S214451F301026FDF717FF092C8046894613DD794B99
S214451F4003EBC60353E91223FDF786FF8046059843
S214451F508946FDF707FF02460B4640464946FDF7CC
S214451F60C5FD804689460F2C36DC079B002B3FF483
S214451F7058AE22DD162B09DC6A4C04EBC304D4E9C3
S214451F80000142464B46FDF767FFC3E7079AC4F193
S214451F902503934220DB634DC4F10F0405EBC401D2
S214451FA042464B46D1E90001FDF756FF079B1C1BF1
S214451FB005EBC405D5E90023E5E7079B16330BDBA0
S214451FC0049B584A5D1B02EBC505D5E900234046F0
S214451FD04946FEF76BF89DE7079BA61B1E44002E59
S214451FE071DD16F00F030AD04E4901EBC301424698
S214451FF04B46D1E90001FDF72FFF8046894636F06E
S2144520000F0650D0B6F59A7F27DD4FF0000BCDF87A
S21445201010B0CDF820B0CDF818B02223DFF80C91DB
S214452020CAF800304FF00008089B002B3FF4F9AD86
S2144520301C99504601F056FE0699504601F052FE50
S2144520400499504601F04EFE0899504601F04AFE66
S2144520505946504601F046FEE3E500233611404614
S21445206049461F46012E21DC0BB1804689462E4B3C
S214452070A9F1547903EBC70742464B46D7E9000119
S214452080FDF7EAFE294B0A460B4029498B42804616
S214452090BBD8A1F580118B4286BFDFF898904FF0EC
S2144520A0FF3802F15479002305937EE0F20707D501
S2144520B01D4B03EBC703D3E90023FDF7CDFE0123F4
S2144520C001377610CEE7EED0764216F00F020AD0EC
S2144520D0144B03EBC20340464946D3E90023FDF7BC
S2144520E0E5FF804689463611DDD01F2E24DD4FF0AC
S2144520F0000BCDF810B0CDF820B0CDF818B022239F
S2144521004FF000084FF00009CAF800308CE700BFD2
S214452110E394460024954600DB94460064964600C4
S214452120F48F4600B0964600889646000000F07F3D
S2144521300000A07CFFFFEF7F16F0100318BF6A2350
S214452140B34F0593404649460023F20704D5D7E9E1
S2144521500023FDF781FE0123761007F10807F4D129
S2144521600BB180468946059BBBB1C9F30A53C3F1FB
S2144521706B03002B494610DD1F2B40F32881342B7B
S214452180DEBF203B4FF0FF3202FA03F34FF0000864
S214452190CCBF4FF05C7903EA010900220023404694
S2144521A04946FEF7C1F80028A1D1069B0093089939
S2144521B023465A46504601F0EAFD089000283FF46B
S2144521C024AF049B5D1B079B002BB4BF2B46002307
S2144521D00E93079B4FF0000B23EAE3731693CDF857
S2144521E010B0089B5046596801F048FD06900028F7
S2144521F03FF413AF089B1A69023203F10C019200B3
S2144522000C3001F02DFD1EAB01931DAB00934246ED
S2144522104B465046CDE90A8902F0A2F81C900028A4
S2144522203FF4FBAE0121504601F03DFE04900346C7
S21445223000283FF4F2AE1D9D1E9A002DABBF0E9BA7
S214452240169B169C0E9EACBFEE185C1B059BED1AA6
S2144522501544704B013D9D42C2F1360280F2C9805D
S2144522605B1B1F2BA2EB03024FF0010700F3B68062
S21445227007FA03F30F930025B718059BBE4214448F
S2144522801C443346A8BF3B46A342A8BF2346002B63
S214452290C2BFFF1AE41AF61A0E9B002B17DD0499E7
S2144522A01A46504601F0A4FE049000283FF4B5AE09
S2144522B001461C9A504601F0FFFD099000283FF460
S2144522C0ACAE1C99504601F00DFD099B1C93002FA2
S2144522D000F39380079B002B08DD169A0699504617
S2144522E001F086FE069000283FF497AE002C08DDE8
S2144522F006992246504601F0C9FE069000283FF44E
S2144523008CAE002E08DD04993246504601F0BEFEDE
S214452310049000283FF481AE069A1C99504601F079
S2144523202FFF834600283FF478AE0024C3680499FF
S214452330C4600D9301F009FFA04271DA0D9B53EA84
S214452340080340F09780C9F31303002B40F09280B2
S21445235029F000431B0D1B05B3F1D66F40F28A806A
S214452360DBF8143023B9DBF81030012B40F38280BC
S21445237059460122504601F089FE0499834601F0EC
S214452380E4FE002876DD0599234A4B46002900F0F1
S214452390928002EA0901B1F1D66F00F38C80B1F163
S2144523A05C7F7FF7ACAE1D4A0023CDE9143240462C
S2144523B0DDE914234946FDF74FFD0B46034308BFA9
S2144523C022238046894608BFCAF8003030E64FF0DB
S2144523D0FF3202FA03F303EA0808DEE6C5F17F4555
S2144523E005F57F0505F57B45E23507FA05F50F97B3
S2144523F042E7012300250F933EE71C993A4650468F
S21445240001F044FE1C9000287FF464AF05E600BF4B
S2144524103895460002FCFFFF0000F07F000050396B
S214452420CDF8249066D10D9AC9F313035AB39C4A46
S21445243093422CD1059B404603B39A4A4B461A40D5
S214452440B2F1D46F4FF0FF311BD8120DC2F16B03BA
S21445245001FA03F398421AD1934B099A9A4202D14C
S21445246001303FF4DAAD8F4B099A1A4002F58019D0
S2144524704FF00008059B002B95D1D9E54FF0FF336B
S214452480E8E70B46E6E753EA08033FF47CAFE5B1D9
S214452490099B1D42EED00D9B059A40464946C3B161
S2144524A0FFF75AFB02460B46DDE90A01FDF71EFB20
S2144524B080468946DEE71340A3F580136FEA135935
S2144524C06FEA09594FF0FF38D4E70F9B13EA080F18
S2144524D0E0E7FFF741FB02460B46DDE90A01FDF75B
S2144524E003FB0022002380468946FDF71DFF002892
S2144524F0C0D004E60499584601F081FF00224FF00B
S214452500804306460F46FDF723FF002875D00D9BF2
S214452510002B47D0654F0026644D099B23F00043AA
S2144525201B0D1B050F930F9A614B9A4240F0C880CE
S214452530DDE90A23CDE91423099BA3F154794046E6
S214452540494601F093FE02460B4630463946FDF7AE
S21445255083FC42464B46FDF7C9FA0B465149554A58
S2144525601940914280465ED90B9B02F154729342C4
S21445257003D10A9B01333FF450ADDFF82C914FF061
S214452580FF381C99504601F0ADFB0699504601F0C0
S214452590A9FB0499504601F0A5FB5946504601F063
S2144525A0A1FB1EE6B8F1000F19D1099BC3F313032F
S2144525B0E3B93E4B002230463946FDF7BFFEC8B963
S2144525C03D4B002230463946FDF746FC04460D464F
S2144525D005F1004318941993DDE918679DE7B8F1AE
S2144525E0010F03D1099B002B3FF489AD334F0026DD
S2144525F0002491E70D9C304DEAE72F4B00223046EC
S2144526003946FDF729FC0D9B04460D4633B901F1C5
S214452610004310901193DDE910677EE702460B46AE
S214452620CDE91023F7E703F15479059B002BA8D194
S21445263029F000430F9A1B0D1B059A42A1D120464F
S2144526402946FEF75DFAFDF7D9FB02460B462046BE
S2144526502946FDF749FA0D9AC9F3130343EA0803D9
S214452660134304460D4666D009A3D3E90023FDF778
S21445267065FE00287FF4DCAC07A3D3E9002320469B
S2144526802946FDF779FE00283FF47BAFD0E400BF2E
S2144526909535A094FFFFDF3F35E5AF350000E03FB9
S2144526A0FFFF0F000000F07FFFFFEF7F0000F03FC9
S2144526B00000E07FFFFF9F7C0000E03F0000F0BF8A
S2144526C0059B13B30F9BB3F1D46F1ED826A3D3E94E
S2144526D0002320462946FDF73BFE90B12946204675
S2144526E0FDF792FE012838BF0120FDF73BFB0D9B09
S2144526F004460D46D3B901F1004312901393DDE924
S21445270012670F9A07F1D6639F1ADDE90A0101F0B1
S214452710ADFD02460B4630463946FDF79DFBDDE9E5
S2144527200A23FDF7E3F9804689467EE702460B46CF
S214452730CDE91223E3E70EA3D3E90023FDF7FEFD1B
S214452740A1E700230C93179A1B9B1360FFF76DBAFE
S214452750652B3FF45EAB452B3FF45BAB0122FFF7A1
S2144527608FBB00BFAFF300800000C0FFFFFFDF4117
S2144527709535A094FFFFCF3F014BFFF711BA00BF39
S214452780902340202DE9F0473A4E86468C466046D3
S2144527901CF8014BA55D15F00805F8D12D2C33D155
S2144527A09CF800404FF0010800F1020C002B5CD06D
S2144527B0102B0CD1302C0AD19CF8000000F0DF001D
S2144527C058284DD19CF8014010230CF1020C08F115
S2144527D00047013F0026B7FBF3F9304603FB197A5D
S2144527E0A4F13005092D18D82C46A34224DD751CC6
S2144527F007D081451DD301D1A2451ADB00FB034016
S21445280001261CF8014BEBE72B2C08BF9CF8004033
S214452810A84608BF00F1020CC8E7A4F14105192DEA
S21445282001D8373CE1E7A4F16105192D04D8573C9A
S214452830DBE74FF0FF36E4E7731C06D12223CEF8DC
S2144528400030384642B9BDE8F087B8F1000F00D0F1
S2144528504042002AF7D00EB10CF1FF311160F2E785
